:100000000C941A2B0D9486130D945B130D943013DE
:100010000D9405130D94DA120D94AF120D94841201
:100020000C94B6CF0C944B2B0C944B2B0C944B2B69
:100030000C944B2B0C94EED40C944B2B0C944B2B1C
:100040000C944B2B0C9435C80C944B2B0C944B2BD1
:100050000C944B2B0C944B2B0C9495C60D94B11314
:100060000C944B2B0C94FCCE0C944B2B0C944B2BE4
:100070000C944B2B0C944B2B0C944B2B0C944B2B28
:100080000C944B2B0C944B2B0C944B2B0C944B2B18
:100090000C944B2B0C944B2B0C944B2B0C944B2B08
:1000A0000C944B2B0C944B2B0C944B2B0C944B2BF8
:1000B0000C944B2B0C944B2B0C944B2B0C944B2BE8
:1000C0000C944B2B0C944B2B0C944B2B0C944B2BD8
:1000D0000C944B2B0C944B2B0C944B2B0C944B2BC8
:1000E0000C944B2BC1AFC1AFC8AFC8AFC8AFCFAF37
:1000F000CFAFCFAFDCAFD6AFD6AFD6AF3CC541C5E3
:1001000046C550C55AC5D3C564C56CC574C57EC542
:1001100088C592C5A1C5ABC5D3C5B5C5BFC5C9C541
:1001200030CF36CF47CF52CF5ACF6FCF5ECF6FCFC2
:1001300062CF66CF6FCF6CCFDA00E000EA00DE005E
:10014000FC000001F000D600DC00FA00EC00F60034
:10015000E200EE000001F200D800FE00084AD73BA2
:100160003BCE016E84BCBFFDC12F3D6C74319ABD86
:1001700056833DDA3D00C77F11BED9E4BB4C3E91AA
:100180006BAAAABE000000803F05A84CCDB2D44E99
:10019000B93836A9020C50B9918688083CA6AAAA9B
:1001A0002ABE000000803F000D9441150D945000C0
:1001B0000D9476000D9445000D9456000D943B006F
:1001C0000D9448000D9468000D94FB130D94EE0EF1
:1001D0000D9429000D9437000D945E000D946C0071
:1001E0000D944C000D9472000D94E3100D94640076
:1001F0000D942B000D945A000D9441000D947A003B
:100200000D947F0047322F47332062616420706174
:1002100072616D65746572730A00205A3A2000207D
:10022000593A200042656420583A20004C756C7A97
:10023000426F742054415A20372072656164792ED0
:1002400000526573756D696E67207072696E740017
:10025000436C69636B20746F20726573756D652ED6
:100260002E2E004E6F206D6F76652E00456E642039
:1002700066696C65206C6973740A00426567696E13
:100280002066696C65206C6973740A004D313235E3
:10029000005344207072696E74696E6720627974CD
:1002A0006520004E6F74205344207072696E74692B
:1002B0006E670A0046696C652064656C65746564E8
:1002C0003A0044656C6574696F6E206661696C659F
:1002D000642C2046696C653A20006F70656E20665C
:1002E00061696C65642C2046696C653A20000001E8
:1002F00025301D0C1824311C0B17232F1B0A1EFF41
:10030000040308060202222B1A4142033809FF3671
:1003100028294527444350726F74656374656420CF
:1003200050696E0A006D0046696C616D656E7420DF
:10033000757365643A200053746174733A20002C1D
:10034000204C6F6E67657374206A6F623A200054A8
:100350006F74616C2074696D653A20005374617428
:10036000733A20002C204661696C65643A20002CA9
:100370002046696E69736865643A20005072696E40
:1003800074733A200053746174733A200045787492
:100390007275646572202573004C756C7A426F74B7
:1003A0002054415A20372072656164792E00436FD2
:1003B0006F6C696E6720646F6E652E0048656174AE
:1003C000696E6720646F6E652E0020573A0045788D
:1003D000747275646572202573004C756C7A426F77
:1003E000742054415A20372072656164792E00428E
:1003F000656420646F6E652E0020573A0042656484
:100400002068656174696E672E0042656420636FC1
:100410006F6C696E672E004C756C7A426F74205455
:10042000415A2037204F66662E007A5F6D61783A18
:1004300020007A5F6D696E3A2000795F6D61783ACD
:100440002000795F6D696E3A2000785F6D61783ABF
:100450002000785F6D696E3A20005265706F72748B
:10046000696E6720656E6473746F70207374617455
:1004700075730A0053657474696E672054726176EF
:10048000656C20416363656C65726174696F6E3A77
:10049000200053657474696E6720526574726163DD
:1004A0007420416363656C65726174696F6E3A2094
:1004B0000053657474696E67205072696E742041D0
:1004C0006363656C65726174696F6E3A2000536591
:1004D0007474696E67205072696E7420616E642056
:1004E00054726176656C20416363656C65726174FA
:1004F000696F6E3A200020643A0020693A0020704B
:100500003A0043290A0061626C656420286D696EB7
:100510002074656D702000436F6C64206578747280
:1005200075646573206172652000426564204C65C6
:1005300076656C696E6720004661696C656420743D
:100540006F20656E61626C6520426564204C657643
:10055000656C696E670A00426564204C6576656C5F
:1005600020436F7272656374696F6E204D6174729F
:1005700069783A003A20007A5F6D696E3A20202D42
:1005800032207A5F6D61783A202035005A204F661C
:1005900066736574200041637469766520457874DC
:1005A00072756465723A2000556E6B6E6F776E20BF
:1005B000636F6D6D616E643A20220020204E6F7A69
:1005C0007A6C653A2000200066696C616D656E7416
:1005D00020756E6C6F6164005761697420666F727C
:1005E000005052494E54205041555345440020205C
:1005F0004E6F7A7A6C653A20006368616E676500B9
:100600006F66207468652066696C616D656E740044
:100610005761697420666F72207374617274005040
:1006200052494E54205041555345440020204E6FAE
:100630007A7A6C653A200020004261636B004D6954
:100640006E696D756D2054656D702069732031324F
:10065000302E0048656174696E67206661696C655B
:10066000640025753A2530327500253032753A25FB
:100670003032750025756420253032753A253032C8
:10068000750000060900FE000000000001090008D6
:10069000FE000005080806000040F0C88888987829
:1006A00010050808060000C0F88888888888F805C2
:1006B00005050600012030F8302005080806000076
:1006C0002070F820202020E00509090600FF207096
:1006D000A8A8B8888870200509090600FFE080C036
:1006E000B0A8283028280509090600FFF8A888883E
:1006F000888888A8F8050A0A0600FE205050505045
:1007000088A8A8887003030306000340A0400006E1
:100710000900FE070192032120FFFF08FF07FF00E9
:10072000000006000001070706020080808080802C
:100730000080030202060105A0A0050707060000CD
:100740005050F850F850500507070600002078A0D8
:100750007028F020050707060000C0C81020409848
:10076000180507070600006090A040A890680203E3
:1007700003060104C04080030707060100204080F3
:100780008080402003070706010080402020204091
:100790008005050506000120A870A82005050506AE
:1007A00000012020F820200203030602FFC0408041
:1007B000050101060003F8020202060200C0C0059E
:1007C0000505060001081020408005070706000007
:1007D0007088888888887003070706010040C04039
:1007E000404040E0050707060000708808708080E0
:1007F000F8050707060000F81020100808F00507A4
:100800000706000010305090F8101005070706008A
:1008100000F880F00808887005070706000070805F
:1008200080F0888870050707060000F8081020206F
:1008300020200507070600007088887088887005EA
:10084000070706000070888878080870020505060A
:100850000200C0C000C0C00206060602FFC0C00001
:10086000C040800407070600001020408040201090
:10087000050303060002F800F804070706010080DC
:1008800040201020408005070706000070880810EF
:1008900020002005070706000070880868A8A870D7
:1008A000050707060000708888F88888880507070C
:1008B000060000F08888F08888F005070706000029
:1008C00070888080808870050707060000F088889F
:1008D000888888F0050707060000F88080F080808F
:1008E000F8050707060000F88080F0808080050783
:1008F00007060000708880B8888870050707060022
:1009000000888888F88888880107070602008080A8
:1009100080808080800507070600003810101010C6
:1009200090600507070600008890A0C0A090880589
:100930000707060000808080808080F80507070692
:10094000000088D8A88888888805070706000088DE
:1009500088C8A898888805070706000070888888D6
:10096000888870050707060000F08888F08080807E
:1009700005070706000070888888A89068050707A3
:10098000060000F08888F0A09088050707060000A0
:10099000788080700808F0050707060000F820201E
:1009A000202020200507070600008888888888887E
:1009B000700507070600008888888888502005078A
:1009C000070600008888888888A850050707060061
:1009D000008888502050888805070706000088880E
:1009E0008850202020050707060000F80810204046
:1009F00080F8030707060100E08080808080E00522
:100A000005050600018040201008030707060100C5
:100A1000E02020202020E005030306000420508869
:100A2000050101060000F8020202060205804005E9
:100A3000050506000070087888780507070600009D
:100A40008080B0C88888F0050505060000708080A9
:100A500088700507070600000808689888887805E8
:100A600005050600007088F880700507070600007D
:100A70003048E0404040400506060600FF70888888
:100A80007808700507070600008080B0C88888884D
:100A9000010707060200800080808080800308082C
:100AA0000601FF200020202020A0400407070600A8
:100AB00000808090A0C0A090030707060100C040FE
:100AC00040404040E0050505060000D0A8A8A8A8C1
:100AD000050505060000B0C88888880505050600DC
:100AE0000070888888700506060600FFF08888F088
:100AF00080800506060600FF7888887808080505C6
:100B000005060000B0C8808080050505060000705D
:100B1000807008F00407070600004040E0404040B5
:100B200030050505060000888888986805050506D3
:100B3000000088888850200505050600008888A8E0
:100B4000A8500505050600008850205088050606B7
:100B50000600FF888888780870050505060000F8FB
:100B6000102040F803070706010020404080404065
:100B700020010707060200808080808080800307B4
:100B80000706010080404020404080050202060028
:100B9000026890000000060000000000060000004F
:100BA0000000060000000000060000000000060033
:100BB0000000000006000000000006000000000029
:100BC0000600000000000600000000000600000013
:100BD0000000060000000000060000000000060003
:100BE00000000000060000000000060000000000F9
:100BF00006000000000006000000000006000000E3
:100C000000000600000000000600000000000600D2
:100C100000000000060000000000060000000000C8
:100C200006000000000006000000000006000000B2
:100C300000000600000000000600000000000600A2
:100C40000000000006000000000006000000000098
:100C50000600000000000600000000000600000181
:100C60000707060200800080808080800507070655
:100C700000002070A8A0A87020050707060000301B
:100C80004040E04050A805050506000088705070FF
:100C900088050707060000885020F820F820010783
:100CA000070602008080800080808005080806001A
:100CB000003048205050209060030101060107A039
:100CC000050707060000F888B8B8B888F8050707D0
:100CD000060001700878887800F80505050600010F
:100CE0002850A05028050303060001F80808020256
:100CF000020602064080050707060000F888A8885B
:100D000098A8F8050101060006F80404040600038B
:100D1000609090600507070600002020F820200062
:100D2000F804050506000360902040F00305050661
:100D30000003E020E020E0020202060206408005F7
:100D400008080600FF8888888898E88080050707DB
:100D50000600007898987818181802020206020215
:100D6000C0C00202020602FF408003050506000320
:100D700040C04040E0050707060001708888887081
:100D800000F8050505060001A0502850A00507073A
:100D90000600008890A858B8080805070706000054
:100DA0008890B848982038050808060000C040C060
:100DB00048D83808080507070600002000204080B2
:100DC00088700508080600004020007088F88888B0
:100DD0000508080600001020007088F888880508BB
:100DE000080600002050007088F88888050808066A
:100DF00000006890007088F88888050808060000E0
:100E00005000708888F8888805080806000020507F
:100E1000207088F888880507070600003860A0B8A9
:100E2000E0A0B80508080600FF7088808088702060
:100E300060050808060000402000F880F080F805F2
:100E40000808060000081000F880F080F80508087F
:100E5000060000205000F880F080F8050707060023
:100E6000005000F880F080F8030808060100804078
:100E700000E0404040E0030808060100204000E098
:100E8000404040E003080806010040A000E0404068
:100E900040E0030707060100A000E0404040E005F5
:100EA0000707060000704848E8484870050808062B
:100EB000000068900088C8A8988805080806000007
:100EC0004020708888888870050808060000102077
:100ED0007088888888700508080600002050007017
:100EE0008888887005080806000068900070888867
:100EF000887005080806000050007088888888708F
:100F000005050506000188502050880508080600E0
:100F1000FF1070A8A8A8A8704005080806000040A7
:100F200020888888888870050808060000102088B6
:100F30008888888870050808060000205000888886
:100F4000888870050808060000500088888888880E
:100F50007005080806000010208850202020200579
:100F600009090600FFC040704848704040E004088E
:100F7000080601FF609090A09090E08005080806A8
:100F800000004020007008788878050808060000F6
:100F900010200070087888780508080600002050A6
:100FA00000700878887805080806000068900070CE
:100FB00008788878050707060000500070087888D0
:100FC0007805080806000020502070087888780509
:100FD0000606060000D02878A0A8500506060600E0
:100FE000FF7080887020600508080600004020001F
:100FF0007088F880700508080600001020007088CE
:10100000F880700508080600002050007088F880FD
:101010007005070706000050007088F8807003080C
:101020000806010080400040C04040E00308080678
:10103000010020400040C04040E0030808060100D5
:1010400040A00040C04040E0030707060100A000A8
:1010500040C04040E0050707060000A040A010780F
:101060008870050808060000689000B0C888888865
:101070000508080600004020007088888870050870
:10108000080600001020007088888870050808068F
:10109000000020500070888888700508080600004D
:1010A0006890007088888870050707060000500067
:1010B00070888888700505050600012000F800206A
:1010C0000507070600FF1070A8A8A87040050808CB
:1010D00006000040200088888898680508080600F7
:1010E00000102000888888986805080806000020FD
:1010F0005000888888986805070706000050008817
:10110000888898680509090600FF102000888888EB
:10111000F808700407070601FFC04060506040E017
:101120000508080600FF50008888887808705A0073
:1011300059005800092000000000000000000000D5
:101140000000007FFFE00000000000000000000041
:1011500000007000E000000000000000000000003F
:101160000061F860000000000000000000000000C6
:1011700041F82000000000000000000000000040D6
:10118000F0200000000000000000000000004060AF
:10119000200000000000000000000000005801A036
:1011A0007F80000000000000004104005C63A0FF9D
:1011B000C0000000000000002082005EF7A0FFC019
:1011C000000000000000002082005EF7A0FFC000C9
:1011D0000000000000004104005C63A07F8000006C
:1011E00000000000008208005801A07F800000007D
:1011F00000000001041000406020FFC0000000005B
:1012000000000104100040F020FFC00000000000BA
:10121000000082080041F820FFC00000000000002C
:101220000041040061F8603F000000000000000081
:101230000000007000E01E0000000000000001FF40
:10124000FF807FFFE00C0000000000000001FFFFB6
:10125000800000000000000000000000000000000E
:101260007FFFE000000000000000000000000070B0
:1012700000E0000000000000000000000000630C1F
:1012800060000000000000000000000000470E2089
:101290000000000000000000000000004F0F2000D0
:1012A00000000000000000000000005F0FA0000030
:1012B000000000000000000000005E07A07F80002A
:1012C000000000000000410400406020FFC000005A
:1012D000000000000020820040F020FFC00000005D
:1012E0000000000020820040F020FFC0000000004D
:1012F0000000004104004060207F800000000000EA
:1013000000008208005E07A07F800000000000004F
:10131000010410005F0FA0FFC000000000000001EA
:101320000410004F0F20FFC00000000000000082EA
:101330000800470E20FFC00000000000000041042C
:1013400000630C603F00000000000000000000008F
:101350007000E01E0000000000000001FFFF807F21
:10136000FFE00C0000000000000001FFFF80000013
:101370000053442063617264206F6B0A006F7065D4
:101380006E526F6F74206661696C65640A00766FD7
:101390006C756D652E696E6974206661696C656433
:1013A0000A00534420696E6974206661696C0A0002
:1013B0007C3C3E5E2B3D3F2F5B5D3B2C2A225C003C
:1013C00020204D383531205A005A2D50726F6265F9
:1013D000204F666673657420286D6D293A0A0020D7
:1013E000440020490020204D333034205000204458
:1013F0000020490020204D33303120500050494416
:101400002073657474696E67733A0A002046002081
:10141000420020480020204D3134352053004D61DA
:1014200074657269616C20686561747570207061A3
:1014300072616D65746572733A0A0020204D343212
:10144000302053004175746F20426564204C6576EE
:10145000656C696E673A0A00205A00205900202006
:101460004D323036205800486F6D65206F666673C8
:1014700065743A0A00204500205A0020590020587F
:101480000020420020540020204D323035205300EF
:10149000416476616E6365643A20533C6D696E5FAA
:1014A00066656564726174653E20543C6D696E5F6B
:1014B00074726176656C5F66656564726174653EC1
:1014C00020423C6D696E5F7365676D656E745F7415
:1014D000696D655F6D733E20583C6D61785F78790A
:1014E0005F6A65726B3E205A3C6D61785F7A5F6A15
:1014F00065726B3E20453C6D61785F655F6A657221
:101500006B3E0A0020540020520020204D3230341F
:10151000205000416363656C65726174696F6E2071
:1015200028756E6974732F7332293A20503C70729B
:10153000696E745F616363656C3E20523C726574D2
:10154000726163745F616363656C3E20543C7472C6
:101550006176656C5F616363656C3E0A00204500DF
:10156000205A0020590020204D3230312058004DA3
:101570006178696D756D20416363656C6572617436
:10158000696F6E2028756E6974732F7332293A0A59
:1015900000204500205A0020590020204D323033D1
:1015A0002058004D6178696D756D206665656472BF
:1015B000617465732028756E6974732F73293A0AF4
:1015C00000204500205A0020590020204D393220AB
:1015D000580053746570732070657220756E69745D
:1015E0003A0A0020204D3230302044300A002020BA
:1015F0004D3230302044002044697361626C656470
:101600000A0046696C616D656E7420736574746957
:101610006E67733A0020204D3134392043203B203F
:10162000556E69747320696E2043656C73697573B8
:101630000A002020473231202020203B20556E69AF
:10164000747320696E206D6D0A0025697300256929
:101650006D20256973002569682025696D2025693D
:101660007300256964202569682025696D20256936
:10167000730025697920256964202569682025691A
:101680006D20256973005072696E742074696D65F0
:101690003A200020746F6F206C6F6E67206578743D
:1016A000727573696F6E2070726576656E746564AD
:1016B0000A0020636F6C6420657874727573696FBB
:1016C0006E2070726576656E7465640A0020746FB2
:1016D0006F206C6F6E6720657874727573696F6EBA
:1016E0002070726576656E7465640A0020636F6CA5
:1016F0006420657874727573696F6E207072657698
:10170000656E7465640A00436172642072656D6F72
:10171000766564004361726420696E7365727465F6
:101720006400004D3234005072696E74207061752F
:10173000736564004D313235004D36303020423013
:10174000004D3234004D3233202573006175746FC3
:1017500025692E67004578747275646572004D6F57
:101760007665205A004D6F76652059004D6F76657D
:101770002058004D6F76656D656E74004D6F76650F
:1017800020617869730044697361626C65207374C9
:10179000657070657273004D383400426564204C8A
:1017A0006576656C696E67004732382058590A4D76
:1017B00031303920533137350A473238205A0A4DF3
:1017C00031303920523134350A4731320A47323903
:1017D0000A4D313034205330004175746F20686FEA
:1017E0006D6500473238004D61696E00434F4D4DC5
:1017F000554E49434154494F4E0044525952554E5B
:10180000004552524F525300494E464F00454348FF
:101810004F001000C90210012C014001220170018B
:101820001801B0010E01F00104015002FA00B002EB
:10183000F0003003E600D003DC009004D200700515
:10184000C800A006BE000008B400B009AA00D00B72
:10185000A000600E960060118C0000158200201917
:101860007800C01D6E00A0226400B0275A00902CA2
:10187000500000314600E0343C0010383200903A0D
:101880002800603C1E00A03D1400803E0A00203F5E
:1018900000004E6F2063617365206C696768740A8D
:1018A000002F2F20004361703A454D455247454E69
:1018B00043595F5041525345523A310A00436170D7
:1018C0003A434153455F4C494748545F4252494768
:1018D00048544E4553533A300A004361703A544FCE
:1018E00047474C455F4C49474854533A300A0043F8
:1018F00061703A534F4654574152455F504F5745D8
:10190000523A300A004361703A4C4556454C494EB4
:10191000475F444154413A310A004361703A5A5F8B
:1019200050524F42453A310A004361703A41555492
:101930004F4C4556454C3A310A004361703A50527B
:10194000494E545F4A4F423A310A004361703A505F
:10195000524F47524553533A300A004361703A415F
:1019600055544F5245504F52545F54454D503A31A3
:101970000A004361703A454550524F4D3A310A00D2
:101980004649524D574152455F4E414D453A4D6192
:10199000726C696E20204649524D574152455F5640
:1019A000455253494F4E3A312E312E352E34342084
:1019B00045585452554445525F545950453A416533
:1019C000726F7374727564657220534F555243453C
:1019D0005F434F44455F55524C3A68747470733A94
:1019E0002F2F636F64652E616C6570686F626A6526
:1019F0006374732E636F6D2F646966667573696FA8
:101A00006E2F4D41524C494E2050524F544F434F30
:101A10004C5F56455253494F4E3A312E30204D417E
:101A20004348494E455F545950453A4C756C7A428B
:101A30006F742054415A203720455854525544451C
:101A4000525F434F554E543A3120555549443A61FF
:101A5000393532353737642D383732322D34383313
:101A6000612D393939642D616364633965373732E3
:101A70006237620A004D31343520533C696E64652B
:101A8000783E206F7574206F662072616E676520E6
:101A900028302D31290A000D1808180118FA17EC02
:101AA000176F66660044454255473A0020706F73D1
:101AB0006974696F6E206F7574206F662072616E35
:101AC00067652E0A003F50726F626520001000ADFE
:101AD0000330016A0150022B0170030A019004F5E2
:101AE00000B005E500D006D800F007CE001009C50B
:101AF00000300ABE00500BB700700CB100900DAB67
:101B000000B00EA600D00FA200F0109D0010129998
:101B100000301395005014920070158E0090168BB3
:101B200000B0178700D0188400F0198100101B7EC8
:101B300000301C7B00501D7900701E7600901F73D2
:101B400000B0207000D0216E00F0226B00102469DC
:101B50000030256600502663007027610090285EE3
:101B600000B0295C00D02A5900F02B5600102D54EB
:101B700000302E5100502F4E0070304B00903148F5
:101B800000B0324500D0334200F0343E0010363B06
:101B900000303737005038330070392E00903A2922
:101BA00000B03B2300D03C1B00F03D1100103F0172
:101BB00000F03F0000506C656173652072657365CD
:101BC00074005052494E5445522048414C544544AB
:101BD000005072696E7465722068616C7465642E61
:101BE000206B696C6C28292063616C6C6564210A28
:101BF000006265640A002C2073797374656D20732C
:101C0000746F7070656421204865617465725F4906
:101C1000443A2000544845524D414C2052554E41C3
:101C20005741592042454400546865726D616C20EB
:101C300052756E6177617900544845524D414C2090
:101C400052554E4157415920453100544845524D57
:101C5000414C2052554E415741592045300048656E
:101C60006174696E67206661696C656420424544F1
:101C70000048656174696E67206661696C6564001F
:101C800048656174696E67206661696C65640048C7
:101C9000656174696E67206661696C6564204530B2
:101CA0000057726974696E6720746F2066696C658D
:101CB0003A20006F70656E206661696C65642C2047
:101CC00046696C653A20006F70656E206661696CCC
:101CD00065642C2046696C653A200046696C652075
:101CE00073656C65637465640A002053697A653AAC
:101CF000200046696C65206F70656E65643A20004F
:101D00006F70656E206661696C65642C2046696C35
:101D1000653A20002066696C653A20004E6F772096
:101D2000002220706F73002220706172656E743A19
:101D30002200535542524F5554494E452043414C81
:101D40004C207461726765743A22004B494C4C45D3
:101D5000442E2000747279696E6720746F2063616D
:101D60006C6C207375622D67636F64652066696CA7
:101D70006573207769746820746F6F206D616E7968
:101D8000206C6576656C732E204D4158206C65760D
:101D9000656C2069733A0043616E6E6F74206F70DA
:101DA000656E20737562646972200001050800FF8A
:101DB000060121023520FFFF07FF06FF0900502220
:101DC0001656808080800080153353A0A0A0025753
:101DD000575050F850F850500257572070A07028B4
:101DE000702013355580A040A02002475740A0A086
:101DF00040A0A0502513538080801226564080803A
:101E000080804012265680404040408002455590D8
:101E100060F060900255552020F820201133536067
:101E20004080044151F011335340E04002465610C7
:101E3000102040808012365640A0A0A0A04012364C
:101E40005640C0404040E00246566090106080F02E
:101E5000024656F020601090600246562060A0F0C6
:101E60002020024656F080E01090600246566080C6
:101E7000E0909060024656F0102020404002465606
:101E80006090609090600246566090907010601272
:101E90002555C0C000C0C01136566060006040804B
:101EA000123656204080804020034353F000F01249
:101EB000365680402020408012365640A0204000F8
:101EC00040015858304898A8A890403002465660C3
:101ED0009090F09090024656E090E09090E002469C
:101EE00056609080809060024656E090909090E01E
:101EF000024656F080E08080F0024656F080E08096
:101F00008080024656609080B09060024656909065
:101F1000F0909090123656E040404040E002465625
:101F200070202020A04002465690A0C0A0A09002A1
:101F300046568080808080F002465690F0F0909067
:101F40009002465690D0F0B0B09002465660909005
:101F5000909060024656E09090E080800147576084
:101F60009090D0B06010024656E09090E0909002C1
:101F70004656609040209060123656E04040404007
:101F800040024656909090909060024656909090F5
:101F9000906060024656909090F0F0900246569005
:101FA000906060909002565688885020202002460B
:101FB00056F010204080F0123656E080808080E09D
:101FC000024656808040201010123656E020202015
:101FD00020E016325240A0014151F01622528040BA
:101FE000024454709090700246568080E09090E0D9
:101FF00012345460808060024656101070909070C9
:1020000002445460B0C060024656205040E0404058
:1020100001455560907010600246568080E09090B7
:10202000901236564000C04040E011375720002043
:102030002020A040024656808090E09090123656B4
:10204000C040404040E0025454D0A8A8A8024454E4
:10205000E090909002445460909060014555E0906B
:10206000E080800145557090701010024454A0D05B
:10207000808012345460C020C00246564040E04088
:10208000502002445490909070123454A0A0A0406C
:1020900002545488A8A850024454906060900145AE
:1020A000559090709060024454F02040F0024757E1
:1020B000304020C0204030221656808080808080B2
:1020C000024757C02040304020C006425250A0FF77
:1020D000FFFFFFFFFFFFFFFFFFFFFFFFFFFFFFFF10
:1020E000FFFFFFFFFFFFFFFFFFFFFFFFFFFFFFFF00
:1020F00009005022165680008080808001465620BC
:1021000070A0A070200246562050E04050A002551A
:102110005588705070880256568850F820F8202252
:102120001757808080008080800247577080E09041
:102130007010E0173151A002565670A8C8C8A87098
:1021400014355560A06000E003435350A050123393
:1021500053E02020143151E002565670E8D8E8D8F8
:1021600070173151E015335340A04012355540E00F
:102170004000E014355540A02040E0143555C02003
:10218000C020C01622524080014555909090E080BA
:1021900002565678E8E86828282411518011225206
:1021A000408014355540C04040E014355540A040B3
:1021B00000E0034353A050A0024757808080A060F6
:1021C000F0200247578080A0D0102070024757802F
:1021D000408060A0F02012365640004080A04002AF
:1021E000475740206090F090900247572040609001
:1021F000F0909002475760906090F090900247579F
:1022000050A06090F0909002475790006090F0903E
:102210009002475760906090F0909002465670A0F0
:10222000A0F0A0B0014757609080809060400247C6
:10223000574020F080E080F00247572040F080E0D7
:1022400080F00247576090F080E080F0024757909E
:1022500000F080E080F01237578040E0404040E0DE
:102260001237572040E0404040E012375740A0E08E
:10227000404040E0123757A000E0404040E00256A6
:10228000567048E848487002475750A090D0B09028
:10229000900247574020609090906002475720403E
:1022A00060909090600247576090609090906002BC
:1022B000475750A060909090600247579000609000
:1022C000909060123353A040A002465670B0B0D038
:1022D000D0E00247574020909090906002475720EE
:1022E00040909090906002475760909090909060DE
:1022F00002475790009090909060025757102088A6
:102300005020202002465680E09090E08002465601
:102310006090A0A090A0024757402000709090705D
:10232000024757204000709090700247572050009D
:102330007090907002475750A000709090700246C5
:102340005650007090907002475760906070909067
:1023500070025454F068B078113555608080604048
:1023600002475740200060B0C0600247572040003D
:1023700060B0C06002475760900060B0C060024625
:1023800056500060B0C060123757804000C04040D7
:10239000E0123757204000C04040E012375740A0BD
:1023A00000C04040E0123656A000C04040E0024766
:1023B00057A040A01070906002475750A000E090D6
:1023C000909002475740200060909060024757204D
:1023D000400060909060024757609000609090606D
:1023E00002475750A00060909060024656900060EF
:1023F0009090601235554000E0004002445470B0A7
:10240000D0E002475740200090909070024757203C
:1024100040009090907002475760900090909070AC
:1024200002465690009090907001485820400090CD
:10243000907090600147578080E090E08080014775
:10244000579000909070906001050700FE0500FB1A
:1024500001F220FFFE05FE05FE0200400215258068
:1024600080800080053242A0A002556550F850F8E7
:10247000500146562070C030E02002556590102073
:10248000404802556560806890680512228080028D
:1024900025354080808040022535804040408004C2
:1024A0003343A040A003334340E040012232408048
:1024B000043141E00211218002556508102040805E
:1024C0000245556090909060022535C040404040E4
:1024D000024555E0106080F0024555E0106010E0C4
:1024E0000245552060A0F020024555F080E010E044
:1024F0000245556080E09060024555F01020404054
:102500000245556090609060024555609070106083
:10251000031323800080021424800080800235454C
:102520002040804020033343E000E00235458040F6
:10253000204080024555E0106000400255657088DB
:10254000B8A870024555609090F090024555E09013
:10255000E090E00235456080808060024555E09063
:102560009090E0023545E080E080E0023545E08073
:10257000E080800245557080B09070024555909083
:10258000F09090023545E0404040E0024555301063
:1025900010906002455590A0C0A090023545808003
:1025A0008080E002556588D8A8888802455590D07B
:1025B000B090900245556090909060024555E09033
:1025C00090E080014656609090906010024555E082
:1025D0009090E09002455570806010E0023545E033
:1025E0004040404002455590909090600245559083
:1025F00090A0A04002556588A8A8A8500245559013
:10260000906090900245559090701060023545E0C2
:10261000204080E0022535C0808080C00255658062
:1026200040201008022535C0404040C005324240DD
:10263000A0024151F0052232804002445470909033
:102640007002455580E09090E002344460808060E4
:10265000024555107090907002445460B0C0600202
:1026600035452040E0404000465670909070106024
:1026700002455580E0909090021525800080808072
:10268000002737400040404040800245558090A0E0
:10269000E0900215258080808080025464F0A8A814
:1026A000A8024454E09090900244546090906000DE
:1026B0004656E09090E080800046567090907010F2
:1026C00010023444A0C0808002445470C030E00244
:1026D000354540E0404020024454909090700244C0
:1026E000549090A040025464A8A85050023444A0D2
:1026F0004040A0004656909090701060024454F004
:102700002040F00235456040804060021525808001
:10271000808080023545C0402040C005425250A014
:10272000FFFFFFFFFFFFFFFFFFFFFFFFFFFFFFFFB9
:10273000FFFFFFFFFFFFFFFFFFFFFFFFFFFFFFFFA9
:10274000FF020040FFFFFFFFFFFFFFFFFFFFFFFF54
:10275000FFFFFFFFFFFFFFFFFFFFFFFFFFFFFFFF89
:10276000FFFFFFFFFFFFFFFFFFFFFFFFFFFFFFFF79
:10277000FFFFFFFFFFFFFFFFFFFFFFFFFFFFFFFF69
:10278000FFFFFFFFFFFFFFFFFFFFFFFFFFFFFFFF59
:10279000FFFFFFFFFFFFFFFFFFFFFFFFFFFFFFFF49
:1027A000FFFFFF01060D00FE09016602D620FFFEB5
:1027B0000BFE0AFE0D0060221969808080808080F7
:1027C000800080183363A0A0A00357675050F850D2
:1027D000F850500259692078A0A0702828F02002F3
:1027E000596948A85010204050A89002586840A04D
:1027F000A040A0989068281363808080113B6B20D4
:1028000040408080808080404020113B6B80404071
:10281000202020202040408006556520A870A82058
:102820000455652020F82020113363604080065154
:1028300061F811336340E040025969080810102024
:1028400040408080025969205088888888885020BC
:102850000259692060A02020202020F802596970C8
:1028600088880810204080F8025969F80810207004
:1028700008088870025969101030505090F81010F4
:10288000025969F88080B0C80808887002596970D8
:10289000888080F088888870025969F808101020B4
:1028A0002040404002596970888888708888887004
:1028B00002596970888888780808887011386840DB
:1028C000E040000040E04011386840E04000006017
:1028D00040800259690810204080402010080454AC
:1028E00064F80000F8025969804020100810204068
:1028F00080025969708888081020200020025969D8
:1029000070888898A8A8B080780259692050888873
:1029100088F8888888025969F048484870484848CB
:10292000F0025969708880808080808870025969BF
:10293000F048484848484848F0025969F880808083
:10294000F0808080F8025969F8808080F080808073
:1029500080025969708880808098888870025969DF
:1029600088888888F888888888123969E0404040DB
:1029700040404040E002596938101010101010908B
:1029800060025969888890A0C0A09088880259691F
:102990008080808080808080F80259698888D8A8EB
:1029A000A88888888802596988C8C8A8A89898887B
:1029B000880259697088888888888888700259696F
:1029C000F0888888F080808080015A6A70888888C2
:1029D000888888A87008025969F0888888F0A090D3
:1029E0008888025969708880807008088870025948
:1029F00069F820202020202020200259698888881A
:102A000088888888887002596988888888505050DA
:102A1000202002596988888888A8A8A8A850025947
:102A20006988885050205050888802596988885099
:102A3000502020202020025969F808101020404022
:102A400080F8113B6BE0808080808080808080E017
:102A5000025969808040402010100808113B6BE04B
:102A6000202020202020202020E0085363205088B0
:102A7000015161F82A226280400256667008788807
:102A80009868025969808080F088888888F00256AA
:102A9000667088808088700259690808087888887C
:102AA0008888780256667088F88088700259693084
:102AB000484040F04040404000586870888888781E
:102AC000088870025969808080B0C8888888881218
:102AD00038684000C040404040E0004A6A10003082
:102AE0001010101090906002596980808090A0C0F2
:102AF000A09088123969C040404040404040E00208
:102B00005666D0A8A8A8A888025666B0C888888843
:102B100088025666708888888870005868F08888AF
:102B200088F080808000586878888888780808084D
:102B3000025666B0C8808080800256667088601039
:102B400088700258684040F0404040483002566665
:102B5000888888889868025666888888505020023D
:102B600056668888A8A8A85002566688502020502B
:102B7000880058688888889868088870025666F8BF
:102B800010204080F8015B6B1820202020C02020FE
:102B900020201822196980808080808080808001B8
:102BA0005B6BC0202020201820202020C008536309
:102BB00048A890FFFFFFFFFFFFFFFFFFFFFFFFFFA2
:102BC000FFFFFFFFFFFFFFFFFFFFFFFFFFFFFFFF15
:102BD000FFFFFFFF0D006022196980008080808068
:102BE0008080800358682070A8A0A0A87020025997
:102BF0006930484040E0404048B003566688705015
:102C000050708802596988885050F820F820202296
:102C10001969808080800080808080124A6A60907C
:102C200080609090601090601A3262A0A003596991
:102C30007088A8D8C8D8A8887004576770087888A2
:102C40007800F80356662850A0A05028045363F873
:102C50000808163161E00359697088E8D8D8E8D8C7
:102C600088700A5161F81744646090906003576758
:102C70002020F8202000F807356540A02040E0071C
:102C8000356540A04020C02A2262408000586888F4
:102C900088888898E8808002596978E8E8E8E868D8
:102CA000282828262161C0202262408007356540FF
:102CB000C04040E0045767708888887000F8035669
:102CC00066A050282850A0025A6A40C04040E00840
:102CD00018283808025A6A40C04040E010280810FE
:102CE00038025A6A40A04020A048182838080259E3
:102CF00069200020204080888870025A6A402000A5
:102D000020508888F88888025A6A1020002050884D
:102D100088F88888025A6A30480020508888F888E5
:102D200088025A6A28500020508888F88888025AF9
:102D30006A50500020508888F88888025A6A2050CB
:102D40002020508888F8888802596958A0A0A0B02F
:102D5000E0A0A0B8005B6B70888080808080887065
:102D60002040025A6A402000F88080F08080F802FB
:102D70005A6A102000F88080F08080F8025A6A3089
:102D80004800F88080F08080F8025A6A505000F8BD
:102D90008080F08080F8123A6A804000E040404035
:102DA0004040E0123A6A204000E04040404040E0AD
:102DB000124A6A609000E04040404040E0123A6AA7
:102DC000A0A000E04040404040E0025969F048487F
:102DD00048E8484848F0025A6A2850008888C8A83D
:102DE000988888025A6A402000708888888888708D
:102DF000025A6A10200070888888888870025A6A8F
:102E000030480070888888888870025A6A28500084
:102E100070888888888870025A6A50500070888844
:102E2000888888700355658850205088015B6B083E
:102E3000709898A8A8A8C8C87080025A6A40200054
:102E400088888888888870025A6A10200088888854
:102E500088888870025A6A304800888888888888FC
:102E600070025A6A50500088888888888870025A90
:102E70006A1020008888502020202002596980F0A4
:102E8000888888F0808080025969609090A0A09026
:102E90008888B002596940200070087888986802D4
:102EA000596910200070087888986802596930487C
:102EB000007008788898680259692850007008786E
:102EC000889868025969505000700878889868029C
:102ED0005A6A3048300070087888986802566670E0
:102EE0002870A0A8500058687088808088702040A2
:102EF0000259694020007088F88088700259691072
:102F000020007088F8808870025969304800708805
:102F1000F88088700259695050007088F880887075
:102F2000123969804000C040404040E012396920B9
:102F30004000C040404040E0124969609000C040FD
:102F4000404040E0123969A0A000C040404040E04D
:102F5000025A6A5020601070888888887002596907
:102F6000285000B0C88888888802596940200070BD
:102F7000888888887002596910200070888888883D
:102F800070025969304800708888888870025969D1
:102F900028500070888888887002596950500070E5
:102FA0008888888870035767202000F80020200157
:102FB0005868087098A8A8C8708002596940200015
:102FC00088888888986802596910200088888888CD
:102FD000986802596930480088888888986802593A
:102FE00069505000888888889868005B6B102000C2
:102FF0008888889868088870005A6A8080B0C88875
:1030000088C8B08080005B6B5050008888889868C2
:1030100008887000000000000000000000000000B0
:1030200000000000000000000000000000000000A0
:103030000000000000000C000000000000000C0078
:10304000000000000000120000000000000023004B
:1030500000000000000021000000000000004C8083
:103060000000000000005E800000000000009240B0
:10307000000000000000A14000000000000121202D
:103080000000000000027F9000000000000200101D
:10309000000000000007FFF8000000000004000826
:1030A0000000000000080004000000000008000606
:1030B00000000000001000020000000000301E01AF
:1030C0000000000000207F81000000000041FFE0C0
:1030D000800000000043FCF08000000000873B7887
:1030E00040000000018EDBFC60000000010FEBCC13
:1030F00020000000021FEDB610000000021FDEB627
:10310000100000000439CD7F080000000436E0FF05
:1031100008000000087EC0BB84000000187F005D2E
:1031200086000000107FC0ED82000000203CC073CC
:1031300001000000203B337F01000000701BE77E90
:1031400003800000C81DEEDE04C00000880FDEDC36
:1031500004400001240FDF3C092000012607DBF8B2
:10316000192000027203E7F0139000025101FFE002
:103170002290000489007F802448000904801E00FA
:103180004824000BFE400000DFF400100040000067
:103190008002001FFFFFFFFFFFFE00000000000095
:1031A000000000000000000000000000000000001F
:1031B0000000001022103C3C0E1F001022100422C0
:1031C0001104001022100822110400102210083CE3
:1031D00011040010221010221104001022102022CD
:1031E0001104001E1C1E3C3C0E04000000000000E8
:1031F00000000000000000000000000000000000CF
:1032000000000000000000000000000000000000BE
:1032100000000000000000000000000000000000AE
:10322000000000000000000000000000000000009E
:10323000000000000000000000000000000000008E
:10324000000000000000000000000000000000007E
:10325000000A003B20454550524F4D20496E6465A1
:10326000783A20005570646174696E67207A6F66E1
:103270006673657420696E20454550524F4D3A2063
:10328000000600060006000600060006000600060E
:103290000006003FC01F800F00060006000F001F41
:1032A000803FC00600060006000600060006000675
:1032B000000600060007F8000C0C001002002001B8
:1032C000006001804000804003E04001C040008079
:1032D0004000004000006000002000001000000CD2
:1032E0000C0007F80001FE00030300040080080042
:1032F000401800601000207C0020380020100020C2
:10330000000020000020000060000040000080035A
:10331000030001FE00FFFFFF7F80FFC0FFC0FFC072
:103320007F807F80FFC0FFC0FFC03F001E000C00F9
:103330005A204F6666736574004D6F76652058009D
:103340004D6F76652059004D6F7665205A0045789F
:1033500074727564657200000080C100809743003C
:103360008095435761726E696E673A20486F6D6948
:103370006E672042756D702044697669736F7220A4
:103380003C20310A000202040000A0400000A040DE
:103390000000004000009E430080A1430080954350
:1033A00000004842000048420000204100000000A8
:1033B000FF01014F6666004F6E2000456E64737416
:1033C0006F702061626F72740053746570732F6D3B
:1033D0006D004A65726B00416363656C6572617470
:1033E000696F6E0056656C6F63697479005A204F7F
:1033F000666673657400416476616E63656420532C
:10340000657474696E6773005654726176206D69D5
:103410006E005654726176206D696E00565472616A
:1034200076206D696E00566D696E00566D696E008E
:10343000566D696E00566D6178204500566D617855
:10344000204500566D6178204500566D6178205A00
:1034500000566D6178205A00566D6178205A0056EA
:103460006D6178205900566D6178205900566D6164
:1034700078205900566D6178205800566D6178208B
:103480005800566D61782058004D6F74696F6E005A
:103490004573746570732F6D6D004573746570733B
:1034A0002F6D6D005A73746570732F6D6D005A73B4
:1034B000746570732F6D6D005973746570732F6D23
:1034C0006D005973746570732F6D6D00587374655A
:1034D00070732F6D6D005873746570732F6D6D0070
:1034E0004D6F74696F6E0056652D6A65726B00567C
:1034F000652D6A65726B0056652D6A65726B0056A4
:103500007A2D6A65726B00567A2D6A65726B005669
:10351000792D6A65726B0056792D6A65726B00565B
:10352000792D6A65726B0056782D6A65726B00564C
:10353000782D6A65726B0056782D6A65726B004D46
:103540006F74696F6E0043616E6E6F7420656E7488
:103550006572207375626469723A2000022E2E0033
:103560004D61696E004D6F766520302E316D6D00B6
:103570004D6F766520316D6D004D6F766520313071
:103580006D6D004D6F7665206178697300457874C4
:103590007275646572004D6F7665205A004D6F76C6
:1035A000652059004D6F7665205800746F20726554
:1035B00073756D65005761697420666F7220707253
:1035C000696E74005052494E542050415553454441
:1035D0000045787472756465206D6F726500526580
:1035E00073756D65207072696E7400524553554D48
:1035F00045204F5054494F4E533A0020204E6F7A89
:103600007A6C653A20002000506C65617365207704
:103610006169742E2E2E0048656174696E67206E94
:103620006F7A7A6C65005052494E54205041555380
:1036300045440020204E6F7A7A6C653A20002000C5
:1036400068656174206E6F7A7A6C652E00507265C1
:10365000737320627574746F6E20746F00505249DA
:103660004E54205041555345440020204E6F7A7AE5
:103670006C653A2000200066696C616D656E74208F
:1036800065787472756465005761697420666F723D
:10369000005052494E54205041555345440020207B
:1036A0004E6F7A7A6C653A2000200066696C616D15
:1036B000656E74206C6F6164005761697420666F79
:1036C00072005052494E54205041555345440020F9
:1036D000204E6F7A7A6C653A2000746F20636F6EAB
:1036E00074696E75652E2E2E00616E642070726591
:1036F000737320627574746F6E00496E73657274B3
:103700002066696C616D656E74005052494E54209C
:10371000504155534544004572726F72207772696B
:1037200074696E6720746F20454550524F4D210AD1
:1037300000486F6D652025732573257320666972B7
:103740007374002066697273740A005A0059005835
:1037500000486F6D65200000060900FE0601890221
:10376000FE20FFFE07FE06FE000000060007010621
:1037700006060200808080800080030303060103A8
:10378000A0A0A00507070600FF5050F850F85050C1
:103790000509090600FE2070A8A07028A870200660
:1037A00008080600FF40A8481020485408050707ED
:1037B0000600FF6090906098906801030306020382
:1037C0008080800207070602FF4080808080804062
:1037D0000207070602FF8040404040408005050583
:1037E0000600008850F850880505050600002020D6
:1037F000F820200204040602FEC0404080050101BA
:10380000060002F8020202060200C0C00406060614
:103810000100101020408080040606060100609020
:103820009090906003060606010040C0404040E0D2
:103830000406060601006090102040F0040606060B
:103840000100F020601010E00506060600001030B0
:103850005090F810040606060100F080E01010E019
:103860000406060601006080E090906004060606EB
:103870000100F01010204040040606060100609090
:1038800060909060040606060100609090701060E1
:10389000020505060200C0C000C0C00207070602FC
:1038A000FEC0C000C040408005050506000018604D
:1038B000806018050303060001F800F805050506F9
:1038C0000000C0300830C0040707060100609010F7
:1038D000604000400506060600007090A8B08070A9
:1038E000050606060000205088F8888805060606AA
:1038F0000000F088F08888F0040606060100609059
:1039000080809060040606060100E090909090E0B0
:10391000040606060100F080E08080F0040606063A
:103920000100F080E08080800406060601006090BF
:1039300080B090600406060601009090F090909090
:10394000030606060100E040404040E0050606068A
:10395000000038101010906004060606010090A0C8
:10396000C0A090900406060601008080808080F050
:1039700005060606000088D8A8A88888040606065A
:10398000010090D0B0909090050606060000708867
:1039900088888870040606060100E09090E0808028
:1039A0000407070601FF609090D0B060100406067F
:1039B000060100E09090E090900406060601006089
:1039C0009040209060050606060000F82020202088
:1039D0002004060606010090909090906004060670
:1039E000060100909090F0606005060606000088D1
:1039F00088A8A8D888050606060000885020205010
:103A00008805060606000088885020202004060647
:103A1000060100F010204080F0030606060100E0D9
:103A200080808080E004060606010080804020102F
:103A300010030606060100E020202020E005030315
:103A40000600032050880501010600FEF80202026C
:103A50000602048040040404060100709090700483
:103A600006060601008080E09090E0040404060150
:103A7000007080807004060606010010107090909F
:103A80007004040406010060B0C07004060606015C
:103A900000205040E040400406060601FE60909081
:103AA0007010600406060601008080E0909090038C
:103AB00006060601004000C04040E0030808060179
:103AC000FE200060202020A04004060606010080A1
:103AD00080A0C0A090030606060100C04040404000
:103AE000E0050404060000D0A8A888040404060128
:103AF00000E090909004040406010060909060043F
:103B000006060601FEE09090E080800406060601AD
:103B1000FE709090701010040404060100A0D08084
:103B20008004040406010070C030E00406060601AB
:103B3000004040E0405020040404060100909090B2
:103B400070040404060100909060600504040600FF
:103B50000088A8A850040404060100906060900446
:103B600006060601FE909090709060040404060121
:103B700000F02040F003070706010020404080408D
:103B800040200107070602FF80808080808080033C
:103B900007070601008040402040408004020206E2
:103BA000010350A0FFFFFFFFFFFFFFFFFFFFFFFF2D
:103BB000FFFFFFFFFFFFFFFFFFFFFFFFFFFFFFFF15
:103BC000FFFFFFFFFF0000000600070106060602D8
:103BD000008000808080800406060601FF2070A01F
:103BE000A070200507070600FF304840F04040F86D
:103BF000050505060000A8508850A8050606060021
:103C0000008850F820F8200107070602FF80808016
:103C1000008080800407070601FF708060906010BC
:103C2000E0030101060105A00607070600007884ED
:103C300094A494847803050506010160A06000E067
:103C40000505050600002850A050280403030601BE
:103C500000F01010040101060102F006070706003B
:103C6000007884B4A4A48478040101060105F0045A
:103C700003030601026090600507070600FF20208D
:103C8000F8202000F803050506010140A02040E0CF
:103C9000030505060101C0204020C0020202060201
:103CA0000440800405050601FF9090B0D080050611
:103CB0000606000078E8E8682828010101060202EB
:103CC000800202020602FE40800305050601014053
:103CD000C04040E003050506010140A04000E005AA
:103CE0000505060000A0502850A00508080600FFA2
:103CF00040C04050703078100508080600FF40C0F2
:103D00004050680810380508080600FFC020403001
:103D1000F030781004070706010020002060809032
:103D200060050707060000402020507088880507BE
:103D3000070600001020205070888805070706003D
:103D40000020502050708888050707060000285082
:103D5000205070888805070706000050002050702A
:103D600088880507070600002050205070888805C5
:103D7000060606000078A0F0A0A0B8040808060116
:103D8000FE6090808090602040040707060100409C
:103D900020F080E080F00407070601002040F0805A
:103DA000E080F00407070601002050F080E080F07A
:103DB0000407070601005000F080E080F0030707C9
:103DC0000601008040E0404040E003070706010094
:103DD0002040E0404040E003070706010040A0E02B
:103DE000404040E0030707060100A000E0404040DB
:103DF000E00506060600007048E84848700407071A
:103E000006010050A090D0B0909004070706010072
:103E100040206090909060040707060100204060F9
:103E200090909060040707060100205060909090E9
:103E30006004070706010050A0609090906004079E
:103E4000070601005000609090906005050506008F
:103E50000088502050880408080601FF1070B0B098
:103E6000D0D0E08004070706010040209090909099
:103E700060040707060100204090909090600407BE
:103E800007060100205090909090600407070601FB
:103E900000500090909090600507070600001020E9
:103EA000885020202004060606010080E09090E063
:103EB000800406060601006090A0A090A0040707F9
:103EC0000601004020007090907004070706010072
:103ED00020400070909070040707060100205000F9
:103EE0007090907004070706010050A00070909039
:103EF00070040606060100500070909070040707D9
:103F00000601002050207090907005040406000007
:103F100070A8B0780406060601FE7080807020400C
:103F200004070706010040200060B0C070040707C6
:103F300006010020400060B0C070040707060100C1
:103F400020500060B0C070040606060100500060FA
:103F5000B0C070030707060100804000C04040E089
:103F6000030707060100204000C04040E0030707A8
:103F700006010040A000C04040E003060606010024
:103F8000A000C04040E00407070601003060107048
:103F900090906004070706010050A000E090909008
:103FA00004070706010040200060909060040707A6
:103FB00006010020400060909060040707060100A1
:103FC0002050006090906004070706010050A00098
:103FD00060909060040606060100500060909060BA
:103FE0000505050600002000F80020040404060171
:103FF0000070B0D0E0040707060100402000909058
:104000009070040707060100204000909090700413
:1040100007070601002050009090907004060606E5
:1040200001005000909090700409090601FE2040A4
:10403000009090907090600408080601FE8080E077
:104040009090E080800408080601FE500090909057
:104050007090605265776970696E670050726F6228
:10406000696E67206661696C65640050726F626991
:104070006E67206661696C65640050524F4245204E
:104080004641494C20434C45414E204E4F5A5A4CD4
:10409000450A005265776970696E670A0052657754
:1040A0006970696E670050726F62696E6720666141
:1040B000696C65640050726F62696E672066616941
:1040C0006C65640050524F4245204641494C2043A4
:1040D0004C45414E204E4F5A5A4C450A0052657786
:1040E0006970696E670A0050726F62696E67206658
:1040F00061696C65640A0050726F62696E67206660
:1041000061696C656400205A3A200020593A200009
:1041100042656420583A20000A0A426564204C65D2
:1041200076656C20436F7272656374696F6E204DA3
:1041300061747269783A00202B000A436F727265CD
:10414000637465642042656420486569676874200B
:1041500076732E2042656420546F706F6C6F6779A0
:104160003A0A00202B000A426564204865696768A6
:104170007420546F706F6772617068793A0A2020FA
:10418000202B2D2D2D204241434B202D2D2B0A205D
:1041900020207C20202020202020202020207C0A7D
:1041A000204C207C20202020282B29202020207C0F
:1041B00020520A2045207C20202020202020202062
:1041C00020207C20490A2046207C20282D29204EB2
:1041D00020282B29207C20470A2054207C202020C6
:1041E00020202020202020207C20480A2020207C05
:1041F00020202020282D29202020207C20540A2027
:1042000020207C20202020202020202020207C0A0C
:104210002020204F2D2D2046524F4E54202D2D2B47
:104220000A2028302C30290A004D65616E206F6607
:104230002073616D706C656420706F696E74733A81
:10424000200020643A200020623A200045716E2050
:10425000636F656666696369656E74733A20613A77
:10426000200052756E6E696E6720696E2044525947
:104270002D52554E206D6F64650A0047323920413A
:1042800075746F20426564204C6576656C696E6755
:104290000A0028422961636B00284629726F6E74F8
:1042A000002852296967687400284C2965667400E3
:1042B0003F4E756D626572206F662070726F626529
:1042C00020706F696E747320697320696D706C6102
:1042D000757369626C65202832206D696E696D7531
:1042E0006D292E0A003F2856296572626F7365207A
:1042F0006C6576656C20697320696D706C6175738F
:1043000069626C652028302D34292E0A00000022B5
:1043100000250028002B002E00310034000201008F
:1043200000050108010B0100000A0B02090C0D0E2B
:104330000807030401000000000000000000000066
:10434000000000000000000000000000000000006D
:10435000000000121110000000000000000000002A
:1043600000000000000000000000000000204200EB
:104370002050006F6B00526573656E643A200045F3
:10438000313A200045303A20005A3A2000593A206C
:1043900000583A20004D53312C4D53322050696E55
:1043A000730A004B494C4C45442E200024F4D43071
:1043B00050C38E20C2A24017828B7011127A910DC9
:1043C000816CD90AA861E108C758660761514306A4
:1043D0001E4B5D05C145A7041A411104093D980310
:1043E000713931034036DB0265339102D430540217
:1043F000802E1D02632CEE01752AC501B028A00194
:10440000102781018F2564012B244B01E022340108
:10441000AC211F018D200D01801FFC00841EED00CA
:10442000971DDF00B81CD200E61BC600201BBC0095
:10443000641AB200B219A8000A19A0006A189900FB
:10444000D117910040178B00B516840031167E00FD
:10445000B31579003A157300C7146F0058146A0039
:10446000EE1366008813630025135E00C7125B001D
:104470006C12570015125400C111510070114F00F9
:1044800021114B00D61049008D1047004610440002
:1044900002104200C00F4000800F3E00420F3C005F
:1044A000060F3B00CB0E3800930E37005C0E350034
:1044B000270E3400F30D3200C10D3100900D300095
:1044C000600D2E00320D2D00050D2C00D90C2B0097
:1044D000AE0C2900850C29005C0C2700350C270048
:1044E0000E0C2600E80B2400C40B2400A00B2300B4
:1044F0007D0B23005A0B2100390B2100180B2000E3
:10450000F80A1F00D90A1E00BB0A1E009D0A1D00E2
:10451000800A1D00630A1C00470A1B002C0A1B00AE
:10452000110A1A00F7091A00DD091900C409190057
:10453000AB091900920917007B09180063091700DD
:104540004C09160036091600200916000A09150044
:10455000F5081500E0081400CC081400B808140091
:10456000A4081400900813007D0812006B081300C3
:1045700058081200460812003408110023081100E0
:104580001208110001081100F0071000E0071000E8
:10459000D0071000C0071000B0070F00A1071000DF
:1045A00091070E0083070F0074070F0065070E00C8
:1045B00057070E0049070E003B070D002E070E009F
:1045C00020070D0013070D0006070D00F9060C006B
:1045D000ED060D00E0060C00D4060C00C8060C0029
:1045E000BC060C00B0060C00A4060B0099060C00DB
:1045F0008D060B0082060B0077060B006C060B0085
:1046000061060A0057060B004C060A0042060A0023
:1046100038060A002E060A0024060A001A060A00B6
:104620001006090007060A00FD050900F405090047
:10463000EB050900E2050900D9050900D0050900CC
:10464000C7050900BE050900B5050800AD0508004D
:10465000A50509009C050800940508008C050800C4
:10466000840508007C050800740508006C05070037
:10467000650508005D050700560508004E050700A2
:104680004705070040050800380507003105070009
:104690002A050700230507001C050600160507006C
:1046A0000F0507000805060002050700FB040600C9
:1046B000F5040700EE040600E8040600E204070023
:1046C000DB040600D5040600CF040600C90406007A
:1046D000C3040600BD040600B7040600B1040500CB
:1046E000AC040600A6040600A00405009B04060016
:1046F00095040500900406008A0405008504050061
:10470000800406007A0405007504050070040500A5
:104710006B04050066040500610405005C040500E7
:1047200057040500520405004D0405004804050027
:10473000430405003E0404003A0405003504050066
:10474000300404002C0405002704040023040500A1
:104750001E0404001A0404001604050011040400D9
:104760000D0404000904050004040400000404000E
:10477000FC030400F8030400F4030400F003040045
:10478000EC030400E8030400E4030400E003040075
:10479000DC030400D8030400D4030400D0030400A5
:1047A000CC030400C8030300C503030024F404D9A8
:1047B000201BC40C5C0E9804C4095F0265077101DC
:1047C000F405F900FB04B30048048700C103690045
:1047D0005803550003034500BE023A00840231002D
:1047E00053022A002902250004022000E4011C00D3
:1047F000C8011900AF0117009801140084011300CB
:10480000710110006101100051010E0043010D0003
:1048100036010B002B010B0020010B0015010900D4
:104820000C01090003010800FB000800F300080068
:10483000EB000700E4000600DE000600D8000600DA
:10484000D2000600CC000500C7000500C20005002C
:10485000BD000400B9000400B5000400B10004006C
:10486000AD000400A9000400A5000300A20003009D
:104870009F0004009B0003009800030095000200C5
:1048800093000300900003008D0002008B000300E2
:1048900088000200860002008400030081000200FC
:1048A0007F0002007D0002007B0002007900020010
:1048B000770001007600020074000200720001001F
:1048C000710002006F0002006D0001006C00020028
:1048D0006A00010069000200670001006600010033
:1048E0006500010064000200620001006100010037
:1048F000600001005F0002005D0001005C0001003B
:104900005B0001005A00010059000100580001003D
:10491000570001005600010055000100540001003D
:10492000530000005300010052000100510001003B
:10493000500001004F0001004E0000004E00010039
:104940004D0001004C0001004B0000004B00010035
:104950004A00010049000100480000004800010031
:10496000470001004600000046000100450000002D
:104970004500010044000100430000004300010025
:10498000420000004200010041000000410001001F
:10499000400001003F0000003F0001003E00000019
:1049A0003E0001003D0000003D0001003C00000011
:1049B0003C0000003C0001003B0000003B00010007
:1049C0003A0000003A0001003900000039000100FF
:1049D00038000000380000003800010037000000F7
:1049E00037000100360000003600000036000100EC
:1049F00035000000350000003500010034000000E3
:104A000034000000340001003300000033000000D7
:104A100033000100320000003200000032000100CB
:104A200031000000310000003100010030000000C2
:104A300030000000300001002F0000002F000000B7
:104A40002F0000002F0001002E0000002E000000AB
:104A50002E0001002D0000002D0000002D000000A0
:104A60002D0001002C0000002C0000002C00000094
:104A70002C0001002B0000002B0000002B00000088
:104A80002B0001002A0000002A0000002A0000007C
:104A90002A00010029000000290000002900000070
:104AA0002900000029000100280000002800000063
:104AB0002800000028000000280001002700000056
:104AC0002700000027000000270000002700010049
:104AD000260000002600000026000000260000003E
:104AE0002600010025000000250000002500000030
:104AF0002500000025000000250001002400000022
:104B00002400000024000000240000002400010014
:104B10002300000023000000230000002300000009
:104B200023000000230000002300010022000000F9
:104B300022000000220000002200000022000000ED
:104B400022000100210000002100000021000000DF
:104B500021000000210000002100000021000100D0
:104B600020000000200000002000000020000000C5
:104B700020000000200000002000000020000100B4
:104B80001F0000001F0000001F0000001F000000A9
:104B90001F0000001F0000001F0001001E00000099
:104BA0001E0000001E0000001E0000004D383420D2
:104BB000582059205A2045004572723A204D494EDE
:104BC00054454D5020424544004D494E54454D50AA
:104BD00020747269676765726564004572723A2075
:104BE0004D494E54454D50204531004572723A2092
:104BF0004D494E54454D50204530004572723A2083
:104C00004D415854454D5020424544004D41585463
:104C1000454D50207472696767657265640045721E
:104C2000723A204D415854454D502045310045724F
:104C3000723A204D415854454D50204530000200F5
:104C4000002100240027002A002D0030003300013D
:104C5000010000040107010A0101021020200808D8
:104C600010204010204080020102010804020101CE
:104C700002040810204080804020100804020180B7
:104C8000040201804020100804020108040201010E
:104C90000204081020408001020408102040800512
:104CA000050505070508080808020202020A0A08A5
:104CB00008040404040101010101010101030303CB
:104CC0000303030303040707070C0C0C0C0C0C0C68
:104CD0000C0202020206060606060606060B0B0B6F
:104CE0000B0B0B0B0B1FFFFFFFFFFFFF6000000014
:104CF0000001FF400000000000FF800000000000F5
:104D00007F83CF00000C303F87FF80000C301F8670
:104D10007980000C000F8C30C7838C30E78C30CF4B
:104D2000C7CC31F38C30DCECEC33B98C30D86C6C04
:104D300033198C30D06C0C33198C30D86C0C33197F
:104D40008C30DC6C0E3B198C30CF7C079F198C307B
:104D5000C77C038F194000000000000260000000C3
:104D60000000061FFFFFFFFFFFF82020506C616E60
:104D70006E657242756666657242797465733A2033
:104D8000002046726565204D656D6F72793A20008E
:104D9000436F6D70696C65643A204E6F76203231D6
:104DA00020323031370A00207C20417574686F72E0
:104DB0003A2028416C657068204F626A656374739D
:104DC00020496E632E2C204C756C7A426F742047FC
:104DD0006974205265706F7369746F7279290A0063
:104DE0004E6F76203231203230313731333A343021
:104DF0003A333700204C61737420557064617465D8
:104E0000643A2000312E312E350A004D61726C69F2
:104E10006E0020536F66747761726520526573650A
:104E2000740A00205761746368646F672052657369
:104E300065740A002042726F776E206F757420527D
:104E4000657365740A002045787465726E616C2024
:104E500052657365740A00506F77657255700A0069
:104E600073746172740A006572726F72207772696E
:104E700074696E6720746F2066696C650A004572FC
:104E8000726F723A00456E6473746F70732025639D
:104E900020256320256320256300205A3A002059ED
:104EA0003A0020583A00656E6473746F707320681E
:104EB00069743A20006563686F3A00446F6E65203C
:104EC000736176696E672066696C652E0A004D32E3
:104ED0003900656E7175657565696E672022004DD4
:104EE00036303020486F74656E6420746F6F2063B5
:104EF0006F6C6420746F206368616E6765206669FB
:104F00006C616D656E740A004B64200023646566F5
:104F1000696E65202044454641554C545F004B69FD
:104F2000200023646566696E65202044454641552E
:104F30004C545F004B70200023646566696E6520E9
:104F40002044454641554C545F005049442041752A
:104F5000746F74756E652066696E69736865642127
:104F60002050757420746865206C617374204B70D8
:104F70002C204B6920616E64204B6420636F6E733C
:104F800074616E74732066726F6D2062656C6F77EA
:104F900020696E746F20436F6E6669677572617405
:104FA000696F6E2E680A00504944204175746F7411
:104FB000756E65206661696C6564212074696D6534
:104FC0006F75740A00504944204175746F74756E92
:104FD00065206661696C6564212054656D70657239
:104FE000617475726520746F6F20686967680A0064
:104FF000204B643A2000204B693A2000204B703A45
:1050000020000A20436C6173736963205049442077
:105010000A002054753A2000204B753A2000206D7C
:1050200061783A2000206D696E3A200020643A20B1
:105030000020626961733A200020496E76616C69D4
:10504000642065787472756465722000290A0020F6
:1050500062797465733B20637263200053657474D6
:10506000696E67732053746F726564202800205A3C
:105070003A0020593A0020436F756E7420583A0068
:1050800020453A00205A3A0020593A00583A002068
:105090005A00205900580020204D61783A20002005
:1050A0005A00205900580020204D696E3A20004FC8
:1050B0006E20004F666600536F667420656E6473E1
:1050C000746F70733A200020643A0020693A00201F
:1050D000703A00526573746F7265206661696C7313
:1050E000616665004D3530320A4D353030004C6F09
:1050F00061642073657474696E67730053746F72B2
:10510000652073657474696E677300416476616EBF
:105110006365642053657474696E6773004D6169DB
:105120006E00536C6565702E2E2E005072696E7481
:105130002061626F727465640041626F757420460D
:1051400069726D77617265004E6F20534420636110
:105150007264005072696E742066726F6D205344E1
:105160000053746F70207072696E740052657375AD
:105170006D65207072696E74005061757365207082
:1051800072696E7400436F6E6669677572617469E7
:105190006F6E0054656D7065726174757265004D57
:1051A0006F76656D656E74004368616E6765206635
:1051B000696C616D656E740054756E6500496E664C
:1051C0006F2073637265656E00202F002042403AA5
:1051D0000020403A006F6B004E6F204C696E6520D6
:1051E0004E756D62657220776974682063686563C7
:1051F0006B73756D2C204C617374204C696E653A2D
:10520000200053544F505045442E20005072696E78
:105210007465722073746F707065642064756520A6
:10522000746F206572726F72732E204669782074D5
:105230006865206572726F7220616E642075736597
:10524000204D39393920746F20726573746172741E
:105250002E202854656D70657261747572652069C1
:10526000732072657365742E2053657420697420F1
:1052700061667465722072657374617274696E67B9
:10528000290A004E6F20436865636B73756D207744
:10529000697468206C696E65206E756D6265722C2C
:1052A000204C617374204C696E653A200063686518
:1052B000636B73756D206D69736D617463682C2009
:1052C0004C617374204C696E653A20004C696E65C0
:1052D000204E756D626572206973206E6F74204C6C
:1052E000617374204C696E65204E756D6265722B1A
:1052F000312C204C617374204C696E653A20004D4E
:10530000313130004D3331004D3834205820592090
:105310005A20450053442072656164206572726FA3
:10532000720A00446F6E65207072696E74696E67F0
:105330002066696C650A004B494C4C45442E2000A0
:105340004B494C4C20636175736564206279204B36
:10535000494C4C20627574746F6E2F70696E0A0030
:105360004B494C4C45442E20004B494C4C2063612A
:105370007573656420627920746F6F206D75636842
:1053800020696E6163746976652074696D65202D8E
:105390002063757272656E7420636F6D6D616E64EB
:1053A0003A2000000020002300260029002C002FB6
:1053B0000032000001000003010601090100008025
:1053C000C10000A0C10000000000009643008097CB
:1053D00043008095434F66667365747320617070F7
:1053E0006C696564004572723A20546F6F20666183
:1053F000722100546F6F206661722066726F6D209B
:105400007265666572656E636520706F696E740A99
:105410000048617264636F64656420446566617509
:105420006C742053657474696E6773204C6F61648B
:1054300065640A0028230000282300000A000000F9
:105440001027000000009643000096430000204112
:105450000000C8410000C9420000C942A5C2DF44A3
:105460000000D243202863616C63756C61746564CD
:1054700029210A0020213D2000454550524F4D2052
:10548000435243206D69736D61746368202D202839
:1054900073746F726564292000290A002062797490
:1054A00065733B2063726320002073746F726564C0
:1054B0002073657474696E677320726574726965B0
:1054C000766564202800204D61726C696E3D56340B
:1054D00030290A0028454550524F4D3D0045455062
:1054E000524F4D2076657273696F6E206D69736DD2
:1054F0006174636820005A204F66667365740046C5
:105500006C6F7700466C6F770046616E2073706534
:10551000656420310046616E2073706565642031DA
:105520000042656400426564004E6F7A7A6C6500E3
:105530004E6F7A7A6C6500537065656400537065D0
:105540006564004D61696E00416D617820450041E0
:105550006D6178204500416D6178205A00416D6190
:1055600078205A00416D6178205900416D617820A2
:105570005900416D6178205800416D6178205800D4
:10558000412D74726176656C00412D74726176658F
:105590006C00412D7265747261637400412D7265F7
:1055A000747261637400416363656C004163636599
:1055B0006C004D6F74696F6E00436F6F6C646F7732
:1055C0006E0046616E20737065656420310046612F
:1055D0006E20737065656420310042656400426529
:1055E00064004E6F7A7A6C65004E6F7A7A6C650053
:1055F0004D61696E004E414E494E495459494E46DF
:10560000CDCCCC3D0AD7233C17B7D13877CC2B3241
:105610009595E6241FB14F0A000020410000C842C2
:1056200000401C4620BCBE4CCA1B0E5AAEC59D7421
:10563000D40097CF11241FBECFEFD1E2DEBFCDBF84
:1056400000E00CBF14E0A0E0B2E0EAE6F4E402E01F
:105650000BBF02C007900D92A831B107D9F725E121
:10566000A8E1B4E001C01D92AE35B207E1F716E53E
:10567000C2E3D6E500E006C022970109FE010BBF98
:105680000F94B521C033D10780E00807A9F70E9425
:10569000E1CF0D9424220C9400002F923F924F9260
:1056A0005F926F927F928F929F92AF92BF92CF92B2
:1056B000DF92EF92FF920F931F93CF93DF93CDB7BB
:1056C000DEB7C958D1090FB6F894DEBF0FBECDBF03
:1056D0000091631020E6029F800111240D51114FAB
:1056E00080919D0680FF1AC0E5EBFEE484917F0166
:1056F0003FEFE31AF30A811102C0780104C00E944F
:10570000857FF701F3CFD7018D917D01882319F0B3
:105710000E94857FF8CF8AE00E94857F10925F0605
:1057200010925E068FE380939C0610929B06109267
:105730009A0610923204109233041092340410929C
:105740003504F80180810F5F1F4F8032D1F38E3412
:10575000B1F4818190ED980F9A3020F08D3211F0E4
:105760008B3269F43296DF0131962C9120532A3026
:10577000D0F3CD01FC01019620812032D9F3F093C2
:105780009406E09393067F01BFEFEB1AFB0A1081AA
:105790006AE270E0C7010F94F521009739F0DC014F
:1057A00011978C918032E1F311961C921D3429F0EF
:1057B000143519F0173409F0CAC0F7014E2F9F2F86
:1057C00081918032D9F380538A3008F0C0C01093A1
:1057D0009C0620919A0630919B06E42FF92F6AE0EF
:1057E000AF014F5F5F4F629FC001639F900D112417
:1057F000208130E020533109820F931F21812053F3
:105800002A3030F090939B0680939A069A0103C049
:105810009C01FA01E5CFD9012F5F3F4F4C914032F7
:10582000D1F31D34D1F48E31910591F03CF48731E0
:10583000910571F08C31910581F40AC0853791058D
:1058400064F08737910524F0803AE3E09E0729F45D
:10585000B0935F06A0935E067AC010925F06109226
:105860005E06D090930641E050E0FD0131962C9108
:10587000222309F46CC02132A1F41D3491F480324A
:10588000910579F4F0935F06E0935E0663E270E0C1
:10589000CF010F94F521009709F459C0DC011C9247
:1058A00056C00FEB020F0A31A0F59F01F90160818C
:1058B0002F5F3F4F6032D1F320ED260F2A3040F0AA
:1058C00023ED260F223020F06B3211F00C94B441FE
:1058D0009F01602F70E0DB01B595A795B595A79561
:1058E000B595A795AE5CBB4F07707A01002E01C03D
:1058F000EE0C0A94EAF7FC90FE28FC922115310583
:1059000011F02D1901C020E0DB01A85EBB4F2C93E4
:105910000AC020915E0630915F06232B21F4B093DC
:105920005F06A0935E06208121542A3110F4DF0126
:105930009CCFDF0131966C9160536A30D0F39D01AA
:10594000F9012F5F3F4F60816032D1F3F0CF80913A
:105950009C068D3409F4A0C7843511F40C9457418A
:10596000873411F00C94974180919A0690919B0690
:105970008A31910509F449C6BCF4843091055CF480
:105980008230910574F597FF02C00C94B1410E94DA
:10599000FD6E0C94B1418430910509F4F0C50C976B
:1059A00009F4F1C50C94B1418E31910509F4C2C6D8
:1059B0003CF48C31910509F4B4C60CF42DC6B6C67E
:1059C0008B35910509F45FC78C35910509F460C7E3
:1059D0008A35910511F00C94B141109299060C94FE
:1059E000B14120911402222311F40C94B14111E031
:1059F000029709F010E00E94FFAE82E50F94ED02DD
:105A0000882309F45CC10F94E3006B017C01409092
:105A1000B10E5090B20E6090B30E7090B40E209103
:105A2000B50E3091B60E4091B70E5091B80E6396F8
:105A30002CAF3DAF4EAF5FAF63978091360490912E
:105A40003704A0913804B091390467968CAF9DAFAC
:105A5000AEAFBFAF679720913A0430913B044091BD
:105A60003C0450913D046F962CAF3DAF4EAF5FAFFD
:105A70006F9720E030E0A901C701B6010F945C1ACE
:105A8000882309F462C5A301920167966CAD7DADD0
:105A90008EAD9FAD67970F945C1A811111C063960C
:105AA0002CAD3DAD4EAD5FAD63976F966CAD7DADEA
:105AB0008EAD9FAD6F970F945C1A882309F445C58E
:105AC00020E030E0A901C701B6010F945C1A881FDD
:105AD0008827881F181759F080E090E0A0E8BFEBF6
:105AE000AB968CAF9DAFAEAFBFAFAB970AC020E017
:105AF00030E040E85FE3AB962CAF3DAF4EAF5FAF19
:105B0000AB97A301920167966CAD7DAD8EAD9FAD55
:105B100067970F94BF1EA3966CAF7DAF8EAF9FAFFC
:105B2000A39763962CAD3DAD4EAD5FAD63976F9679
:105B30006CAD7DAD8EAD9FAD6F970F94BF1EA796D8
:105B40006CAF7DAF8EAF9FAFA797A3962CAD3DAD49
:105B50004EAD5FADA397CA01B9010F94C11A4B01B5
:105B60005C01A7962CAD3DAD4EAD5FADA797CA01C8
:105B7000B9010F94C11A9B01AC01C501B4010F9486
:105B8000C01E0F942B216B966CAF7DAF8EAF9FAF75
:105B90006B9720E030E040E05FE30F94C11A4B01C7
:105BA0005C01A7019601C701B6010F94C11A6B01F0
:105BB0007C01A5019401C501B4010F94C11A9B0198
:105BC000AC01C701B6010F94BF1E0F942B219B019E
:105BD000AC01AB966CAD7DAD8EAD9FADAB970F9428
:105BE000C11A4B015C0167962CAD3DAD4EAD5FAD6A
:105BF0006797C301B2010F94C01E20E030E040E07F
:105C00005FE30F94C11A6B017C01A7966CAD7DAD6B
:105C10008EAD9FADA79790586B962CAD3DAD4EAD18
:105C20005FAD6B970F949C1F9B01AC01C501B40144
:105C30000F94C11A9B01AC01C701B6010F94C01E9D
:105C4000A30192010F94BF1E6B017C016F962CADD6
:105C50003DAD4EAD5FAD6F9763966CAD7DAD8EADD6
:105C60009FAD63970F94C01E20E030E040E05FE3FB
:105C70000F94C11A2B013C016B962CAD3DAD4EAD7E
:105C80005FAD6B97A3966CAD7DAD8EAD9FADA397C9
:105C90000F949C1F9B01AC01C501B4010F94C11A64
:105CA0009B01AC01C301B2010F94C01E63962CADE1
:105CB0003DAD4EAD5FAD63970F94BF1E14C089E438
:105CC0000F94ED02882329F00F94E3006B017C010F
:105CD00003C0C12CD12C76018AE40F94ED028823F5
:105CE000F9F00F94E3006F966CAF7DAF8EAF9FAF6E
:105CF0006F9720E030E0A901C701B6010F945C1A4C
:105D000081111EC020E030E0A9016F966CAD7DAD21
:105D10008EAD9FAD6F970F945C1A811111C015C4A1
:105D200020E030E0A901C701B6010F945C1A882376
:105D300009F40BC46F961CAE1DAE1EAE1FAE6F975E
:105D4000D701C601B05863968CAF9DAFAEAFBFAF61
:105D500063976F962CAD3DAD4EAD5FAD6F975058CC
:105D600067962CAF3DAF4EAF5FAF67979C01AD011B
:105D7000BC01CD010F94C11A4B015C0167962CAD9B
:105D80003DAD4EAD5FAD6797CA01B9010F94C11A21
:105D90009B01AC01C501B4010F94C01E0F942B21CF
:105DA000EB966CAF7DAF8EAF9FAFEB978091B10E4E
:105DB0009091B20EA091B30EB091B40EA3968CAF99
:105DC0009DAFAEAFBFAFA397A7019601BC01CD01B8
:105DD0000F94C01EAB966CAF7DAF8EAF9FAFAB97ED
:105DE0002091B50E3091B60E4091B70E5091B80E7D
:105DF000A7962CAF3DAF4EAF5FAFA7976F962CAD78
:105E00003DAD4EAD5FAD6F97A7966CAD7DAD8EADE0
:105E10009FADA7970F94C01EAF966CAF7DAF8EAFAE
:105E20009FAFAF978091360490913704A0913804CA
:105E3000B0913904E3968CAF9DAFAEAFBFAFE3979F
:105E4000AB962CAD3DAD4EAD5FADAB97BC01CD017A
:105E50000F94BF1E6B017C0120913A0430913B04EA
:105E600040913C0450913D04E7962CAF3DAF4EAFBE
:105E70005FAFE797AF962CAD3DAD4EAD5FADAF9741
:105E8000E7966CAD7DAD8EAD9FADE7970F94BF1ECD
:105E90004B015C018091B90E9091BA0EA091BB0E9E
:105EA000B091BC0EC158DF4F88839983AA83BB830E
:105EB000CF57D0409C01AD0160913E0470913F04EA
:105EC00080914004909141040F94BF1E6B966CAF7B
:105ED0007DAF8EAF9FAF6B972091BD0E3091BE0E00
:105EE0004091BF0E5091C00ECD57DF4F28833983AC
:105EF0004A835B83C358D04060914204709143044D
:105F000080914404909145040F94BF1EEF966CAFAE
:105F10007DAF8EAF9FAFEF97A701960163966CADF3
:105F20007DAD8EAD9FAD63970F94C11A2B013C01DF
:105F3000A501940167966CAD7DAD8EAD9FAD679761
:105F40000F94C11A9B01AC01C301B2010F94C01E92
:105F50002B013C01A501940163966CAD7DAD8EAD26
:105F60009FAD63970F94C11A4B015C01A701960185
:105F700067966CAD7DAD8EAD9FAD67970F94C11ADE
:105F80009B01AC01C501B4010F94BF1EA301920196
:105F90000F94331F6B017C0120E030E0A9010F94C6
:105FA0005C1A87FF0AC02BED3FE049EC50E4C701C3
:105FB000B6010F94C01E6B017C01112351F02BED33
:105FC0003FE049EC50E4C701B6010F94BF1E6B01DE
:105FD0007C0120E030E0A901C701B6010F945C1AF2
:105FE000811128C0E3962CAD3DAD4EAD5FADE3977A
:105FF000A3966CAD7DAD8EAD9FADA3970F945C1A4B
:10600000811118C0E7962CAD3DAD4EAD5FADE79761
:10601000A7966CAD7DAD8EAD9FADA7970F945C1A22
:10602000811108C08BEDC82E8FE0D82E89ECE82EA8
:1060300080E4F82EEB962CAD3DAD4EAD5FADEB9709
:10604000C701B6010F94C11A9B01AC010F94C11A8C
:106050004B015C016B962CAD3DAD4EAD5FAD6B97CA
:10606000CA01B9010F94C11A9B01AC01C501B40169
:106070000F94C01E0F942B214B015C012FE632E1DF
:1060800043E85AE30F945C1A87FD5BC2C501B40173
:106090000F9435200F9409201B016115710519F427
:1060A00022242394312CB10180E090E00F94601AF7
:1060B0004B015C019B01AC01C701B6010F949C1F11
:1060C000A3966CAF7DAF8EAF9FAFA397A501940150
:1060D0006B966CAD7DAD8EAD9FAD6B970F949C1F95
:1060E000EB966CAF7DAF8EAF9FAFEB97A5019401A0
:1060F000EF966CAD7DAD8EAD9FADEF970F949C1F6D
:10610000EF966CAF7DAF8EAF9FAFEF97A3962CADA0
:106110003DAD4EAD5FADA397CA01B9010F94C11A51
:1061200020E030E040E05FE30F94C11A9B01AC0136
:1061300060E070E080E89FE30F94BF1EE3966CAFD1
:106140007DAF8EAF9FAFE397C158DF4F88819981B4
:10615000AA81BB81CF57D04089879A87AB87BC87FC
:10616000CD57DF4F288139814A815B81C358D040A8
:106170002D873E874F87588B6091A6027091A702AA
:10618000882777FD8095982F0F94621A20910A0234
:1061900030910B0240910C0250910D020F94C11AE4
:1061A0002AE037ED43E25CE30F94C11AE7966CAF47
:1061B0007DAF8EAF9FAFE7970F94A204DC01CB01B8
:1061C00088539F4FAF4FBF4F6B968CAF9DAFAEAF15
:1061D000BFAF6B9760964FAC609761965FAC61976D
:1061E00062966FAC629763967FAC6397A1E0B0E074
:1061F000A596BFAFAEAFA59719E1B12EA5962EAD6E
:106200003FADA5972215330508F057C10E94AB8812
:106210000F94A2046B962CAD3DAD4EAD5FAD6B9768
:10622000621B730B840B950B97FD11C00F94A20496
:10623000DC01CB0188539F4FAF4FBF4F6B968CAFA4
:106240009DAFAEAFBFAF6B9780E00E946BFCBA947E
:1062500009F44FC0E3962CAD3DAD4EAD5FADE39775
:1062600067966CAD7DAD8EAD9FAD67970F94C11AEB
:106270006B017C01A3962CAD3DAD4EAD5FADA397F8
:10628000B201C3010F94C11AA70196010F94C01E59
:10629000162FA72E982E892EE3962CAD3DAD4EAD30
:1062A0005FADE397B201C3010F94C11A6B017C018A
:1062B000A3962CAD3DAD4EAD5FADA39767966CAD8B
:1062C0007DAD8EAD9FAD67970F94C11A9B01AC0158
:1062D000C701B6010F94BF1E2B013C01812F9A2DDF
:1062E000A92DB82D67968CAF9DAFAEAFBFAF6797A6
:1062F0005FC0A596AEADBFADA597BD0180E090E0B3
:106300000F94601AA3962CAD3DAD4EAD5FADA39733
:106310000F94C11A4B015C010F94991F6B017C0112
:10632000C501B4010F9421214B015C01A701960125
:1063300063966CAD7DAD8EAD9FAD63970F94C11A22
:106340002B013C01A50194016F966CAD7DAD8EAD26
:106350009FAD6F970F94C11A9B01AC01C301B201AD
:106360000F94C01E2B013C01A501940163966CADF6
:106370007DAD8EAD9FAD63970F94C11A4B015C014B
:10638000A70196016F966CAD7DAD8EAD9FAD6F97F9
:106390000F94C11A9B01AC01C501B4010F94BF1E3B
:1063A00067966CAF7DAF8EAF9FAF6797B9E1BB2E9D
:1063B0009201A301AB966CAD7DAD8EAD9FADAB9759
:1063C0000F94C01E69837A838B839C8367962CAD60
:1063D0003DAD4EAD5FAD6797AF966CAD7DAD8EAD0B
:1063E0009FADAF970F94C01E6D837E838F83988778
:1063F000EB962CAD3DAD4EAD5FADEB9769857A85E3
:106400008B859C850F94C01E69877A878B879C87B4
:10641000EF962CAD3DAD4EAD5FADEF976D857E85B2
:106420008F8598890F94C01E6D877E878F87988B84
:10643000CE0101960F946501C090920689819A81E0
:10644000AB81BC8188A399A3AAA3BBA38D819E81A4
:10645000AF81B8858CA39DA3AEA3BFA389859A8580
:10646000AB85BC8588A799A7AAA7BBA7AE01485D45
:106470005F4FBE016C5D7F4FCE0180960E9474DD40
:10648000E796ECACFDAC0EAD1FADE7979E01235F28
:106490003F4FAE01485D5F4FBE016C5D7F4FCE0147
:1064A00080960E94DA5EA596EEADFFADA597319677
:1064B000A596FFAFEEAFA597A1CEC09092068091B2
:1064C000360490913704A0913804B091390488A320
:1064D00099A3AAA3BBA380913A0490913B04A091F5
:1064E0003C04B0913D048CA39DA3AEA3BFA38091B7
:1064F0003E0490913F04A0914004B091410488A7CC
:1065000099A7AAA7BBA7AE01485D5F4FBE016C5D0E
:106510007F4FCE0180960E9474DDE796ECACFDAC17
:106520000EAD1FADE79722E434E0AE01485D5F4F4A
:10653000BE016C5D7F4FCE0180960E94DA5E0F94A3
:10654000C4010F94D7040C94B141EEE7FEE48491AA
:106550008F010F5F1F4F882321F00E94857FF80174
:10656000F6CFE4E0F2E084918F010F5F1F4F8823A4
:1065700011F40C94B1410E94857FF801F4CF0E9480
:1065800006F90C94B1410E942AAE81110C94B141DC
:1065900080E50F94ED02882319F00F94B30001C039
:1065A00060E06FAF83E50F94ED02882319F00F943C
:1065B000B30001C06CE06BAF84E50F94ED0288235B
:1065C00019F00F94B30001C063E068A382E50F9453
:1065D000ED02882319F00F94E30004C060E070E03E
:1065E00080ED90E469837A838B839C839E01205E97
:1065F0003F4FAE014F5F5F4FBE01655C7F4FCE01E5
:10660000CF960E9433F30C94B14181E08093140241
:10661000109291060C94B1410E942AAE81110C9403
:10662000B14180E50F94ED02882321F00F94B3006F
:10663000462F01C040E06091B90E7091BA0E809172
:10664000BB0E9091BC0E00E010E020EC30EC098312
:106650001A832B833C8300E010E822E933E40D83A6
:106660001E832F83388700E010E020EA31E4098799
:106670001A872B873C8700E010E020EC3FE70D876E
:106680001E872F87388B413089F1423039F518A2A7
:1066900019A21AA21BA220E030E040EA51E40F94B4
:1066A000C01E7B018C0120E030E845E953E40F94E3
:1066B000E62018162CF4E12C80E805E913E401C06B
:1066C0008F2D4E2D582FB8014BAF5CAF6DAF7EAF05
:1066D000BE01605E7F4FCE01CB9611C020E030E05E
:1066E00040EA51E40F945C1A87FF0BC018A219A26C
:1066F0001AA21BA2BE01605E7F4FCE0109960E94C6
:106700002CF318A219A21AA21BA2AE01405E5F4F81
:10671000BE016B5F7F4FCE0101960E9428F30C945F
:10672000B14180E00E94719D0C94B1410E94E4B39C
:106730000C94B14120E030E0A9016091B10E70915C
:10674000B20E8091B30E9091B40E0F94C01E182F0C
:1067500088E5C957DF4F6883C758D040C857DF4F17
:106760007883C858D040C757DF4F9883C958D04066
:106770000F94ED02C957DF4F6881C758D040C85702
:10678000DF4F7881C858D040C757DF4F9881C9582C
:10679000D040882321F00F94E3009B0102C09B01AD
:1067A000812FA901BC0148A359A36AA37BA320E0C0
:1067B00030E0A9016091B50E7091B60E8091B70ED0
:1067C0009091B80E0F94C01E5B018C0189E50F9467
:1067D000ED02882321F00F94E3005B018C01A501F9
:1067E000B80149835A836B837C8340904A0450905C
:1067F0004B0460904C0470904D04209146043091FD
:106800004704409148045091490468A179A18AA1A4
:106810009BA10F94BF1E6B017C012CE032E040E88D
:1068200051EC0F94E62087FF02C00C94B14121E2A5
:1068300030E046E953E4C701B6010F945C1A18161C
:1068400014F40C94B141A3019201B501C8010F9455
:10685000BF1E6B017C012CE032E040EA51EC0F944A
:10686000E62087FF02C00C94B14121E230E847E9FD
:1068700053E4C701B6010F945C1A181614F40C9473
:10688000B1410C94C54181E0809399060C94B141CB
:106890000E9458F60C94B14180919A0690919B0603
:1068A0008837910511F40C949A3C0CF0D4C08D34C7
:1068B000910509F4A2C40CF056C08931910509F480
:1068C000CAC21CF58431910509F455C27CF48131AA
:1068D000910509F445C22CF4029708F4BEC10C944A
:1068E000B141429709F4ECC60C94B141863191054F
:1068F00009F488C20CF482C28731910509F488C278
:10690000489709F489C20C94B1418F31910509F47B
:1069100025C47CF48B31910509F4B9C20CF4A9C2E9
:106920008C31910509F4EFC24E9709F4F0C20C9432
:10693000B1418A32910509F415C444F4809711F0ED
:106940000C94B1410E9412F60C94B1418B34910524
:1069500009F44FC48C34910511F00C94B1410E949C
:106960009DAF0C94B1418A36910509F4F4C5CCF57C
:106970008435910509F4A4C6CCF48135910509F458
:1069800082C634F48E34910509F43BC40C94B141B1
:106990008235910509F491C68335910511F00C9467
:1069A000B14181E0809398060C94B1418C359105FA
:1069B00009F4BBC64CF48535910511F00C94B14136
:1069C0000F94D7020C94B1418836910509F42BC578
:1069D0008936910511F00C94B1410E94A3FF0C94EB
:1069E00099458237910509F4A3C6DCF48D369105EB
:1069F00009F485C54CF48B36910511F00C94B14126
:106A00000F94F9020C94B1418E36910509F457C5E3
:106A10008F36910511F00C94B1410E94C27F0C9405
:106A2000B1418537910509F488C64CF48337910547
:106A300011F00C94B1410E94A0800C94B1418637B2
:106A4000910509F482C68737910511F00C94B14184
:106A5000EAE5F4E07DC68F3231E0930711F40C943F
:106A6000BF3E0CF077C08C3C910509F4E8C7ECF50B
:106A70008B39910509F440C5ECF48D37910509F483
:106A80008DC55CF48937910511F00C94B1411092D9
:106A9000A00E109260060C94B1418C38910509F457
:106AA00011C58139910511F00C94B1410E942D80DE
:106AB0000C94B141883C910509F442C734F48E3BF3
:106AC000910509F434C50C94B141893C910509F450
:106AD0007FC78B3C910511F00C94B1410CE213E09F
:106AE00027E6E22E26E0F22E9BC78D3D910511F49C
:106AF0000C949F3DA4F48E3C910511F40C948C3DB4
:106B000014F40C94893D833D910511F40C948F3D50
:106B10008C3D910511F40C94923D0C94B1418C3252
:106B200051E0950711F40C94E63D3CF4823E91054A
:106B300011F40C94A23D0C94B1418D32B1E09B074D
:106B400011F40C94E93D8E32914011F40C94693E9D
:106B50000C94B141843FF1E09F0711F40C94223F63
:106B6000E4F5803931E0930711F40C94C23EECF463
:106B70008E3551E0950711F40C94BF403CF48033FE
:106B8000914011F40C94EC3D0C94B1418F35E1E04F
:106B90009E0711F40C94F3408336914011F00C944D
:106BA000B1410E9452810C94B141823921E0920797
:106BB00011F40C94C93E14F40C94C53E843A41E09F
:106BC000940711F40C94CD3E8C3A914011F00C9442
:106BD000B1410F94900D0C94B1418835A2E09A0711
:106BE00011F40C94773FB4F4863FE1E09E0711F472
:106BF0000C94283F14F40C94253F873F21E0920722
:106C000011F40C942B3F8C31924011F40C94393FC9
:106C10000C94B1418C3843E0940711F40C94A540D6
:106C200084F48335A3E09A0711F40C94443F8B3825
:106C3000934011F00C94B1410CE213E0F12C0C9450
:106C40007E40803AE3E09E0709F484C2873E934089
:106C500011F40C9445410C94B14100915E061091E1
:106C60005F0680E50F94ED02882369F00F94A3007E
:106C70006B017C01BB24B3946115710581059105FD
:106C800031F4B12C04C0B12CC12CD12C760183E598
:106C90000F94ED028823F9F00F94E30020E030E038
:106CA0004AE754E40F94C11A0F9409206B017C0148
:106CB000B11013C0611571058105910571F40115BD
:106CC000110559F0D8018C91882339F061E0C80191
:106CD0000E94BBDE07C0BB2091F360E080E592E03C
:106CE0000E94CBDE81E08093BB080F9419050F94BE
:106CF000D704C114D104E104F104D1F0809052040E
:106D000090905304A0905404B09055048C0C9D1C9A
:106D1000AE1CBF1C0F94A204681979098A099B094B
:106D200097FF1AC08091BB0881110C941B4214C0BC
:106D30008091BB08882321F080E00E946BFCF8CF93
:106D40008091A71260E0882319F081E492E002C0EC
:106D50008CE292E00E94CBDE1092BB080C94B14111
:106D600060E083E692E00E94CBDE179816981598B3
:106D700014980C94B141EBE7F2E084918F010F5F1E
:106D80001F4F882321F00E94857FF801F6CF1092D3
:106D9000531540E050E0BA018FEF92E10E94D9AB69
:106DA0008BE1EFEFF2E1DE01159601900D928A95ED
:106DB000E1F78091FD129091FE129C838B8384E217
:106DC00093E09A83898340E050E0BE016F5F7F4F7C
:106DD00088EA93E00E949892CE0101960E944A545C
:106DE000ECE6F2E084918F010F5F1F4F882311F4CE
:106DF0000C94B1410E94857FF801F4CF0E940852A3
:106E00000C94B1411092A7121092A8120C94B141A7
:106E10000E942A770C94B14119821A821B821C822B
:106E200018A219A21AA21BA280919006882341F0F1
:106E300040E0BE016F5F7F4FCE0180960E94B8E6B2
:106E40008091A812882319F081E08093A7120E94F4
:106E5000A6C40C94B1411092A7120E949DAF8CE879
:106E600092E09093400980933F090E9432740C9401
:106E7000B1418091A812882311F40C94B14183E5AB
:106E80000F94ED0281110C9420420C94B141809139
:106E9000A812882351F1E1E9F2E084918F010F5F9C
:106EA0001F4F882321F00E94857FF801F6CF609163
:106EB0004A1570914B1580914C1590914D154AE0F3
:106EC0000E94A0C28FE20E94857F6091461570915A
:106ED000471580914815909149154AE00E94A0C23B
:106EE0008AE00E94857F0C94B141E3EAF2E084914C
:106EF0008F010F5F1F4F882311F40C94B1410E9442
:106F0000857FF801F4CF0E9422770C94B1418091E3
:106F1000A812882311F40C94B14189E994E10E94EC
:106F2000F34D89E994E10E94F6511092A612109255
:106F3000A512E0905E06F0905F068091A81288236B
:106F400011F40C94B1410E94FE511D8218861C82DE
:106F50001B8284E293E09A8389838BEF92E1909382
:106F60001B1380931A13F70180818F3209F06BC0D5
:106F70006FE270E0C7010F94F5218C010F5F1F4F86
:106F80009E012F5F3F4F59010115110509F461C0A2
:106F90006FE270E0C8010F94F5216C01009709F4CD
:106FA00059C00817190708F055C04C01801A910AFA
:106FB000A401B801CE0180960F941522E0E2F0E022
:106FC000EC0FFD1FE80DF91D10828E01005E1F4FB2
:106FD000D8018D918D01882319F00E94857FF8CF0B
:106FE0008AE00E94857F60911A1370911B136115CE
:106FF000710519F06C5F7F4F02C060E070E021E026
:10700000AE01405E5F4FCE0105960E94555381113F
:1070100012C0BE01605E7F4F8AED92E00E945AD698
:107020008EE20E94857F8AE00E94857FC5010E94D2
:107030004A540C94B141B0921B13A0921A138601CA
:107040000F5F1F4FA1CF8CE193E190931B138093AF
:107050001A13870160911A1370911B136115710542
:1070600019F06C5F7F4F02C060E070E018A21BA2B5
:1070700022E0A801CE0180960E945553F82E882365
:1070800011F1CE0180960E94314EF82E8823D9F05E
:107090006CA57DA58EA59FA541E00E9450A8F82E65
:1070A000882389F0E8A9B0E2EB9FF0011124EA5AA5
:1070B000FB4F309739F085EE80831BA20E9412A807
:1070C000F82E01C0F12CCE0180960E945053FF2073
:1070D00011F1A4EBEA2EA2E0FA2EF70184918823A5
:1070E00031F0FFEFEF1AFF0A0E94857FF6CFD8013B
:1070F0008D918D01882319F00E94857FF8CF8AE059
:107100000E94857F10924A1510924B1510924C15D3
:1071100010924D1519C0F2ECEF2EF2E0FF2EF701A0
:107120008491882331F0FFEFEF1AFF0A0E94857FD8
:10713000F6CFD8018D918D01882319F00E94857FAB
:10714000F8CF8EE20E94857FCE0101960E944A54BC
:107150000C94B1410E943E770C94B1410E94C157FA
:107160000C94B14183E50F94ED02882311F40C9443
:10717000B1410F94C300E82E80E50F94ED028823FF
:1071800011F40C94B14180E50F94ED02882341F095
:107190000F94B30077FF02C00C94B1418B0102C081
:1071A0000DE010E0802FEEEEF2E09491891739F0B7
:1071B0003196B3E0E631FB07C1F70C943142EEE7BC
:1071C000FEE484918F010F5F1F4F882321F00E94FE
:1071D000857FF801F6CFE6E1F3E084918F010F5F40
:1071E0001F4F882311F40C94B1410E94857FF80150
:1071F000F4CF0E94A6C40C94B1410E94CC830C949D
:10720000B14183E50F94ED02882359F00F94B30048
:107210006E34710531F48DE792E10E9472E90C94AD
:10722000B14118A219A21AA21BA2E5E8F3E08491C9
:107230008F010F5F1F4F882321F00E94857FF80187
:10724000F6CFECE7F3E084918F010F5F1F4F8823A7
:1072500021F00E94857FF801F6CF60918A1270912B
:107260008B1280E090E04AE00E94A0C2EFE6F3E0DB
:1072700084918F010F5F1F4F882321F00E94857F2B
:10728000F801F6CF60918C1270918D1280E090E041
:107290004AE00E94A0C2E4E6F3E084918F010F5F10
:1072A0001F4F882321F00E94857FF801F6CF80913F
:1072B0008A1290918B1220918C1230918D12821B28
:1072C000930B40917D12415021E030E0423010F0AC
:1072D00020E030E0BC01621B730B80E090E04AE0EC
:1072E0000E94A0C28AE00E94857FECE5F3E08491D1
:1072F0008F010F5F1F4F882321F00E94857FF801C7
:10730000F6CF80918E1290918F12A0919012B09131
:10731000911288A399A3AAA3BBA3BE016F5F7F4F5D
:10732000CE0180960E940D57EFE4F3E084918F0127
:107330000F5F1F4F811104C08E010F5F1F4F04C0EC
:107340000E94857FF801F2CFF80181918F01882397
:1073500019F00E94857FF8CF80919212909193123C
:10736000A0919412B091951288A399A3AAA3BBA34C
:10737000BE016F5F7F4FCE0180960E940D57EFE3F5
:10738000F3E084918F010F5F1F4F811104C08E01C4
:107390000F5F1F4F04C00E94857FF801F2CFD80114
:1073A0008D918D01882319F00E94857FF8CF8AE0A6
:1073B0000E94857FE7E3F3E084918F010F5F1F4F09
:1073C000882321F00E94857FF801F6CFE7E2F3E001
:1073D00084918F010F5F1F4F882321F00E94857FCA
:1073E000F801F6CF20E030E04AE754E460919612CD
:1073F0007091971280919812909199120F949C1FFE
:1074000042E00E94B8E9E5E2F3E084918F010F5F6A
:107410001F4F882321F00E94857FF801F6CF8AE074
:107420000E94857F9EC788E690E00E94D5F081117A
:1074300098C780919D0683FD94C783E50F94ED0264
:10744000882309F48EC70F94E3000F9404207093EF
:107450007B0E60937A0E80E00E9476780F94E300B2
:1074600020E030E040E752E40F945C1A18163CF03C
:107470000E94CC8360E089E993E00E94CBDE0F9408
:10748000E3002091560630915706409158065091DE
:1074900059060F94E62018160CF063C78EED92E0A3
:1074A0009F938F938DE893E09F938F931F920E94F9
:1074B0000FAE0F900F900F900F900F9052C70F9438
:1074C0000C034FC780919D0683FD4BC783E50F9446
:1074D000ED02882309F445C70F94E3000F940420BC
:1074E0006739710514F066E970E07093770E609368
:1074F000760E0E942C7835C70F94AE0432C78DE605
:1075000090E00E94D5F081112CC780919D0683FDEB
:1075100028C783E50F94ED0260968FAF60978111C5
:10752000BDC782E50F94ED028111B8C71AC78091DB
:107530009D0683FD16C783E50F94ED026C968FAF11
:107540006C9781110C94F14382E50F94ED02811147
:107550000C94F14306C783E50F94ED02882339F0BC
:107560000F94B3008B016F3F710519F010F00FEF0E
:1075700010E080E50F94ED02882331F00F94C300F2
:10758000823008F0EEC601C080E0E82FF0E0EE0F98
:10759000FF1FE356FE4E11830083E3C68CE40F9475
:1075A0004D02882319F00F94E30004C060E070E0FE
:1075B00080E090EC27966CAF7DAF8EAF9FAF2797A2
:1075C0008AE50F94ED02882319F00F94E30003C0BD
:1075D00060E070E0CB0120E030E040E251E40F9445
:1075E000C01E23966CAF7DAF8EAF9FAF239788E50B
:1075F0000F94ED02882319F00F94E30003C060E0BC
:1076000070E0CB0120E030E040E251E40F94C01E76
:107610006BAF7CAF8DAF9EAF89E50F94ED028823F1
:1076200019F00F94E30003C060E070E0CB0120E0AC
:1076300030E847E953E40F94C01E20E030E040E218
:1076400051E40F94BF1E68A379A38AA39BA3198258
:107650001A821B821C8280919006811182C6C12CE5
:10766000E12C8E010F5F1F4F9E01205E3F4FAE0148
:10767000455C5F4FBE01615C7F4FCE018D5B9F4FCC
:107680000E94DCE76EC60E9453840F9419050F9484
:10769000160110929E1110929D111092A01110923D
:1076A0009F1168EE73E080E090E00E945B8B60E0E9
:1076B00087E194E00E94CBDE54C61092980651C632
:1076C00083E50F94ED02882399F00F94E30020E006
:1076D00030E04AE754E40F94C11A0F9409206093F4
:1076E0000E0270930F02809310029093110239C61C
:1076F00088E50F944D0281110C94764589E50F942D
:107700004D0281110C9476458AE50F944D0281114A
:107710000C94764585E40F944D0281110C947645C6
:107720000F9419050F9416011CC60F94A60C19C6C8
:107730000F9419050E9490EB14C660E080915E06DC
:1077400090915F060E94BBDE0CC60E941D8109C697
:1077500084918F010F5F1F4F882321F00E94857F46
:10776000F801F6CFE2E5F4E084918F010F5F1F4F3F
:10777000882321F00E94857FF801F6CF1E9B03C06D
:1077800009EF12E002C004EF12E0D8018D918D01E3
:10779000882319F00E94857FF8CF8AE00E94857FB8
:1077A000EAE4F4E084918F010F5F1F4F882321F0FA
:1077B0000E94857FF801F6CF029B03C009EF12E01B
:1077C00002C004EF12E0F80181918F01882319F0C3
:1077D0000E94857FF8CF8AE00E94857FE2E4F4E092
:1077E00084918F010F5F1F4F882321F00E94857FB6
:1077F000F801F6CF1D9B03C009EF12E002C004EFB1
:1078000012E0D8018D918D01882319F00E94857FA7
:10781000F8CF8AE00E94857FEAE3F4E084918F014B
:107820000F5F1F4F882321F00E94857FF801F6CF5C
:10783000019B03C009EF12E002C004EF12E0F8015F
:1078400081918F01882319F00E94857FF8CF8AE00B
:107850000E94857FE2E3F4E084918F010F5F1F4F68
:10786000882321F00E94857FF801F6CF1C9903C080
:1078700009EF12E002C004EF12E0D8018D918D01F2
:10788000882319F00E94857FF8CF8AE00E94857FC7
:10789000EAE2F4E084918F010F5F1F4F882321F00B
:1078A0000E94857FF801F6CF379B03C009EF12E0F5
:1078B00002C004EF12E0F80181918F018823B1F139
:1078C0000E94857FF8CF8AE50F944D02882309F442
:1078D00001C30F94E3006B017C0120E030E040E045
:1078E00050EC0F94E62087FDE8C220E030E040EA4B
:1078F00050E4C701B6010F945C1A18160CF4DDC2EF
:10790000C0928506D0928606E0928706F09288069D
:1079100080E00E94045A60918506709186068091ED
:1079200087069091880642E00E94B8E98AE00E94AA
:10793000857F17C581E08093A00E8093600611C5F6
:1079400088EC90E00E94D5F081110BC584E40F947F
:107950004D028823D1F10F94E30011E020E030E0E4
:10796000A9010F945C1A811101C010E01093660602
:10797000112359F10091650610E00F94E300F8011E
:10798000EE0FFF1FEE0FFF1FEF59F94F608371835A
:107990008283938320E030E0A901609161067091B9
:1079A000620680916306909164060F945C1A8111BF
:1079B0000CC080E090E0A0E4B0E480936106909376
:1079C0006206A0936306B09364060F942001C9C4B5
:1079D0000CE213E036EAE32E31E1F32ED8018D916B
:1079E0008D010F944D02882349F00F94E3000F940A
:1079F0000920F7016083718382839383F4E0EF0EA3
:107A0000F11C23E00033120749F70E947F7EA9C4CE
:107A1000F4E0EF0EF11C23E00033120709F4A1C4D7
:107A2000D8018D918D010F944D02882389F30F9415
:107A3000E300F7016083718382839383E9CF83E559
:107A40000F944D028823D9F00F94E300AB01BC01E1
:107A50004093BE115093BF116093C0117093C11138
:107A60004093B6115093B7116093B8117093B91148
:107A70008EEC94E00E942EEA8AE00E94857F80E5E9
:107A80000F944D02882399F00F94E300AB01BC01E1
:107A90004093BE115093BF116093C0117093C111F8
:107AA00081EB94E00E942EEA8AE00E94857F82E5C5
:107AB0000F944D02882399F00F94E300AB01BC01B1
:107AC0004093BA115093BB116093BC117093BD11D8
:107AD00082E994E00E942EEA8AE00E94857F84E594
:107AE0000F944D02882309F43CC40F94E300AB01CA
:107AF000BC014093B6115093B7116093B8117093C5
:107B0000B91184E794E00E942EEA8AE00E94857F02
:107B100028C40F947B0225C40F949F0E22C40E9498
:107B20004AEA1FC483E50F94ED02882309F419C4BF
:107B30000F94B3007093A7026093A60212C40E9430
:107B400015F10FC480E50F944D02882309F409C490
:107B50000F94B300F62E062F172F83E50F94ED0236
:107B6000882321F00F94B3006B0103C0CC24CA9486
:107B7000DC2C96012F5F3F4F2330310508F0F1C315
:107B800017FDEFC30F9419053FEFC316D30631F06D
:107B9000CA94CD2871F000E010E00DC08F2D0F9435
:107BA000450431E020E0892B09F030E0032F122F4B
:107BB00002C001E010E08F2D0F944504801791075B
:107BC00009F4CFC380E00E946BFCF5CF0E94278BA5
:107BD000C8C30E94F6EAC5C380E50F944D0288230E
:107BE00051F00F94E30060937F06709380068093BA
:107BF00081069093820689E40F944D02882381F0D8
:107C00000F94E3002CEA35EC47E25EE30F94C11ACF
:107C100060937B0670937C0680937D0690937E062E
:107C200084E40F944D02882381F00F94E3002CEA42
:107C300035EC47E25EE30F949C1F609377067093E8
:107C400078068093790690937A06E5EBFEE48491BA
:107C50008F010F5F1F4F882321F00E94857FF8015D
:107C6000F6CF40917F065091800660918106709119
:107C700082068EEF94E00E942EEA2CEA35EC47E271
:107C80005EE360917B0670917C0680917D06909109
:107C90007E060F949C1FAB01BC018AEF94E00E940A
:107CA000DAEA2CEA35EC47E25EE360917706709100
:107CB00078068091790690917A060F94C11AAB01EB
:107CC000BC0186EF94E00E94DAEA8AE00E94857F98
:107CD00048C383E50F944D02182F882371F00F9449
:107CE000E3000F940420709313026093120221E0CA
:107CF000672B09F020E02093830680E50F944D0266
:107D0000882369F08091120290911302892B19F057
:107D10000F94D40001C081E08093830622C3111127
:107D200020C3E5EBFEE484918F010F5F1F4F882392
:107D300021F00E94857FF801F6CF80918306882389
:107D400019F066EF72E002C063E073E087E195E04E
:107D50000E945AD6609112027091130286E095E05B
:107D60000E948DC4E2E0F5E084918F010F5F1F4F08
:107D7000882309F4F6C20E94857FF801F5CF0E949E
:107D80000DE2EFC20F941905ECC281E00E943CF5B0
:107D9000E8C280E00E943CF5E4C286E50F944D0203
:107DA000882321F087E595E00E94615A83E50F94CE
:107DB0004D02882321F00F94D400182F01C010E049
:107DC00083E50F944D02882319F0812F0E94A95456
:107DD000F0908406111103C0E5EBFEE41AC0F11027
:107DE000FBCFEEE7FEE484918F010F5F1F4F8823E6
:107DF00021F00E94857FF801F6CFE8E3F5E0849159
:107E00008F010F5F1F4F882339F30E94857FF80190
:107E1000F6CF84918F010F5F1F4F882321F00E94BE
:107E2000857FF801F6CFFF2019F067E073E002C00C
:107E30006BE073E08AE295E00E945AD68AE00E94E5
:107E4000857F8FC20E9468EC8CC20F94BE0789C2E6
:107E50000F94780686C283E50F944D02882319F0AB
:107E60000F94D40001C081E091E089270E94A15ABB
:107E700078C283E50F944D02882309F472C20F94EF
:107E8000D4008093C50E6DC2E5EBFEE484918F01B2
:107E90000F5F1F4F882321F00E94857FF801F6CFE6
:107EA000ECE8F5E084918F010F5F1F4F882309F400
:107EB0000ACD0E94857FF801F5CFE7E7F5E08491D0
:107EC0008F010F5F1F4F882309F430CD0E94857FFB
:107ED000F801F5CF4091850650918606609187069E
:107EE0007091880684E795E00E942EEA1FCD0E94DB
:107EF0002AAE882319F081E00E94719D85E40F94D9
:107F00004D02882319F00F94E30004C060E070E094
:107F100080E090EC2F966CAF7DAF8EAF9FAF2F9728
:107F20008AE50F94ED02882319F00F94E30004C052
:107F300060E070E080E291E42B966CAF7DAF8EAF95
:107F40009FAF2B9788E50F94ED02882319F00F94CB
:107F5000E30004C060E070E080E291E427966CAF3B
:107F60007DAF8EAF9FAF279789E50F94ED028823F1
:107F700019F00F94E30004C060E070E882E993E434
:107F800023966CAF7DAF8EAF9FAF239785E50F949F
:107F90004D02882319F00F94E30004C060E070E004
:107FA00088EC92EC6BAF7CAF8DAF9EAF8CE40F94FE
:107FB0004D02882319F00F94E30003C060E070E0E5
:107FC000CB0168A379A38AA39BA382E40F94ED025B
:107FD000882321F00F94B300F62E02C085E0F82E1E
:107FE000D0907D128091900681117EC0CC24C394E4
:107FF000EF2C8E01055C1F4F9E01215C3F4FAE01AF
:108000004D5B5F4FBE01695B7F4FCE01855B9F4F2C
:108010000E94DCE7882309F467C081E08093BB08F5
:1080200011E08091BB08882309F44AC060E08F2DDD
:108030000E94B08A80918F068823F1F110938A06FE
:1080400040E050E0BA018FEB92EA0E948CE180910F
:10805000BB08882321F081E00E946BFCF8CF1092CE
:108060008B0610928C0610928D0610928E0610923E
:108070008F060E9476780E9446FF10938A0640E0A1
:1080800050E0BA0185E191EA0E948CE10F94A204CC
:10809000685370458F4F9F4F60938B0670938C068B
:1080A00080938D0690938E0610928F061093BB08D6
:1080B00061E08F2D0E94B08A81E00E946BFCB1CFFD
:1080C00000E010E028E432E409831A832B833C8328
:1080D00080919006882341F04F2DBE016F5F7F4F46
:1080E000CE0180960E94B8E651E0D5123AC10E94B6
:1080F000A6C437C1F394B4E0FB1669F0D8018D91A2
:108100008D010F944D028823A9F30F94B3008F2D96
:108110000E94E459EFCF82E40F944D02882329F0A6
:108120000F94B30084E00E94E45983E50F944D025C
:10813000882309F416C110E00F94B300812F0E9428
:10814000E4591F5F1530C1F70CC183E50F94ED02B0
:10815000882321F00F94B3008B0102C000E010E0EF
:1081600080E50F94ED02882321F00F94B300CB013A
:1081700002C080E090E0B8010E94D559F2C083E5CA
:108180000F944D02811104C00CE213E0F12C0FC0DA
:1081900010E00F94C300682F812F0E94557D1F5F50
:1081A0001530B9F7F1CFF394F4E0FF1671F0F80150
:1081B00081918F010F944D028823A9F30F94C3007E
:1081C000682F8F2D0E94557DEECF82E40F944D02D3
:1081D000882331F00F94C300682F84E00E94557DFE
:1081E0000E9411C3BEC083E50F94ED02882309F4F9
:1081F00049C00F94C300813039F0823009F042C089
:108200000CE213E0F12C23C00CE213E0F12CD801B6
:108210008D918D010F94ED02882339F00F94C300E6
:108220004FEF682F8F2D0E94AB7CF394B4E0FB12CC
:10823000EECF82E40F94ED02882321F10F94C30066
:108240004FEF682F1CC0F394F4E0FF1679F0F801AB
:1082500081918F010F94ED028823A9F30F94C3003D
:10826000482F6FEF8F2D0E94AB7CEDCF82E40F94EF
:10827000ED02882339F00F94C300482F6FEF84E09C
:108280000E94AB7C0E9411C36CC081E080931402F9
:108290001092910683E50F944D02811103C00E9454
:1082A00025C45FC00F94D40081115BC0F8CFF0905B
:1082B0009A06FF2021F1E5EBFEE484918F010F5F28
:1082C0001F4F882321F00E94857FF801F6CF84E5B7
:1082D0000E94857F6F2D70E080E090E04AE00E9470
:1082E000A0C280E20E94857F0FE013E0D8018D914B
:1082F0008D01882309F41ACB0E94857FF7CF109255
:108300009206E5EBFEE484918F010F5F1F4F8823F7
:1083100021F00E94857FF801F6CF60E070E086E9E9
:1083200095E00E948DC48AE00E94857F1AC0E5EB2B
:10833000FEE484918F010F5F1F4F882321F00E947C
:10834000857FF801F6CF609193067091940688EAD4
:1083500095E00E945AD682E20E94857F8AE00E94C0
:10836000857F0E94BDC3E5C320915E0630915F0604
:10837000232B39F49F012150310930935F0620935C
:108380005E0620E030E00C94692C80E00E94A95445
:108390000F94FA0483E50F944D02882309F449C031
:1083A0000F94D40021E0482FBE016F5F7F4FCE01B4
:1083B00080960E9487B06B017C019B01AC010F94F9
:1083C0006C21811131C02CEA35EC47E257E368A1FA
:1083D00079A18AA19BA10F94C01EAB01BC0184E2CC
:1083E00092E00E94DAEA2CEA35EC47E257E3698131
:1083F0007A818B819C810F94C01EAB01BC018FE1FF
:1084000092E00E94DAEA2CEA35EC47E257E3C70132
:10841000B6010F94C01EAB01BC018AE192E00E943C
:10842000DAEA8AE00E94857F0F94E1040E9490EBD3
:1084300098CF81E0B7CF80E00E946BFC0C948A3625
:108440000F94B300AB01BC0140934A1550934B15F8
:1084500060934C1570934D1589E994E10E94D9AB56
:1084600080CF802F0E94F9C46E2D802F0F946D0451
:10847000F12CB701802F0E9418C50630110529F490
:10848000F092A011E0929F116CCF0830110509F015
:1084900068CFF0929E11E0929D1163CF0F94E3009C
:1084A0000F94042070937B0E60937A0E80E00E94FC
:1084B00076780F94E30020E030E040E752E40F9438
:1084C0005C1A181644F00E94CC8360E08AED93E0B9
:1084D0000E94CBDE02C00E94A6C460917A0E709109
:1084E0007B0E882777FD8095982F0F94621A209134
:1084F00056063091570640915806509159060F94F0
:10850000E62018160CF065C18EED92E09F938F93D4
:108510008EEC93E09F938F931F920E940FAE0F906B
:108520000F900F900F900F9081E08093420267961A
:108530001CAE1DAE1EAE1FAE67976B961CAE1DAE79
:108540001EAE1FAE6B9710E0A0961FAEA097BCE3C7
:10855000A496BFAFA497ECE1A896EFAFA897F6E476
:10856000AC96FFAFAC97D12CE12CE0E8FE2E0FEBE0
:10857000812C912C540160917A0E70917B0E88278A
:1085800077FD8095982F0F94621A762E672E582EBD
:10859000492E262F372F482F592F6D2D7E2D8F2DA9
:1085A000902F0F945C1A8823D9F0209156063091B1
:1085B00057064091580650915906672D762D852D06
:1085C000942D0F945C1A182F111F1127111F6096FC
:1085D0002FAD6097222341F0112331F011E0E7C065
:1085E0007D2C6E2C5F2C402E0F94A2046B017C011D
:1085F000DC01CB016B962CAD3DAD4EAD5FAD6B9705
:10860000821B930BA40BB50BB7FD3BC0D701C60172
:1086100088519C4FAF4FBF4F6B968CAF9DAFAEAFA5
:10862000BFAF6B970E94DFFBEAECF3E084911F0180
:108630009FEF291A390A882321F00E94857FF101D2
:10864000F5CF81149104A104B104A9F0C501B401CE
:1086500068517C4F8F4F9F4F6C197D098E099F0980
:1086600028EE33E040E050E00F94621ECA01B901E9
:108670000E9485C203C08FE30E94857F8AE00E942A
:10868000857F80E00E946BFC0F94D704A091560672
:108690006C96AFAF6C9720905706309058060091BB
:1086A00059062A2F322D432D502F672D762D852DDB
:1086B000942D0F94BF1E9F7720E030E040E251E4FC
:1086C00081149104A104B10429F40F945C1A87FD6C
:1086D00005C006C00F94E620181614F44601570191
:1086E000112309F44AC067962CAD3DAD4EAD5FAD88
:1086F0006797211531054105510541F0D701C601A4
:10870000821B930BA40BB50BB7FD37C06C962FAD36
:108710006C97322D432D502FA0966FADA097A49645
:108720007FADA497A8968FADA897AC969FADAC9758
:108730000F94BF1E20E030E040EC5FE30F945C1A22
:1087400087FD4CCFD701C601805A9541AF4FBF4F2F
:1087500067968CAF9DAFAEAFBFAF67976C969FAD7E
:108760006C97A0969FAFA097A4962FAEA497A896BB
:108770003FAEA897AC960FAFAC978091420288238A
:10878000B1F081149104A104B10429F4D72CE62C92
:10879000F52C042DF0CEA8EECA1AA3E0DA0AE108FF
:1087A000F108C818D908EA08FB08F7FCEFCF809158
:1087B0004202882309F4D5CD60E0112329F08EEA26
:1087C00093E00E94CBDECDCD8CEB93E00E94CBDE1C
:1087D000C8CD6096BFAD6097B111A6CE89EE92E08C
:1087E00095CE0F94E3000F9404206739710514F0BF
:1087F00066E970E07093770E6093760E0E942C7895
:108800000F94E30020E030E040EA50E40F94E620CB
:10881000181614F40E94A6C46091760E7091770E1B
:10882000882777FD8095982F0F94621A20915A0619
:1088300030915B0640915C0650915D060F945C1A86
:1088400060E087FF03C08AE094E002C08DEF93E010
:108850000E94CBDE81E08093420280919206809359
:10886000650667961CAE1DAE1EAE1FAE67976B9673
:108870001CAE1DAE1EAE1FAE6B9760961FAE60970E
:10888000A0961FAEA097BCE3A496BFAFA497ECE15F
:10889000A896EFAFA897F6E4AC96FFAFAC97C12CC3
:1088A000D12C60E8E62E7FEBF72E812C912C540121
:1088B0006091760E7091770E882777FD8095982FBE
:1088C0000F94621A162F072F782E692E262F372F16
:1088D000482F592FB601C7010F945C1A882331F134
:1088E00020915A0630915B0640915C0650915D06DE
:1088F000612F702F872D962D0F945C1A881F882763
:10890000881F60968FAF60976C962FAD6C9722236F
:1089100089F0882379F080914202882309F421CDDF
:1089200060E08FEE93E00E94CBDE1BCD1C2D0D2D61
:108930007E2C6F2C0F94A2046B017C01DC01CB0117
:108940006B962CAD3DAD4EAD5FAD6B97821B930B1F
:10895000A40BB50BB7FD3BC0D701C60188519C4F96
:10896000AF4FBF4F6B968CAF9DAFAEAFBFAF6B97A6
:108970000E94DFFBE9EFF3E084912F019FEF491A9A
:10898000590A882321F00E94857FF201F5CF8114D6
:108990009104A104B104A9F0C501B40168517C4F50
:1089A0008F4F9F4F6C197D098E099F0928EE33E088
:1089B00040E050E00F94621ECA01B9010E9485C2D6
:1089C00003C08FE30E94857F8AE00E94857F80E05C
:1089D0000E946BFC0F94D70420905A0630905B06DF
:1089E00040905C0650905D069101A201612F702FAE
:1089F000872D962D0F94BF1E9F7720E030E040EA30
:108A000050E481149104A104B10429F40F945C1A78
:108A100087FD05C006C00F94E620181614F4460121
:108A200057016096AFAD6097AA2309F443C06796DB
:108A30002CAD3DAD4EAD5FAD6797211531054105BC
:108A4000510541F0D701C601821B930BA40BB50B56
:108A5000B7FD30C09101A201A0966FADA097A4967A
:108A60007FADA497A8968FADA897AC969FADAC9715
:108A70000F94BF1E20E030E040EC5FE30F945C1ADF
:108A800087FD49CFD701C601805A9541AF4FBF4FEF
:108A900067968CAF9DAFAEAFBFAF6797A0962FAE76
:108AA000A097A4963FAEA497A8964FAEA897AC9671
:108AB0005FAEAC9780914202882309F42CCF8114D9
:108AC0009104A104B10429F4C12ED02EE72CF62C78
:108AD000EFCE98EEC91A93E0D90AE108F108C81858
:108AE000D908EA08FB08F7FE16CFEECF0F94190558
:108AF00088E50F944D02882319F0179A1092A10E61
:108B000089E50F944D02882319F0169A1092A20E4F
:108B10008AE50F944D02882319F0159A1092A30E3E
:108B200085E40F944D02882309F41BCC0F941401A3
:108B300018CCC757DF4F0FB6F894DEBF0FBECDBFBE
:108B4000DF91CF911F910F91FF90EF90DF90CF9029
:108B5000BF90AF909F908F907F906F905F904F905D
:108B60003F902F9008950F93CF93DF93C82FD62F68
:108B700004E0262F41E3682F8BED91E10F948403ED
:108B80008823C9F02D2F41E36C2F8BED91E10E94DA
:108B9000AF718C2F0E94E0558FEF8D0F8C0F0E94CC
:108BA000E0552D2F44E36C2F8BED91E1DF91CF91B8
:108BB0000F910C94AF71DF91CF910F9108957F9237
:108BC0008F929F92AF92BF92CF92DF92EF92FF92DD
:108BD0000F931F93CF93DF93CDB7DEB72A970FB6CE
:108BE000F894DEBF0FBECDBF1092CA118091C211A2
:108BF000882351F00E944F9240E050E0BA0187EE86
:108C000096EF0E948CE1CBC44091A6025091A7023E
:108C10008091C6119091C711A091C811B091C9114E
:108C20009A01280F391F4436510524F425363105A1
:108C30003CF41CC04436510551F024363105B4F4DF
:108C400084E690E09093A7028093A60213C08B3035
:108C50009105A105B1051CF02A50310907C0863FD6
:108C60009F4FAF4FBF4F74F4265F3F4F3093A70223
:108C70002093A6021092C6111092C7111092C8112B
:108C80001092C9118091A6029091A7028A30910595
:108C90003CF0883E23E092072CF087EE93E002C080
:108CA0008AE090E09093A7028093A6020E94E8DEFB
:108CB000782E0E945BA780910F12853198F477205F
:108CC00049F080919D1190919E11892B19F004E536
:108CD00012E102C007E311E123E14FE061E089E026
:108CE0000E940D5580910F128D3108F084C188309B
:108CF00008F03FC080918F06711002C0811139C009
:108D000060917A0E70917B0E882777FD8095982F61
:108D10000F94621A20E030E040E05FE30F94C01E41
:108D20000F940420643671052CF46A30710524F028
:108D30004CE003C042E101C046E022E130E0241BE8
:108D4000310937FF02C02F5F3F4F35952795319589
:108D5000219531092B5F2093121227E020931312E3
:108D6000CB010E942BD90E943CC684E391E10E9472
:108D70002EC680910F128D31D0F580911112853160
:108D8000B0F120E030E040E05FE360915606709182
:108D9000570680915806909159060F94C01E0F9463
:108DA00004209B01643671050CF0F6C22A303105AF
:108DB0000CF4F0C24CE022E130E0241B310937FF13
:108DC00002C02F5F3F4F3595279531952195310989
:108DD0002B5F209312122CE120931312CB010E94DF
:108DE0002BD90E943CC684E391E10E942EC680915B
:108DF0000F12853140F580911112813120F160917F
:108E00007A0E70917B0E882777FD8095982F0F94AE
:108E1000621A20915606309157064091580650919B
:108E200059060F94E62018160CF0B8C21092FB11E8
:108E300002E022E041E16DE08BED91E10E942F72B2
:108E400081E08093FB1180910F12883008F03FC0C1
:108E50008091A106711002C0811139C06091760E17
:108E60007091770E882777FD8095982F0F94621A5E
:108E700020E030E040E05FE30F94C01E0F94042038
:108E8000643671052CF46A30710524F04CE003C09F
:108E900042E101C046E022E130E0241B310937FF06
:108EA00002C02F5F3F4F35952795319521953109A8
:108EB0002F5A2093121227E020931312CB010E9405
:108EC0002BD90E943CC684E391E10E942EC680917A
:108ED0000F128D31D0F5809111128531B0F120E063
:108EE00030E040E05FE360915A0670915B0680914C
:108EF0005C0690915D060F94C01E0F9404209B01A8
:108F0000643671050CF055C22A3031050CF44FC29D
:108F10004CE022E130E0241B310937FF02C02F5F13
:108F20003F4F359527953195219531092F5A20933B
:108F300012122CE120931312CB010E942BD90E9414
:108F40003CC684E391E10E942EC680910F128531C8
:108F500040F580911112813120F16091760E70916F
:108F6000770E882777FD8095982F0F94621A2091AD
:108F70005A0630915B0640915C0650915D060F9455
:108F8000E62018160CF017C21092FB1102E022E046
:108F900042E168E58BED91E10E942F7281E08093C0
:108FA000FB1180910F128C3130F5809111128431B8
:108FB00010F180919D1190919E11019644E6489F79
:108FC0009001499F300D112437FF02C021503F4FBF
:108FD000832F932F990F990B009769F028E6209320
:108FE00012122BE1209313120E942BD90E943CC62F
:108FF00085E20E947AA780910F12843328F4809131
:1090000011128A3208F0E0C180910F12853328F4E2
:1090100080911112813308F0FCC18091A71288233E
:1090200009F44DC080910F12843308F048C080913C
:109030001112823308F443C080919C14882309F4F0
:10904000ECC18091461590914715A0914815B091BB
:1090500049150097A105B10509F4DFC1BC01CD0197
:109060006D597F4F8F4F9F4F24E630E040E050E036
:109070000F94621E60914A1570914B1580914C15AA
:1090800090914D150F94621E622F48E4649FB001C9
:109090001124882777FD8095982F0F94621A2AE073
:1090A00037ED43E25CE30F94C11A0F940920262F99
:1090B00002E042E367E38BED91E10E942F72809121
:1090C0000F12813308F05FC080911112893208F4C9
:1090D0005AC08DE792E10E9461D96B017C018CE35B
:1090E000882E912CA12CB12CC701B601A5019401A9
:1090F0000F94621ECA01B901A50194010F94621E6A
:10910000CA01962E872E59018E010F5F1F4F41E82D
:10911000C41641E5D40641E0E406F10408F47FC139
:10912000B90128E130E040E050E00F94621E79017F
:109130008F929F92C50168E170E00F9488219F9300
:109140008F933F932F9324E736E03F932F931F9302
:109150000F930F94F6190FB6F894DEBF0FBECDBF74
:109160009AE0E916F10408F489C198E0892F880F84
:10917000890F8195855A8093121280E38093131290
:10918000C8010E943CC6E091D511F091D6118481AE
:109190008111CCC06091B10E7091B20E8091B30E6E
:1091A0009091B40E0F940420CB010E94C2D8BC0150
:1091B00087EB96E00F9400226091B50E7091B60E89
:1091C0008091B70E9091B80E0F940420CB010E94AD
:1091D000C2D8BC0182EB96E00F9400222CEA35EC59
:1091E00047E257E36091B90E7091BA0E8091BB0EC1
:1091F0009091BC0E0F94C01E20E030E048EC52E489
:109200000F94C11A0F9404206B017C0197FD19C0C3
:1092100090E1C91697E2D906E104F104E4F0C70130
:10922000B60120E137E240E050E00F94841ECA010D
:10923000B9012AE030E040E050E00F94841E605D08
:109240000BC0F094E094D094C094C11CD11CE11CDC
:10925000F11C6DE201C060E26093A30628EEC21625
:1092600023E0D206E104F10494F0C701B60128EE30
:1092700033E040E050E00F94841ECA01B9012AE0B7
:1092800030E040E050E00F94841E605D01C060E279
:109290006093A406C701B60124E630E040E050E048
:1092A0000F94841E9AE0892E912CA12CB12CCA0116
:1092B000B901A50194010F94841E605D6093A50619
:1092C000C701B601A50194010F94841E162F6623D1
:1092D00081F08EE28093A606CA01B901A50194012E
:1092E0000F94841E605D6093A706105D1093A8061E
:1092F00017C0CA01B901A50194010F94841E662309
:1093000039F08EE28093A606605D6093A70605C0E3
:1093100080E28093A7068093A60680E28093A80649
:1093200063EA76E08BEA96E00F94002280910F12B8
:109330008632A8F4809111128E3188F008E020E87E
:109340004EE160E08BED91E10E942F7280910F124F
:10935000863228F4809111128F3108F091C08091EB
:109360000F12823328F4809111128C3208F0F8C069
:1093700080910F128F3308F012C18091111288333F
:1093800008F40DC1109212128EE3809313120E9402
:1093900097A705C146E00FCD42E10DCD02E022E0E6
:1093A00041E16DE08BED91E10E942F724CCD46E0E2
:1093B000B0CD42E1AECD02E022E042E168E58BEDC6
:1093C00091E10E942F72EDCD07E028E04AE26AE2C7
:1093D0008BED91E10E942F7205E022E04CE262E306
:1093E0008BED91E10E942F726AE08AE2BCDB609112
:1093F000DD117091DE1182E38093F7118BE280938F
:10940000F81127EF31E142E38BED91E10F94A603D0
:10941000FBCD6AE486E3A7DB00CE60E036CE44E60F
:10942000A416B104C0F48F929F92C50168E170E068
:109430000F9488219F938F938AE696E09F938F9352
:109440001F930F930F94F6190FB6F894DEBF0FBE5B
:10945000CDBF95E08BCE8F929F923F932F9382E664
:1094600096E09F938F931F930F930F94F6190FB667
:10947000F894DEBF0FBECDBF96E078CE97E076CEF3
:109480001092FB1183E08093121285E280931312F5
:10949000772029F082E391E10E942EC60DC08091D1
:1094A0005A08811102C08FE305C08091A10E81117D
:1094B000F1CF80E20E947AA78BE08093121215E22E
:1094C0001093131287EB96E00E943CC68BE28093C8
:1094D000121210931312772029F080E391E10E9479
:1094E0002EC60DC080915B08811102C08FE305C0BC
:1094F0008091A20E8111F1CF80E20E947AA783E3CE
:109500008093121215E21093131282EB96E00E94E0
:109510003CC683E58093121210931312772029F032
:109520008EE291E10E942EC60DC080915C088111EF
:1095300002C08FE305C08091A30E8111F1CF80E2BC
:109540000E947AA78BE58093121285E28093131212
:109550008BEA96E00E943CC681E08093FB11FFCE2F
:1095600084E00E9462A783E08093121212E31093BA
:10957000131286E00E9485A70E945BA78CE080936F
:109580001212109313128091A6029091A7020E94CA
:109590002BD90E943CC685E20E947AA7E9CE2A9682
:1095A0000FB6F894DEBF0FBECDBFDF91CF911F91F4
:1095B0000F91FF90EF90DF90CF90BF90AF909F9072
:1095C0008F907F9008951F93CF93DF931092CA11CD
:1095D0008091C6119091C711A091C811B091C91185
:1095E00081309048A105B10540F01092C61110924B
:1095F000C7111092C8111092C911C091C6114091A3
:109600009F06141604F5842F992787FD90950597DA
:109610002C2F332727FD309528173907A4F0453024
:109620001CF0CBEFC40F01C0C0E08C2F992787FD41
:109630009095A92FB92F8093C6119093C711A0932D
:10964000C811B093C911C093C311D0E012E0C11189
:1096500009C08091A8028823D9F121E041E06FE19F
:1096600076E020C0C13049F48091A802882381F1BE
:1096700020E041E060E176E015C0C23049F480911D
:10968000A802882329F120E041E060E076E00AC0EA
:10969000C33061F48091A8028823D1F020E041E03A
:1096A00069EF75E08D2F0E94B0A012C0C43081F424
:1096B0008091A802882351F021E040E06EEE75E031
:1096C0008D2F0E94B0A08D2F0E9448C61093A80233
:1096D000DF5FCF5FD53009F0BACFD0939F06DF911F
:1096E000CF911F9108951F93CF93DF931092CA11CA
:1096F0008091C6119091C711A091C811B091C91164
:1097000081309048A105B10540F01092C611109229
:10971000C7111092C8111092C911C091C611409181
:109720009E06141604F5842F992787FD90950597BA
:109730002C2F332727FD309528173907A4F0453003
:109740001CF0CBEFC40F01C0C0E08C2F992787FD20
:109750009095A92FB92F8093C6119093C711A0930C
:10976000C811B093C911C093C311D0E012E0C11168
:1097700009C08091A8028823D9F121E041E061EE7F
:1097800075E020C0C13049F48091A802882381F19E
:1097900020E041E068ED75E015C0C23049F48091E9
:1097A000A802882329F120E041E068EC75E00AC0B6
:1097B000C33061F48091A8028823D1F020E041E019
:1097C00066EC75E08D2F0E94B0A012C0C43081F409
:1097D0008091A802882351F021E040E06BEB75E016
:1097E0008D2F0E94B0A08D2F0E9448C61093A80212
:1097F000DF5FCF5FD53009F0BACFD0939E06DF91FF
:10980000CF911F9108950F931F93CF93DF931092E1
:10981000CA118091C6119091C711A091C811B09141
:10982000C91181309048A105B10540F01092C611D0
:109830001092C7111092C8111092C911C091C6118F
:109840004091A0061416D4F4842F992787FD909593
:1098500001972C2F332727FD30952817390774F0EF
:10986000CFEFC40F8C2F90E0A0E0B0E08093C61142
:109870009093C711A093C811B093C9111092C4114D
:109880008091C311C81714F4C093C3118091C31100
:10989000992787FD909504962C2F332727FD309527
:1098A0008217930724F48CEF8C0F8093C3111091CF
:1098B000C311D0E081E002E0111123C08823B9F088
:1098C0001C16ACF04091C6115091C7116091C8119F
:1098D0007091C9114F5F5F4F6F4F7F4F4093C6111B
:1098E0005093C7116093C8117093C911CF5F8091D5
:1098F000A802882309F469C021E041E063E576E02D
:109900004EC0113019F58823B9F0C230ACF4409143
:10991000C6115091C7116091C8117091C9114F5F64
:109920005F4F6F4F7F4F4093C6115093C7116093A5
:10993000C8117093C911CF5F8091A802882309F4E0
:1099400044C020E040E06EE376E029C01230E9F444
:109950008091C211811105C08091A8028823A9F1CC
:1099600009C0C230C9F70E94EAE18091C41188237E
:1099700099F333C081E0C23009F080E024E049E38C
:1099800056E06D2F0E94FB7220C0133061F480916D
:10999000A8028823D1F020E041E067E376E08D2F34
:1099A0000E94B0A012C0143081F48091A8028823D4
:1099B00051F021E040E06CE276E08D2F0E94B0A0F3
:1099C0008D2F0E9448C60093A802DF5F1F5FD5302D
:1099D00011F080E071CFD093A006DF91CF911F915D
:1099E0000F9108952F923F924F925F926F927F92C4
:1099F0008F929F92AF92BF92CF92DF92EF92FF929F
:109A00000F931F93CF93DF93CDB7DEB72B970FB68E
:109A1000F894DEBF0FBECDBF9E838D83DC015996C7
:109A20002D903C905A97F101418452846384748450
:109A3000FFEF4F1A5F0A6F0A7F0A1496CD90DD90F0
:109A4000ED90FC901797C114D104E104F10439F0B2
:109A50002FEFC21AD20AE20AF20A1B8607C0D1010E
:109A6000CD90DD90ED90FC90B1E0BB8746015701B1
:109A70001F82188619861A86F10181859285A38531
:109A8000B4852F81388549855A85281739074A07B3
:109A90005B0708F08DC04C145D046E047F0450F425
:109AA00082E0C82ED12CE12CF12C92E0892E912C51
:109AB000A12CB12C9E012F5F3F4FB701A601C10120
:109AC0000E94E0A9882309F473C089819A81AB813F
:109AD000BC81892B8A2B8B2B41F0460157013FEF2C
:109AE000831A930AA30AB30A05C0C814D904EA0466
:109AF000FB0489F08F819885A985BA850196A11DFF
:109B0000B11D8F839887A987BA879FEFC91AD90A91
:109B1000E90AF90AB1CF0FEF1FEF2FEF3FE0B501D0
:109B2000A401C1010E9429ADF82E882309F440C088
:109B3000ED81FE8144815581668177814115510512
:109B40006105710539F095018401C1010E9429ADBB
:109B5000882371F1AD81BE8114968D929D92AD9254
:109B6000BC921797BB85BB2351F0D501C401019668
:109B7000A11DB11DF10180839183A283B383ED8187
:109B8000FE8185899689A789B08D892B8A2B8B2B9D
:109B900081F4AD81BE8155968D929D92AD92BC921D
:109BA000589711968C911197806811968C9301C0EB
:109BB000F12C8F2D2B960FB6F894DEBF0FBECDBFC4
:109BC000DF91CF911F910F91FF90EF90DF90CF9099
:109BD000BF90AF909F908F907F906F905F904F90CD
:109BE0003F902F900895CF93DF93EC018B818823D2
:109BF00091F1898187FF2BC06C857D858E859F853E
:109C000041E00E9450A8882331F1E88980E2E89F72
:109C1000F0011124EA5AFB4F3097E9F08081853E2C
:109C2000D1F08B81823040F449895A896B897C89D3
:109C3000448F558F668F778F4D895E896F89788DB8
:109C4000538F428F758B648B89818F778983DF91E6
:109C5000CF910C9412A881E0888380E0DF91CF91AE
:109C60000895CF93DF93EC018B81813099F4898142
:109C700081FF10C049895A896B897C89452B462B05
:109C8000472B59F140E050E0BA01CE010E94D9AB18
:109C9000811102C080E022C04D895E896F89788D74
:109CA000898D9A8D0E94B8AD8823A1F31D8A1E8AE2
:109CB0001F8A188E198A1A8A1B8A1C8A89818068D1
:109CC0008983CE0190DF882329F340E050E0BA0178
:109CD000CE01DF91CF910C94D9AB81E0DF91CF9190
:109CE00008956F927F928F929F92AF92BF92CF9280
:109CF000DF92EF92FF920F931F93CF93DF931F9208
:109D0000CDB7DEB78C015B014A01722EDB0159969B
:109D10008D919C915A97F801928F818F40E050E08D
:109D2000BA01C5010E94D9ABE12CF501808591856E
:109D3000A285B385418952896389748984179507FF
:109D4000A607B70708F0CEC035E0B695A79597955A
:109D500087953A95D1F7F82FFF70FF2ED50113960E
:109D60008C91823008F49BC141E050E0BE016F5FEE
:109D70007F4FC5010E945FAA019719F4898190E085
:109D800002C08FEF9FEF019609F489C1F50180852C
:109D90009185A285B3854F96A11DB11D80879187BE
:109DA000A287B387F0E2FF9EB00111246A5A7B4F6D
:109DB0006115710509F473C1DB018C91882311F0E1
:109DC000853EB9F4E1100EC08091BF069091C006A7
:109DD000A091C106B091C206F80184879587A68735
:109DE000B787F08ADB018C91EE24E39481119DCF3B
:109DF00079C04BE050E0C4010F94C121892B09F0D8
:109E000094CF77FC4CC120E2F29EF0011124EA5A73
:109E1000FB4F8385817121F0872D827109F05EC02F
:109E20004091BF065091C0066091C1067091C20674
:109E3000D8011C964D935D936D937C931F9750961C
:109E4000FC924489558960E070E0BA0155274427A7
:109E5000828D938DA0E0B0E0482B592B6A2B7B2B91
:109E6000D80155964D935D936D937C935897838558
:109E7000887159F4848D958DA68DB78DF801818BED
:109E8000928BA38BB48B81E010C0803139F598019F
:109E90002F5E3F4FD80159968D919C915A970E9401
:109EA00072AC8823D9F084E0F8018383872D8F700A
:109EB000D80111968C931197F8011482158216829D
:109EC000178218961D921D921D921C921B9774FE6C
:109ED000D9C0C801C6DE8111D5C0E2C0D801139631
:109EE0001C92DDC0872D8274823409F0D8C0EE2028
:109EF000E1F0D8015096FC9050971C966D917D91A1
:109F00008D919C911F9741E00E9450A8882309F4ED
:109F1000C6C0F8018089F0E28F9FC00111248A5ADF
:109F20009B4F009709F08EC0BAC0D50113968C9153
:109F30001397823009F4B3C051968D919D910D9085
:109F4000BC91A02D803E9F4FAF41B10508F0A7C046
:109F5000C50148DD882309F4A2C00E9412A8882305
:109F600009F49DC0D5015996ED91FC915A9714962C
:109F7000CD90DD90ED90FC901797B2E0CB1AD10810
:109F8000E108F108058404C0CC0CDD1CEE1CFF1CAC
:109F90000A94D2F786859785A089B189C80ED91E03
:109FA000EA1EFB1E81E08093BE06C092BF06D092DF
:109FB000C006E092C106F092C20680E092E0E6E5BB
:109FC000F4E0DF019C011D9221503040E1F766244E
:109FD0006394D5015996ED91FC915A978481681646
:109FE00098F426E534E0B701A601460D511D611D28
:109FF000711D8091BC069091BD060E94A6A7882382
:10A0000009F44DC06394E5CF40E052E060E070E0B9
:10A01000058404C0440F551F661F771F0A94D2F7AA
:10A0200051968D919D910D90BC91A02D840F951FFF
:10A03000A61FB71FF501818B928BA38BB48B86E58E
:10A0400094E0F12C20E2DC011D922A95E9F72BE047
:10A05000F401DC0101900D922A95E1F721E238E24A
:10A06000FC01318B208B40E058E057874687338BCB
:10A07000228B318F208F578B468B0E9412A8811123
:10A08000C2CE0DC075FE09C0F801418952896389AD
:10A090007489C8010E94D9AB03C081E001C080E08F
:10A0A0000F90DF91CF911F910F91FF90EF90DF9074
:10A0B000CF90BF90AF909F908F907F906F900895BA
:10A0C0002F923F924F925F926F927F928F929F92C8
:10A0D000AF92BF92CF92DF92EF92FF920F931F93B6
:10A0E000CF93DF9300D01F921F92CDB7DEB78C01C4
:10A0F0005B014D83252EDC0113968C9113978130E3
:10A10000C9F411968C9181FF15C082FF19C0F80126
:10A11000418952896389748980859185A285B38537
:10A1200084179507A607B70759F0C8010E94D9AB55
:10A13000811106C081E0F80180838FEF9FEF2DC170
:10A14000ED80F22C80C0D8015996ED91FC915A9780
:10A1500034803A94DB01CA0169E0B695A7959795DA
:10A1600087956A95D1F738224A01B1E09B223320C6
:10A1700009F475C080E092E08819990967018E158D
:10A180009F0508F46C01D8015996ED91FC915A97FE
:10A1900014964D905D906D907C901797B2E04B1A9D
:10A1A000510861087108058404C0440C551C661CE4
:10A1B000771C0A94D2F786859785A089B189480EC5
:10A1C000591E6A1E7B1E430C511C611C711CC1145C
:10A1D000E2E0DE0609F08BC08091BF069091C006D8
:10A1E000A091C106B091C20684159505A605B705D4
:10A1F00069F41092BE068FEF9FEFDC018093BF06DB
:10A200009093C006A093C106B093C2069501B30116
:10A21000A2018091BC069091BD060E94A6A788234A
:10A2200009F488CFF80180859185A285B3858C0DCE
:10A230009D1DA11DB11D80879187A287B387AC0C9E
:10A24000BD1CEC18FD08D80118964D915D916D91DB
:10A250007C911B97E114F10409F075CF7EC0811445
:10A26000910409F087CFD80114964D915D916D91BD
:10A270007C911797411551056105710559F4559663
:10A280008D919D910D90BC91A02D0097A105B105D8
:10A2900041F522C09E012F5F3F4FCF010E94E0A9F0
:10A2A000882309F447CF89819A81AB81BC81F80169
:10A2B000218D328DF9012789203139F4883FFFEF54
:10A2C0009F07A105B10540F40CC0883F2FEF92070E
:10A2D000A2072FE0B20728F0C80184DB81114ACF22
:10A2E00029CFF80184839583A683B78343CF811454
:10A2F000910419F5D80118964D915D916D917C915D
:10A300001B9751968D919D910D90BC91A02D481752
:10A3100059076A077B0788F00E9412A8882309F46E
:10A3200009CF81E08093BE064092BF065092C006DE
:10A330006092C1067092C20608C041E0C301B2013A
:10A340000E9450A8882309F4F5CEA601B501C401E6
:10A350008A5A9B4F0F94CE2165CF51968D919D9136
:10A360000D90BC91A02D84179507A607B70740F460
:10A37000F801418B528B638B748B81818068818360
:10A38000D80111968C9183FD03C08D81922D05C05B
:10A39000C80129DC8111F9CFCDCE0F900F900F901D
:10A3A0000F900F90DF91CF911F910F91FF90EF9041
:10A3B000DF90CF90BF90AF909F908F907F906F90E5
:10A3C0005F904F903F902F900895CF93DF931F920F
:10A3D000CDB7DEB7698341E050E0BE016F5F7F4FCC
:10A3E00004966EDE0F90DF91CF910895CF93DF93A7
:10A3F000EC01F9DB1B82DF91CF9108951092A71237
:10A4000080919C14882319F089E994E1EFCF089595
:10A41000CF92DF92EF92FF921F93CF93DF93109230
:10A42000A81280910213882319F08FEF92E1DEDFEA
:10A43000109276141092731485E3809372140F9423
:10A44000A204EB01A895809172140E94F9C482E7DE
:10A4500094E10E94E97E2398229A219A209A289AD0
:10A4600085E08093741482E58CBD1DBC1AE08FEFEB
:10A470000E94EE7E1150D9F720E030E0A90160E0A3
:10A4800082E794E10E94147F182F80937514813025
:10A4900049F00F94A2046C1B7D0B613D774060F383
:10A4A00081E054C02AEA31E040E050E068E082E711
:10A4B00094E10E94147F82FF03C0109376140EC0B3
:10A4C00014E00E94F37E809375141150D1F78A3AFC
:10A4D00011F082E03BC082E0809376148091761484
:10A4E000823031F4C12CD12CE12C70E4F72E03C062
:10A4F000C12CD12C760120E030E0A90167E382E78E
:10A5000094E10E94147FA701960169E282E794E139
:10A510000E94147F80937514882349F00F94A2043D
:10A520006C1B7D0B613D774030F38AE00FC080915A
:10A530007614823011F520E030E0A9016AE382E769
:10A5400094E10E94147F882351F088E08093731473
:10A5500082E794E10E94E97EE5EBFEE41AC00E94E6
:10A56000F37E807C803C19F483E0809376140E9413
:10A57000F37E0E94F37E0E94F37E82E794E10E94C4
:10A58000E97E1092741481E00E9487A8811132C084
:10A5900015C08491EF012196882321F00E94857FC8
:10A5A000FE01F7CFE2EAF3E18491EF0121968823DF
:10A5B00009F457C00E94857FFE01F6CF80E00E941B
:10A5C00087A8811117C0EEE7FEE48491EF01219680
:10A5D000882321F00E94857FFE01F7CFEEE8F3E1AA
:10A5E0008491EF012196882309F43BC00E94857F66
:10A5F000FE01F6CF67E774E18FEF92E10E94D8ACDD
:10A60000811116C0EEE7FEE48491EF0121968823C4
:10A6100021F00E94857FFE01F7CFEDE7F3E1849101
:10A62000EF0121968823E9F00E94857FFE01F7CF94
:10A6300081E08093A812E5EBFEE48491EF0121967E
:10A64000882321F00E94857FFE01F7CFE1E7F3E147
:10A650008491EF012196882321F00E94857FFE01DD
:10A66000F7CF8BE1EFEFF2E1A0E2B3E101900D92C1
:10A670008A95E1F78091FD129091FE1290931F133D
:10A6800080931E138BEF92E190931B1380931A1308
:10A69000DF91CF911F91FF90EF90DF90CF900895C1
:10A6A000FC0123812111A2CE08952F923F924F9257
:10A6B0005F926F927F928F929F92AF92BF92CF9252
:10A6C000DF92EF92FF920F931F93CF93DF93CDB75B
:10A6D000DEB7C454D1090FB6F894DEBF0FBECDBFAC
:10A6E0004C015B017A01322E1C8E1F8E19821C8256
:10A6F0006115710511F410E0ACC0FC01838181117A
:10A70000FACFFA0180818F3261F4CA017C0101968F
:10A71000F70120812F32D1F3F501838182508230FD
:10A7200010F465010BC0618D728DCE0101960E94FF
:10A73000D8AC882301F3CE0101966C018E01045E32
:10A740001F4F2801E7E36E2E712C6C0E7D1E9BE0DF
:10A75000690E711CFE0131962496FFAFEEAF24976F
:10A7600025960FAF2597212E35C080E28193E615FF
:10A77000F705D9F7D70120E097E04A2F3B2F8D91BD
:10A7800081112BC08FA9803209F4B5CF842F932F6C
:10A790007C01FC01208101962F32D1F3222309F4A0
:10A7A00050C021E0AE01495C5F4FB601C80199DAA3
:10A7B000882309F4A0CFCA14DB0411F0C60116DE09
:10A7C00004151505B9F125969FAD2597822D6801D1
:10A7D000092F182FFE01F796C8CF8F3299F28E32CB
:10A7E00019F0E0EBF3E10AC09A3009F484CF28E0D5
:10A7F0009AE0C3CF3196381709F47DCF34913111E7
:10A80000F9CF921708F477CF813208F474CF8F37DD
:10A8100009F471CF31E0320FE7E3F0E0EC0FFD1FF8
:10A82000E20FF11D2FE9280F2A3108F480528083AE
:10A83000232FA3CF23969FAD239724968FAD2497E4
:10A84000C6CF232DAE01495C5F4FB601C40149DA82
:10A85000182FCE01019624DFCE014C9621DF812FE7
:10A86000CC5BDF4F0FB6F894DEBF0FBECDBFDF91DC
:10A87000CF911F910F91FF90EF90DF90CF90BF90FD
:10A88000AF909F908F907F906F905F904F903F9090
:10A890002F90089524E233E0FC0131832083049655
:10A8A000FFCECF92DF92EF92FF920F931F93CF9341
:10A8B000DF938C01EB016A0179010E9456DF23E0EE
:10A8C0002093A8021093850800938408D0938308EE
:10A8D000C0938208A601662757FD6095762F4093A6
:10A8E0007E0850937F086093800870938108C701A9
:10A8F000AA2797FDA095BA2F841B950BA60BB70B23
:10A9000080937A0890937B08A0937C08B0937D088D
:10A9100088819981AA2797FDA095BA2F841B950B52
:10A92000A60BB70B8093C6119093C711A093C811C3
:10A93000B093C9118FEF9EE890932C0280932B0265
:10A94000DF91CF911F910F91FF90EF90DF90CF900B
:10A95000089590918406891781F08093840681116F
:10A9600008C00E948F7D8FEA98E00E94FCDB0D9466
:10A97000210381EB9EE00C94FCDB089580E0E9DF8D
:10A9800080E090E0A0E8BFE3809315129093161248
:10A99000A0931712B09318121092191210921A1253
:10A9A00010921B1210921C1210921D1210921E1265
:10A9B00010921F1210922012109221121092221245
:10A9C0001092231210922412809325129093261233
:10A9D000A0932712B09328121092291210922A12D3
:10A9E00010922B1210922C1210922D1210922E12E5
:10A9F00010922F12109230121092311210923212C5
:10AA000010923312109234128093351290933612B2
:10AA1000A0933712B093381208958F929F92AF92FD
:10AA2000BF92CF92DF92EF92FF920F931F93CF933B
:10AA3000DF93882EB62EA42EF22EE801242F220FAB
:10AA4000220F220F0F2D462F682F8BED91E10F94CF
:10AA50008403882351F10B2D0F0DCA2CD12CB01675
:10AA600021F17E019A2C182D9920D9F0F7018491BB
:10AA70006091DD117091DE111093F711B092F81111
:10AA80001092FA118093F91127EF31E14BE38BED2E
:10AA900091E10F94A603FFEFEF1AFF0A9A94185F53
:10AAA000E3CFCC0DDD1DB394DACFDF91CF911F91B1
:10AAB0000F91FF90EF90DF90CF90BF90AF909F905D
:10AAC0008F900895CF93DF93C0917114CC23C1F080
:10AAD000C150C09371148FE1C89FE0011124C55C7F
:10AAE000DC4E8BE1FE013496A0E2B3E101900D92C1
:10AAF0008A95E1F78A819B8190931F1380931E139F
:10AB00001092C31181E08093C41183E08093A80266
:10AB1000DF91CF910895CF92DF92EF92FF920F9342
:10AB20001F93CF93DF93EC010F94A2040E811F813A
:10AB300028853985011511052105310559F53C8513
:10AB40003323A9F12A8531503C8731E0320F3A870F
:10AB50004D85341301C01A86FE0134E0239FE00DB9
:10AB6000F11D112406851785208931890A831B83ED
:10AB70002C833D836B017C01C00ED11EE11CF11CB6
:10AB8000CE82DF82E886F9868C819D81892B79F0DF
:10AB9000769A0DC06B017C01C01AD10AE20AF30A51
:10ABA000F7FC05C076981E821F8218861986DF91F1
:10ABB000CF911F910F91FF90EF90DF90CF9008956C
:10ABC0006091DD117091DE118093F71181E3809324
:10ABD000F81181E08093FA1180EF8093F91127EF4B
:10ABE00031E14BE38BED91E10D94A6030F931F939D
:10ABF000CF93DF938C01EB01DC0113968C918823BA
:10AC0000C1F18250823028F48FE28883198281E07A
:10AC100031C0F801648575858685978540E00E947E
:10AC200050A8882339F1D8015096EC91B0E2EB9FFF
:10AC3000F0011124EA5AFB4F3097D9F090E020E060
:10AC40003EE24081403269F0283029F4DE01A90F4C
:10AC5000B11D3C939F5F4081DE01A90FB11D4C9354
:10AC60009F5F2F5F31962B3061F7C90FD11D18827E
:10AC700001C080E0DF91CF911F910F910895CF9394
:10AC8000DF9380911412811107C081E08093141228
:10AC90008BED91E10F94AA03C091DD11D091DE11EB
:10ACA000E0910C12F0910D1282E01995E0910C12D6
:10ACB000F0910D1281E0199520E030E044E1BE01F1
:10ACC0008BED91E10F94A6032EE032E147E1BE0146
:10ACD0008BED91E10F94A603E0910C12F0910D120F
:10ACE00080E0DF91CF91199490915D1280915E1276
:10ACF000981731F080915E128F5F8F7080935E1293
:10AD000008950F931F93CF93DF93EC01FC01E65A54
:10AD1000FF4F1082138234971382128284E293E0F1
:10AD200091838083B59610821382349713821282A6
:10AD3000918380838E010A561F4F9E0124533E4FFC
:10AD4000F801B8016C5F7F4FAC01CF01801B910B04
:10AD5000860F971FDC011C9213961C92138212829D
:10AD6000518340837F96E217F30779F7CE0183532F
:10AD70009E4F29E1DC0111962C93119714961C9299
:10AD80000596DC0157961C928296DC011C92139664
:10AD90001C920497DC0113961C921E92129724E2D7
:10ADA00033E02D933C93198218821B821A828F54B0
:10ADB0009F4FDC011D921D921D921C9213970496C9
:10ADC000DC011D921D921D921C9213971082FE01B0
:10ADD000E15FFD4F108286E391E0F8019C01119242
:10ADE00021503040E1F7FE01E355FD4F81E08083C3
:10ADF000E955F240118210820F94A204C755DD4F2D
:10AE000068577C4E8F4F9F4F688379838A839B83DB
:10AE1000DF91CF911F910F910895CF92DF92EF9222
:10AE2000FF920F931F93CF93DF93EB01FC0160819F
:10AE30007181828193812CE3C22ED12CE12CF12CE3
:10AE4000A70196010F94621E162F072FCA01B901A0
:10AE5000A70196010F94621EF62EE72ECA01B901D2
:10AE600028E130E040E050E00F94621EFB01C90190
:10AE70006DE671E00F9488219B014F2D5E2D211509
:10AE80003105D9F00F931F93EF92FF92FF93EF9349
:10AE90009F938F933F932F9382E796E19F938F9396
:10AEA000DF93CF930F94F6198DB79EB70E960FB61A
:10AEB000F8949EBF0FBE8DBF5BC00097C9F00F9383
:10AEC0001F93EF92FF92FF93EF939F938F9382E6EE
:10AED00096E19F938F93DF93CF930F94F619EDB77D
:10AEE000FEB73C960FB6F894FEBF0FBEEDBF40C054
:10AEF0003097B9F00F931F93EF92FF92FF93EF9368
:10AF000086E596E19F938F93DF93CF930F94F61985
:10AF10008DB79EB70A960FB6F8949EBF0FBE8DBF31
:10AF200027C0452BA9F00F931F93EF92FF928EE459
:10AF300096E19F938F93DF93CF930F94F619EDB71C
:10AF4000FEB738960FB6F894FEBF0FBEEDBF10C027
:10AF50000F931F938AE496E19F938F93DF93CF9390
:10AF60000F94F6190F900F900F900F900F900F9075
:10AF7000DF91CF911F910F91FF90EF90DF90CF90D5
:10AF800008950F931F93CF93DF93CDB7DEB76997E3
:10AF90000FB6F894DEBF0FBECDBF8DE792E10E94E1
:10AFA00061D96E8B7F8B888F998FBE016F5F7F4FCA
:10AFB000CE01469632DF60E0CE0101960E94BBDEF4
:10AFC000E5EBFEE484918F010F5F1F4F882321F092
:10AFD0000E94857FF801F6CFBE016F5F7F4F86E844
:10AFE00096E10E945AD68AE00E94857F69960FB644
:10AFF000F894DEBF0FBECDBFDF91CF911F910F91AF
:10B0000008952F923F924F925F926F927F928F920C
:10B010009F92AF92BF92CF92DF92EF92FF920F93E7
:10B020001F93CF93DF93CDB7DEB768970FB6F89431
:10B03000DEBF0FBECDBF1C015B018A01DC01D796CC
:10B040006D917D918D919C91DA970F94601A6B01AF
:10B050007C01F50120813181428153810F94C11A15
:10B060000F94861F0F94092069877A878B879C87A6
:10B07000D8012D913D914D915C91C701B6010F947E
:10B08000C11A0F94861F0F9409206D877E878F87C2
:10B09000988B29853A854B855C8528373105410594
:10B0A000510540F488E790E0A0E0B0E089879A87F6
:10B0B000AB87BC872D853E854F855889283731055C
:10B0C0004105510540F488E790E0A0E0B0E08D87AD
:10B0D0009E87AF87B88B91012D5B3F4FD9018D9132
:10B0E0009D910D90BC91A02D8D839E83AF83B887D9
:10B0F000BC01CD010F94621A69837A838B839C8390
:10B1000069857A858B859C850F94601A698B7A8B0B
:10B110008B8B9C8B20E030E0A90169817A818B8147
:10B120009C810F945C1A882339F1A7019601C7010D
:10B13000B6010F94C11A4B015C0129893A894B89E8
:10B140005C89CA01B9010F94C11A9B01AC01C50108
:10B15000B4010F94BF1E4B015C0129813A814B81E0
:10B160005C81CA01B9010F94C01E9B01AC01C501ED
:10B17000B4010F949C1F03C060E070E0CB010F94FA
:10B18000861F0F9404202B013C016D817E818F81ED
:10B19000988590958095709561957F4F8F4F9F4FC3
:10B1A0000F94621A4B015C016D857E858F859889AD
:10B1B0000F94601A6D837E838F83988720E030E040
:10B1C000A901C501B4010F945C1A882349F12D81AE
:10B1D0003E814F815885CA01B9010F94C11A6D8B08
:10B1E0007E8B8F8B988FA7019601C701B6010F94B4
:10B1F000C11A9B01AC016D897E898F89988D0F944E
:10B20000BF1E6B017C01A5019401C501B4010F941F
:10B21000C01E9B01AC01C701B6010F949C1F03C067
:10B2200060E070E0CB010F943520F10182889388B3
:10B23000A488B58875016401C418D508E608F70824
:10B240000F940420C61AD70AE80AF90AF7FE6BC061
:10B2500020E030E0A90169817A818B819C810F9483
:10B260005C1A882309F447C029813A814B815C81AB
:10B27000CA01B9010F94C01E6B017C01C501B40164
:10B280000F94601A9B01AC01C701B6010F94C11A5B
:10B290006B017C0129893A894B895C89CA01B90112
:10B2A0000F94C11A9B01AC01C701B6010F94BF1ED8
:10B2B0006B017C012D813E814F815885CA01B90106
:10B2C0000F94C11A9B01AC01C701B6010F94C01EB7
:10B2D0006B017C0120E030E040E850E469817A8134
:10B2E0008B819C810F94C11A9B01AC01C701B601EF
:10B2F0000F949C1F03C060E070E0CB010F94861F89
:10B300000F9404202B013C0197FF03C0412C512CCA
:10B310003201481459046A047B0410F024013501F9
:10B32000C12CD12C76018FB7F894D1019C9193FD5B
:10B3300022C0F101468A578A608E718EC40CD51CDA
:10B34000E61CF71C5A96CD92DD92ED92FC925D9729
:10B3500029853A854B855C85DB962D933D934D93EE
:10B360005C93DE97FF962D853E854F855889208317
:10B370003183428353838FBF68960FB6F894DEBF44
:10B380000FBECDBFDF91CF911F910F91FF90EF9036
:10B39000DF90CF90BF90AF909F908F907F906F90F5
:10B3A0005F904F903F902F9008955F988EBD000062
:10B3B0000DB407FEFDCF8EB56EBD00000DB407FEC7
:10B3C000FDCF8EB55F9A0895CF93DF9300D01F9283
:10B3D0001F92CDB7DEB795E0E9EAF2E0DE01119603
:10B3E00001900D929A95E1F7E1E0F0E0EC0FFD1F7E
:10B3F000E80FF11D808190E00F900F900F900F905B
:10B400000F90DF91CF91D1CF8F929F92AF92BF9249
:10B41000CF92DF92EF92FF92CF93C82FC090150288
:10B42000D0901602E0901702F0901802A701960142
:10B43000C701B6010F946C21809085069090860616
:10B44000A0908706B0908806811129C0C11127C03D
:10B4500080918406882319F1A7019601C501B401E2
:10B460000F94BF1E209171083091720840917308AB
:10B47000509174080F94C11A0F94F1207195619541
:10B4800071098091A30E882351F08091740E9091E0
:10B49000750E860F971F9093750E8093740E809291
:10B4A000150290921602A0921702B0921802CF9144
:10B4B000FF90EF90DF90CF90BF90AF909F908F90D4
:10B4C00008950F931F93CF93DF93FC018491EF01B5
:10B4D0002196811102C010E004C00E94857FFE0108
:10B4E000F5CF03E0010F84E0189FE0011124FE0175
:10B4F000EB5EFD4E20E030E0A90160817181828128
:10B5000093810F94E62087FD03C08BE20E94857F24
:10B51000CB5EDD4E688179818A819B8146E00E9405
:10B52000B8E980E20E94857F1F5F1013DCCF8AE0BC
:10B530000E94857F1930A9F6DF91CF911F910F915D
:10B540000895AF92BF92CF92DF92EF92FF920F9346
:10B550001F93CF93C82F882319F0E2E3F6E10CC0C4
:10B56000E5EBFEE484918F010F5F1F4F8823A9F361
:10B570000E94857FF801F6CF84918F010F5F1F4FE6
:10B58000882321F00E94857FF801F6CFCC2319F0A3
:10B59000E5E1F6E10CC0E5EBFEE484918F010F5F7D
:10B5A0001F4F8823A9F30E94857FF801F6CF84916D
:10B5B0008F010F5F1F4F882321F00E94857FF801C4
:10B5C000F6CF8AE00E94857FC1112DC0E5EBFEE435
:10B5D00084918F010F5F1F4F882321F00E94857F88
:10B5E000F801F6CFE2E0F6E184918F010F5F1F4F83
:10B5F000882321F00E94857FF801F6CF80916606AE
:10B60000882321F08AE00E94857FC7C3E7EFF5E138
:10B6100084918F010F5F1F4F882309F4BEC30E94DE
:10B62000857FF801F5CF40916106509162066091E7
:10B630006306709164068EEE95E10E942EEA8AE020
:10B640000E94857F8091660681111BC0CC2319F072
:10B65000E3EEF5E10CC0E5EBFEE484918F010F5FB2
:10B660001F4F8823A9F30E94857FF801F6CF8491AC
:10B670008F010F5F1F4F882321F00E94857FF80103
:10B68000F6CFC11124C0E5EBFEE484918F010F5F7A
:10B690001F4F882321F00E94857FF801F6CFE2ED4D
:10B6A000F5E184918F010F5F1F4F882321F00E94E5
:10B6B000857FF801F6CFE5EBFEE484918F010F5F03
:10B6C0001F4F882321F00E94857FF801F6CF40911B
:10B6D000690850916A0860916B0870916C088AEC57
:10B6E00095E10E942EEA40916D0850916E0860919C
:10B6F0006F087091700887EC95E10E942EEA4091E6
:10B70000710850917208609173087091740884EC0C
:10B7100095E10E942EEA409175085091760860915B
:10B7200077087091780881EC95E10E942EEA8AE012
:10B730000E94857FC11124C0E5EBFEE484918F0156
:10B740000F5F1F4F882321F00E94857FF801F6CFFD
:10B75000E3EAF5E184918F010F5F1F4F882321F009
:10B760000E94857FF801F6CFE5EBFEE484918F011E
:10B770000F5F1F4F882321F00E94857FF801F6CFCD
:10B7800040916706509168066091690670916A065B
:10B790008AE995E10E942EEA40916B0650916C0671
:10B7A00060916D0670916E0687E995E10E942EEA20
:10B7B00040916F065091700660917106709172060B
:10B7C00084E995E10E942EEA409173065091740637
:10B7D000609175067091760681E995E10E942EEAE6
:10B7E0008AE00E94857FC11124C0E5EBFEE48491CC
:10B7F0008F010F5F1F4F882321F00E94857FF80182
:10B80000F6CFEFE6F5E184918F010F5F1F4F88239C
:10B8100021F00E94857FF801F6CFE5EBFEE48491EC
:10B820008F010F5F1F4F882321F00E94857FF80151
:10B83000F6CF4091A6115091A7116091A811709177
:10B84000A91186E695E10E944BEC4091AA11509116
:10B85000AB116091AC117091AD1183E695E10E943E
:10B860004BEC4091AE115091AF116091B0117091BD
:10B87000B11180E695E10E944BEC4091B2115091DC
:10B88000B3116091B4117091B5118DE595E10E94ED
:10B890004BEC8AE00E94857FC11124C0E5EBFEE4F9
:10B8A00084918F010F5F1F4F882321F00E94857FB5
:10B8B000F801F6CFE3E1F5E184918F010F5F1F4FAF
:10B8C000882321F00E94857FF801F6CFE5EBFEE4A6
:10B8D00084918F010F5F1F4F882321F00E94857F85
:10B8E000F801F6CF4091BE115091BF116091C01187
:10B8F0007091C1118AE095E10E942EEA4091BA113F
:10B900005091BB116091BC117091BD1187E095E120
:10B910000E942EEA4091B6115091B7116091B81172
:10B920007091B91184E095E10E942EEA8AE00E94AC
:10B93000857FC11124C0E5EBFEE484918F010F5F88
:10B940001F4F882321F00E94857FF801F6CFE0E9A0
:10B95000F4E184918F010F5F1F4F882321F00E9433
:10B96000857FF801F6CFE5EBFEE484918F010F5F50
:10B970001F4F882321F00E94857FF801F6CF409168
:10B98000640850916508609166087091670887E8BF
:10B9900094E10E942EEA4091600850916108609104
:10B9A00062087091630884E894E10E942EEA409155
:10B9B000991150919A1160919B1170919C1181E89D
:10B9C00094E10E944BEC4091860850918708609169
:10B9D0008808709189088EE794E10E942EEA4091D0
:10B9E0008A0850918B0860918C0870918D088BE7C4
:10B9F00094E10E942EEA40918E0850918F08609148
:10BA000090087091910888E794E10E942EEA409195
:10BA1000920850919308609194087091950885E779
:10BA200094E10E942EEA8AE00E94857FC11124C021
:10BA3000E5EBFEE484918F010F5F1F4F882321F017
:10BA40000E94857FF801F6CFE7E6F4E184918F014B
:10BA50000F5F1F4F882321F00E94857FF801F6CFEA
:10BA6000E5EBFEE484918F010F5F1F4F882321F0E7
:10BA70000E94857FF801F6CF4091A50E5091A60E49
:10BA80006091A70E7091A80E8EE594E10E942EEAB7
:10BA90004091A90E5091AA0E6091AB0E7091AC0E20
:10BAA0008BE594E10E942EEA4091AD0E5091AE0ECE
:10BAB0006091AF0E7091B00E88E594E10E942EEA7D
:10BAC0008AE00E94857FC11124C0E5EBFEE48491E9
:10BAD0008F010F5F1F4F882321F00E94857FF8019F
:10BAE000F6CFE4E4F4E184918F010F5F1F4F8823C8
:10BAF00021F00E94857FF801F6CFE5EBFEE484910A
:10BB00008F010F5F1F4F882321F00E94857FF8016E
:10BB1000F6CF6091840670E08BE394E10E948DC4BF
:10BB20008AE00E94857FCC2379F035E9A32E31E1AC
:10BB3000B32E41E9C42E41E1D42E5DE8E52E51E15A
:10BB4000F52E00E010E024C0E5EBFEE484918F01C7
:10BB50000F5F1F4F882321F00E94857FF801F6CFE9
:10BB6000EEE1F4E184918F010F5F1F4F882321F0F4
:10BB70000E94857FF801F6CFE5EBFEE484918F010A
:10BB80000F5F1F4F882389F20E94857FF801F6CF4F
:10BB9000B80185E194E10E948DC4F5016191719134
:10BBA0005F0182E194E10E948DC4F601619171917F
:10BBB0006F018FE094E10E948DC4F7016191719152
:10BBC0007F018CE094E10E948DC48AE00E94857F11
:10BBD0000F5F1F4F02301105D9F6C11124C0E5EBEC
:10BBE000FEE484918F010F5F1F4F882321F00E9494
:10BBF000857FF801F6CFEDEFF3E184918F010F5FC0
:10BC00001F4F882321F00E94857FF801F6CFE5EBD6
:10BC1000FEE484918F010F5F1F4F882321F00E9463
:10BC2000857FF801F6CF4091AB105091AC10609138
:10BC3000AD107091AE1084EF93E10E942EEA2CEAD1
:10BC400035EC47E25EE36091A7107091A8108091F7
:10BC5000A9109091AA100F949C1FAB01BC0181EF19
:10BC600093E10E94DAEA2CEA35EC47E25EE3609168
:10BC7000A3107091A4108091A5109091A6100F941C
:10BC8000C11AAB01BC018EEE93E10E94DAEA8AE0B0
:10BC90000E94857FC1110CC0E5EBFEE484918F0109
:10BCA0000F5F1F4F882321F00E94857FF801F6CF98
:10BCB00040917F06509180066091810670918206C6
:10BCC00085EE93E10E942EEA2CEA35EC47E25EE332
:10BCD00060917B0670917C0680917D0690917E0636
:10BCE0000F949C1FAB01BC0182EE93E10E94DAEA43
:10BCF0002CEA35EC47E25EE36091770670917806B6
:10BD00008091790690917A060F94C11AAB01BC011B
:10BD10008FED93E10E94DAEA8AE00E94857FC111EB
:10BD200024C0E5EBFEE484918F010F5F1F4F882351
:10BD300021F00E94857FF801F6CFE9ECF3E18491D0
:10BD40008F010F5F1F4F882321F00E94857FF8012C
:10BD5000F6CFE5EBFEE484918F010F5F1F4F882340
:10BD600021F00E94857FF801F6CF40918506509121
:10BD70008606609187067091880680EC93E10E94A8
:10BD80002EEA8AE0CF911F910F91FF90EF90DF9004
:10BD9000CF90BF90AF900C94857FE5EBFEE484914B
:10BDA0008F010F5F1F4F882309F43DCC0E94857FD0
:10BDB000F801F5CF2F923F924F925F926F927F9250
:10BDC0008F929F92AF92BF92CF92DF92EF92FF92AB
:10BDD0000F931F93CF93DF93CDB7DEB7C857D10929
:10BDE0000FB6F894DEBF0FBECDBF5B014A0139012B
:10BDF000EBAAFFAE21960FAF219722961FAF229795
:10BE0000CFA62091690830916A0840916B08509143
:10BE10006C08DC016D917D918D919C910F94C11AFC
:10BE20000F94F120E0966CAF7DAF8EAF9FAFE0979F
:10BE300020916D0830916E0840916F085091700804
:10BE4000F50160817181828193810F94C11A0F94F1
:10BE5000F120E4966CAF7DAF8EAF9FAFE497209159
:10BE60007108309172084091730850917408D401A0
:10BE70006D917D918D919C910F94C11A0F94F12039
:10BE8000E8966CAF7DAF8EAF9FAFE89720917508B5
:10BE9000309176084091770850917808F3016081DD
:10BEA0007181828193810F94C11A0F94F120699658
:10BEB0006CAF7DAF8EAF9FAF699780914D1290911F
:10BEC0004E12A0914F12B0915012E096CCACDDAC66
:10BED000EEACFFACE097C81AD90AEA0AFB0A8091D7
:10BEE000511290915212A0915312B0915412E496B3
:10BEF0008CAC9DACAEACBFACE497881A990AAA0A88
:10BF0000BB0A8091551290915612A0915712B09190
:10BF10005812E8962CAD3DAD4EAD5FADE897281BAD
:10BF2000390B4A0B5B0B2BAF3CAF4DAF5EAF809133
:10BF30009D0683FF0EC069964CAD5DAD6EAD7FADC5
:10BF400069974093591250935A1260935B12709301
:10BF50005C128091591290915A12A0915B12B0918B
:10BF60005C1269964CAC5DAC6EAC7FAC6997481ABC
:10BF7000590A6A0A7B0A09F495C0809183068111E7
:10BF800041C06091120270911302882777FD80955D
:10BF9000982F0F94621A9B01AC0160915606709124
:10BFA000570680915806909159060F945C1A87FFA6
:10BFB00029C069966CAD7DAD8EAD9FAD69976093DC
:10BFC000591270935A1280935B1290935C12E5EBB6
:10BFD000FEE484918F010F5F1F4F882321F00E94A0
:10BFE000857FF801F6CFE2EBF6E184918F010F5FD8
:10BFF0001F4F882321F00E94857FF801F6CF412C46
:10C00000512C32014BA65CA66DA67EA677FE0BC016
:10C0100088279927DC0184199509A609B7098BA7F8
:10C020009CA7ADA7BEA76091750870917608809116
:10C030007708909178080F9404209B01AC01A8EC3C
:10C04000B0E00F94A01E2BA53CA54DA55EA56217E0
:10C050007307840795074CF569964CAD5DAD6EADE1
:10C060007FAD69974093591250935A1260935B12B7
:10C0700070935C12E5EBFEE484918F010F5F1F4F1C
:10C08000882321F00E94857FF801F6CFE3E9F6E1ED
:10C0900084918F010F5F1F4F882321F00E94857FBD
:10C0A000F801F6CF412C512C3201D701C601882767
:10C0B000B7FD83959927AA27BB278BA7B7FE03C097
:10C0C000582F52605BA76BAD7CAD8DAD9EAD97FFD9
:10C0D00003C07BA574607BA777FE03C08BA5886037
:10C0E0008BA79FA5092F10E0C301B2010F94621A1C
:10C0F000F801EE0FFF1FEE0FFF1FE453F94F2081F1
:10C100003181428153810F94C11A2B013C01F80106
:10C11000EE0FFF1FEC55FD4F60817181882777FD81
:10C120008095982F0F94621A9B01AC01C301B20154
:10C130000F94C11A2AE037ED43E25CE30F94C11A71
:10C140002B013C0120E030E0A9010F94E6201816F5
:10C150004CF420E030E040E05FE3C301B2010F9413
:10C16000C01E08C0A301920160E070E080E09FE380
:10C170000F94BF1E0F9404206FAB78AF89AF9AAFB6
:10C18000A0915D12AF5FAF706596AFAF659780917C
:10C190005E126596BFAD65978B1304C080E00E9468
:10C1A0006BFCF5CF80915D12EFE48E9F100111249E
:10C1B00091012B5B364F1901D9011C92EBA5929688
:10C1C000EC9397018601F7FE07C00027112798011D
:10C1D0000C191D092E093F09D10112960D931D93CB
:10C1E0002D933C9315978BA69CA6ADA6BEA6B7FE35
:10C1F0000BC044275527BA01481959096A097B0918
:10C200004BA75CA76DA77EA76BA57CA58DA59EA55A
:10C21000D10116966D937D938D939C9319974BAD99
:10C220005CAD6DAD7EAD77FF07C0709560955095A4
:10C2300041955F4F6F4F7F4FF1014287538764876E
:10C2400075878FA998ADA9ADBAAD86879787A08B62
:10C25000B18B8BA59CA5ADA5BEA580179107A207A4
:10C26000B30714F4D901C80184179507A607B707C7
:10C2700014F4DB01CA014FA958AD69AD7AAD481776
:10C2800059076A077B0714F0DB01CA01F101828BB1
:10C29000938BA48BB58B0697A105B10510F40C9474
:10C2A000016B80919D1190919E11E95BFF4F9183ED
:10C2B000808380919F119091A01132969183808309
:10C2C000EFA5D1011196EC93012B022B032B09F062
:10C2D0001798F10186819781A085B185892B8A2BDA
:10C2E0008B2B09F01698F10182859385A485B5857D
:10C2F000892B8A2B8B2B09F015982FA938AD49ADC6
:10C300005AAD232B242B252BD9F08091CB068823E3
:10C3100019F081508093CB063FA5311104C01498C9
:10C3200080E28093CB06B0916408BBA7E0916508DA
:10C33000EFA700916608109167082B2F3E2F0CC0C5
:10C34000309160083BA7409161084FA700916208B7
:10C3500010916308232F342FA8016BA97FAD21967C
:10C360008FAD219722969FAD22970F945C1A87FD7F
:10C3700002C00C94F56AC701B6010F94621A2091AD
:10C38000C60E3091C70E4091C80E5091C90E0F9441
:10C39000C11A6BAB7CAB8DAB9EAB698B7A8B8B8BF5
:10C3A0009C8BC501B4010F94621A2091CA0E309182
:10C3B000CB0E4091CC0E5091CD0E0F94C11A4B0173
:10C3C0005C016D8B7E8B8F8B988F6BAD7CAD8DAD53
:10C3D0009EAD0F94621A2091CE0E3091CF0E4091F7
:10C3E000D00E5091D10E0F94C11A6B017C01698F50
:10C3F0007A8F8B8F9C8F2091D20E3091D30E4091EB
:10C40000D40E5091D50EC301B2010F94C11A6D8F95
:10C410007E8F8F8F98A3D10112964D905D906D9075
:10C420007C901597B6E04B165104610471040CF52D
:10C43000F1014680578060847184F6E04F16510404
:10C4400061047104B4F4D1011A964D905D906D9021
:10C450007C901D97B6E04B165104610471044CF4B6
:10C46000DC01CB01BF77F10187A790ABA1ABB2ABE9
:10C470002DC02BA93CA94DA95EA9CA01B9010F94F1
:10C48000C11A2B013C01A5019401C501B4010F940F
:10C49000C11A9B01AC01C301B2010F94C01E4B0134
:10C4A0005C01A7019601C701B6010F94C11A9B0157
:10C4B000AC01C501B4010F94C01E0F942B21D10112
:10C4C0009F966D937D938D939C93D297F10127A5B1
:10C4D00030A941A952A960E070E080E89FE30F9481
:10C4E0009C1F27966CAF7DAF8EAF9FAF27979B01A8
:10C4F000AC016BA57FA5C8010F94C11A2B013C01AB
:10C500000F941A032C968FAF2C97A301920160E031
:10C5100074E284E799E40F949C1F0F94F1206B015F
:10C520007C012C968FAD2C978250863008F044C049
:10C530008091991190919A11A0919B11B0919C11A9
:10C54000C816D906EA06FB06B8F5BC01CD016C1980
:10C550007D098E099F09660F771F881F991F2C96EA
:10C56000FFAD2C970F2F10E020E030E0A9019801DB
:10C570000F94621ECA01B9010F94601A0F94F12042
:10C580006C0D7D1D8E1D9F1D0F94601A9B01AC01CB
:10C5900060E074E284E799E40F949C1F2B013C0156
:10C5A0009B01AC0160E074E284E799E40F949C1F66
:10C5B0000F94F1206B017C012FB7F8948091410911
:10C5C00090914209A0914309B09144098C0D9D1DA1
:10C5D000AE1DBF1D8093410990934209A09343096A
:10C5E000B09344092FBFD1019F962D913D914D915C
:10C5F0005C91D297A3962CAF3DAF4EAF5FAFA397A0
:10C60000A3019201A3966CAD7DAD8EAD9FADA397B6
:10C610000F94C11A2B966CAF7DAF8EAF9FAF2B9747
:10C62000F10163A374A385A396A322893389448966
:10C6300055892BA73CA74DA75EA7CA01B9010F9446
:10C64000601A6BAF7CAF8DAF9EAFA30192010F94C8
:10C65000C11A0F94861F0F9409206B017C01F10110
:10C6600067AB70AF81AF92AF9E012F5E3F4F2396B5
:10C670003FAF2EAF239747E656E064965FAF4EAFCD
:10C680006497BE016F5D7F4F7AA769A7CE010196BF
:10C6900062969FAF8EAF62971FA61BAA90E89FAFCE
:10C6A000AFE32196AFAF21972396EEADFFAD239771
:10C6B00061917191819191912396FFAFEEAF239794
:10C6C000A30192010F94C11A6296AEADBFAD6297FD
:10C6D0006D937D938D939D936296BFAFAEAF62973E
:10C6E0009B01AC015F7760962CAF3DAF4EAF5FAF63
:10C6F00060976496AEADBFAD64978D909D90AD9000
:10C70000BD906496BFAFAEAF6497A50194016096EB
:10C710006CAD7DAD8EAD9FAD60970F94E620181681
:10C7200014F560962CAD3DAD4EAD5FAD6097C50183
:10C73000B4010F949C1F162F072FB82EA92E262F59
:10C74000372F482F592F6FA57BA98FAD21969FAD0D
:10C7500021970F94E620181634F41FA70BABBFAE39
:10C760002196AFAE21972396EEADFFAD239729A575
:10C770003AA5E217F30709F097CF20E030E040E850
:10C780005FE36FA57BA98FAD21969FAD21970F9495
:10C790005C1A87FF45C05E0131E1A30EB11C8E011A
:10C7A0000F5F1F4F2FA53BA94FAD21965FAD21977E
:10C7B000D8016D917D918D919C910F94C11AF801D2
:10C7C00061937193819391938F01EA15FB0551F762
:10C7D0002FA53BA94FAD21965FAD21972B966CAD50
:10C7E0007DAD8EAD9FAD2B970F94C11AD10193965D
:10C7F0006D937D938D939C939697C701B6010F948B
:10C80000601A2FA53BA94FAD21965FAD21970F94DC
:10C81000C11A0F940920F10167AB70AF81AF92AFDD
:10C8200027962CAD3DAD4EAD5FAD27976BAD7CAD82
:10C830008DAD9EAD0F94C11A6BAB7CAB8DAB9EAB37
:10C84000D10112968D909D90AD90BC901597169643
:10C850004D905D906D907C9019971A962D913D9119
:10C860004D915C911D972FA738AB49AB5AAB811402
:10C870009104A104B104B1F44114510461047104A0
:10C8800089F4232B242B252B69F42091BA113091A4
:10C89000BB114091BC115091BD110F94C11A0F945E
:10C8A000861F00C22FA938AD49AD5AAD232B242BCA
:10C8B000252B49F06091BE117091BF118091C0117C
:10C8C0009091C11108C06091B6117091B71180911B
:10C8D000B8119091B9112BA93CA94DA95EA90F944B
:10C8E000C11A0F94861F0F9409206B017C0180915F
:10C8F000C7069091C806A091C906B091CA06F10179
:10C9000046855785608971894FAB58AF69AF7AAF5B
:10C910002BA53CA54DA55EA582179307A407B507D7
:10C9200008F4CCC081149104A104B10471F12091E8
:10C930007C1130917D1140917E1150917F112C1509
:10C940003D054E055F0508F56BA57CA58DA59EA54B
:10C950000F94531E6BAF7CAF8DAF9EAFA7019601B6
:10C96000C501B4010F94531E2BAD3CAD4DAD5EAD72
:10C97000261737074807590740F4CA01B901A5012E
:10C9800094010F94621E69017A01411451046104FB
:10C99000710441F1209180113091811140918211F7
:10C9A000509183112C153D054E055F05D8F46BA5FC
:10C9B0007CA58DA59EA50F94531E4B015C01A7017C
:10C9C0009601C301B2010F94531E86169706A8065E
:10C9D000B90640F4C501B401A30192010F94621E8F
:10C9E00069017A014FA558A969A97AA9452B462B57
:10C9F000472B61F12091841130918511409186116E
:10CA0000509187112C153D054E055F05F8F46BA577
:10CA10007CA58DA59EA50F94531E4B015C01A7011B
:10CA200096016FA578A989A99AA90F94531E861615
:10CA30009706A806B90650F4C501B4012FA538A978
:10CA400049A95AA90F94621E69017A016FA978ADAC
:10CA500089AD9AAD672B682B692B09F427C120910A
:10CA600088113091891140918A1150918B112C15A8
:10CA70003D054E055F0508F019C16BA57CA58DA588
:10CA80009EA50F94531E4B015C01A70196016FA94F
:10CA900078AD89AD9AAD0F94531E86169706A806F9
:10CAA000B90608F003C1C501B4012FA938AD49ADDD
:10CAB0005AAD0F94621E69017A01F8C08114910485
:10CAC000A104B104D9F160917C1170917D11809124
:10CAD0007E1190917F116C157D058E059F0570F577
:10CAE0000F94601A2BAD3CAD4DAD5EAD0F94C11AE5
:10CAF0006BA77CA78DA79EA7C501B4010F94621AEE
:10CB00004B015C01C701B6010F94601AA5019401A5
:10CB10000F94C11A2BA53CA54DA55EA50F94E62048
:10CB2000181664F4A50194016BA57CA58DA59EA59E
:10CB30000F949C1F0F9409206B017C014114510438
:10CB400061047104A9F1609180117091811180914B
:10CB50008211909183116C157D058E059F0540F51E
:10CB60000F94601A2BAD3CAD4DAD5EAD0F94C11A64
:10CB70004B015C01C301B2010F94621A2B013C010D
:10CB8000C701B6010F94601AA30192010F94C11A54
:10CB9000A50194010F94E620181654F4A301920104
:10CBA000C501B4010F949C1F0F9409206B017C01F7
:10CBB0008FA598A9A9A9BAA9892B8A2B8B2BB9F182
:10CBC00060918411709185118091861190918711E7
:10CBD0006C157D058E059F0550F50F94601A2BADE1
:10CBE0003CAD4DAD5EAD0F94C11A4B015C016FA51C
:10CBF00078A989A99AA90F94621A2B013C01C7014F
:10CC0000B6010F94601AA30192010F94C11AA501F5
:10CC100094010F94E620181654F4A3019201C50163
:10CC2000B4010F949C1F0F9409206B017C012FA964
:10CC300038AD49AD5AAD232B242B252BB9F160918A
:10CC400088117091891180918A1190918B116C15C6
:10CC50007D058E059F0550F50F94601A2BAD3CADF8
:10CC60004DAD5EAD0F94C11A4B015C016FA978AD5B
:10CC700089AD9AAD0F94621A2B013C01C701B60130
:10CC80000F94601AA30192010F94C11AA501940197
:10CC90000F94E620181654F4A3019201C501B401C3
:10CCA0000F949C1F0F9409206B017C01F101ED5B37
:10CCB000FF4FC082D182E282F382C701B6010F9496
:10CCC000601A6B017C012BA93CA94DA95EA90F94A8
:10CCD0009C1FA7966CAF7DAF8EAF9FAFA797D1017A
:10CCE000D3966D937D938D939C93D69720E030E0FF
:10CCF00040E85BE4C701B6010F94C11A20E034E2BA
:10CD000044EF59E40F949C1F0F940420F101668FA7
:10CD1000778F80A391A3F3A1FBAFD1019496BC912F
:10CD2000BFA7F101F5A1FBABD1019696BC91BFAFB6
:10CD30002E01E1E14E0E511C26E838E03CA72BA75E
:10CD4000AE014F5F5F4F3A015BAD21965FAF219718
:10CD50006FA522966FAF22972496FFAF249728964F
:10CD6000BFAF289710E0D3018D909D90AD90BD90FE
:10CD70003D01E894B7F8EBA5FCA5C190D190E190F6
:10CD8000F190FCA7EBA7A7019601C501B4010F9490
:10CD9000E62018160CF042C0112399F12BAD3FA5E7
:10CDA0004BA95FADC701B6010F94C11A6B017C019D
:10CDB00021962FAD219722963FAD229724964FAD15
:10CDC000249728965FAD2897C501B4010F94C11A26
:10CDD000A70196010F94E6201816FCF4A501940112
:10CDE000C701B6010F949C1F21966FAF2197229621
:10CDF0007FAF229724968FAF249728969FAF2897CE
:10CE00000CC02196CFAE21972296DFAE22972496B2
:10CE1000EFAE24972896FFAE289711E064147504AE
:10CE200009F0A1CF2C96FFAD2C97F23008F485C104
:10CE3000209139122BA730913A123FAB00913B124F
:10CE400010913C1227E137EB41ED58E36BA57FA928
:10CE5000C8010F94E62018160CF06FC141E0A896A7
:10CE60004FAFA8972BAD3FA54BA95FAD6BA57FA991
:10CE7000C8010F94E62018169CF0A8961FAEA8973C
:10CE80002BAD3FA54BA95FAD6BA57FA9C8010F9442
:10CE90009C1F6F966CAF7DAF8EAF9FAF6F9715C025
:10CEA0002BA53FA9A8016BAD7FA58BA99FAD0F94C2
:10CEB0009C1F6F966CAF7DAF8EAF9FAF6F975BADD2
:10CEC0005BA76FA56FAB0BA91FAD8DE392E16B96CE
:10CED0009FAF8EAF6B97A6E8B8E0AA96BFAFAEAF94
:10CEE000AA97FE013196AC96FFAFEEAFAC97412CFE
:10CEF000512C40E8642E4FE3742E63961FAE639767
:10CF00006B96AEADBFAD6B97CD90DD90ED90FD9083
:10CF10006B96BFAFAEAF6B97AC96EEADFFADAC9777
:10CF200081909190A190B190AC96FFAFEEAFAC978D
:10CF3000A896FFADA897FF2361F06F962CAD3DAD8D
:10CF40004EAD5FAD6F97C701B6010F94C11A6B016B
:10CF50007C0163962FAD6397222381F0A301920198
:10CF6000C701B6010F94C11A6B017C01A3019201A4
:10CF7000C501B4010F94C11A4B015C01A5019401D4
:10CF8000C701B6010F94E62020E030E0A901181691
:10CF9000CCF4C501B4010F94E62018164CF020E043
:10CFA00030E0A901C701B6010F945C1A87FF05C0E4
:10CFB000A5019401C701B60118C0B7FAB094B7F83B
:10CFC000B09424C0C501B4010F945C1A87FD09C058
:10CFD00020E030E0A901C701B6010F94E620181641
:10CFE0008CF4A7019601C501B4010F94BF1E2C96C5
:10CFF0006FAF2C972D967FAF2D9761968FAF61976E
:10D00000B92E20C0F7FAF094F7F8F094A501940136
:10D01000C701B6010F94E62018165CF42C96CFAE2B
:10D020002C972D96DFAE2D976196EFAE6197BF2CB2
:10D0300009C02C968FAE2C972D969FAE2D9761969A
:10D04000AFAE6197AA96AEADBFADAA97CD90DD9079
:10D05000ED90FD90AA96BFAFAEAFAA97A70196013B
:10D060002C966FAD2C972D967FAD2D9761968FAD39
:10D0700061979B2D0F94E6201816ECF42C962FAD9B
:10D080002C972D963FAD2D9761964FAD61975B2DF7
:10D09000C701B6010F949C1F9B01AC01C301B201F3
:10D0A0000F94C11A2B013C016396BFAD6397BF5F1C
:10D0B0006396BFAF63976B96EEADFFAD6B97ED5484
:10D0C000F24109F01DCF63963FAD6397332351F0D2
:10D0D000A30192016BA57FA9C8010F94C11A6BA788
:10D0E0007FAB8C0124EA30E74DE75FE36BA57FA9B6
:10D0F000C8010F94C11A6B017C019B01AC016091C6
:10D10000C3067091C4068091C5069091C6060F941F
:10D11000E620181624F5A701960121966FAD2197F8
:10D1200022967FAD229724968FAD249728969FADA7
:10D1300028970F94E620181694F4D1018C918460FE
:10D140008C932196BFAD2197BBA72296EFAD229776
:10D15000EFAB24960FAD249728961FAD28978BA58B
:10D160009FA9D801F10183A794A7A5A7B6A7A79661
:10D170006CAD7DAD8EAD9FADA79790589B01AC0176
:10D180000F94C01EA3962CAD3DAD4EAD5FADA397E1
:10D190000F94C11A9B01AC016BE077ED83E29BE336
:10D1A0000F94BF1E0F942B21762E872EF82EE92E7A
:10D1B000262F372F482F592F6BA57FA9C8010F9411
:10D1C0005C1A87FF05C09BA4AFA8B02EC12E04C077
:10D1D000972CA82CBF2CCE2C892D9A2DAB2DBC2D95
:10D1E000F10187A390A7A1A7B2A7D080272D382D42
:10D1F0004F2D5E2D6BAD7FA58BA99FAD0F945C1A53
:10D20000181614F083E001C081E0D82AD101DC9225
:10D2100080E1FE013196ADE3B2E101900D928A9575
:10D22000E1F78BAD9FA5ABA9BFAD80933912909369
:10D230003A12A0933B12B0933C1221968FAD2197E6
:10D2400022969FAD22972496AFAD24972896BFAD26
:10D2500028978093C3069093C406A093C506B09305
:10D26000C6062BAD3FA54BA95FADBC01CD010F9408
:10D270009C1F6DA37EA38FA398A72BAD3FA54BA9A1
:10D280005FAD692D7A2D8B2D9C2D0F949C1F69A36A
:10D290007AA38BA39CA3AE014B5D5F4FBE016F5D74
:10D2A0007F4FC1010E9401586596BFAD6597B0934D
:10D2B0005D12E0962CAD3DAD4EAD5FADE097209395
:10D2C0004D1230934E1240934F1250935012E496E9
:10D2D0004CAD5DAD6EAD7FADE49740935112509370
:10D2E00052126093531270935412E8966CAD7DAD58
:10D2F0008EAD9FADE8976093551270935612809350
:10D3000057129093581269968CAD9DADAEADBFADDE
:10D3100069978093591290935A12A0935B12B0931D
:10D320005C120F941A03843048F420915E12E12CB1
:10D33000F12C80E090E03FE4D32EAAC090915E12E1
:10D340009BA7B0905D12ADEFBA0EBB2DBF70BB2E88
:10D35000C12CD12CE12CF12CFBA5BF1631F3E1142B
:10D36000F10421F0F701808182FDDFCFBA94FB2D1B
:10D37000FF70BF2E2FE42F9F800111240B5B164FEF
:10D38000E114F10409F476C0C114D10409F472C0A7
:10D39000D7019B967C909B979C968C909C979D9692
:10D3A0009C909D979E96AC909E97272D382D492D49
:10D3B0005A2D97966D917D918D919C919A970F948E
:10D3C0005C1A882309F456C0F701608061FC46C0EE
:10D3D000D60197962D903D904D905C909A97A20122
:10D3E0009101672D782D892D9A2D0F945C1A1816AE
:10D3F000ACF5A2019101C201B1010F94C11A1B0148
:10D400002C01F70183A994A9A5A9B6A9BC01CD0156
:10D4100090589B01AC010F94C01ED7019F962D918F
:10D420003D914D915C91D2970F94C11A9B01AC0133
:10D43000C201B1010F94BF1E0F942B211B016C017F
:10D440009B01AC01672D782D892D9A2D0F945C1AC4
:10D4500087FD04C0722C832C9C2CAD2C872D982D1D
:10D46000A92DBA2DF70187A390A7A1A7B2A7862D52
:10D4700081608083670178016FCFD29E8001112483
:10D480000B5B164F009749F42F5F2F70C70178018F
:10D4900030915D122313F1CF0EC0DC013C9131FDC0
:10D4A000F3CFB701E9962FAFE9970E940F7EE99677
:10D4B0002FADE997E9CF009739F0FC01208121FDDC
:10D4C00003C0B7010E940F7E90905E1200E010E052
:10D4D0008FE4882E892D992787FD909520915D12E4
:10D4E00030E08217930709F44AC0889E5001899E54
:10D4F000B00C112495012B5B364F59010115110514
:10D50000C1F1D8018C9180FD04C0F901808180FFB8
:10D5100030C0D8019396CD90DD90ED90FC90969719
:10D52000A7019601F50167A170A581A592A50F94A9
:10D530009C1F69A37AA38BA39CA3A7019601D80182
:10D5400097966D917D918D919C919A970F949C1FC8
:10D550006DA37EA38FA398A7AE014F5D5F4FBE0161
:10D560006B5D7F4FC8010E940158F80180818E7F5A
:10D5700080839394F92DFF709F2E8501ABCF011509
:10D58000110569F1D8019396CD90DD90ED90FC9056
:10D590009697A70196016DEC7CEC8CE49DE30F94CB
:10D5A0009C1F69A37AA38BA39CA3A7019601F801F2
:10D5B00067A170A581A592A50F949C1F6DA37EA362
:10D5C0008FA398A7AE014F5D5F4FBE016B5D7F4F8C
:10D5D000C8010E940158D8018C918E7F8C93809154
:10D5E0006F00826080936F000CC0FBA9FBA72FAD7A
:10D5F0002FA721960FAD219722961FAD22970C944D
:10D60000BB61C858DF4F0FB6F894DEBF0FBECDBF69
:10D61000DF91CF911F910F91FF90EF90DF90CF900E
:10D62000BF90AF909F908F907F906F905F904F9042
:10D630003F902F9008954F925F926F927F928F92BA
:10D640009F92AF92BF92CF92DF92EF92FF920F9391
:10D650001F93CF93DF93CDB7DEB72E970FB6F89415
:10D66000DEBF0FBECDBF109119021F3FE9F00F942E
:10D67000A204C090D006D090D106E090D206F090DF
:10D68000D3066C197D098E099F0997FD0DC0209165
:10D690005E1280915D1230E090E001968F709927C4
:10D6A0002817390709F02DC20E9447DE8091E8064D
:10D6B00082FF3EC08091E70681113CC091E09093CB
:10D6C000E7068091BB0889278093C2111092BB089E
:10D6D00083E08093A8021092E8060F94A2046C5095
:10D6E0007E4F8F4F9F4F6093D4067093D5068093E3
:10D6F000D6069093D70688E893E19E878D8782E0CF
:10D7000090E09A838983BE01635F7F4FCE010196CB
:10D710000E943A8A16E0115069F08FE592E10E946A
:10D720008B5562E070E080E090E00F940F04F3CF3F
:10D730001092E706F9B0F4FAFF24F0F881E0F82639
:10D740004091E6062F2D30E0842F90E0281739070E
:10D75000A9F0FF2009F428C20E9408528091E60631
:10D76000823029F060E084E197E10E94CBDEF09204
:10D77000E60683E08093A8020E944F920F94A204D1
:10D780006B017C018091E2069091E306A091E40692
:10D79000B091E506A7019601281B390B4A0B5B0BDC
:10D7A00057FF05C08091E106882309F449C2D701DB
:10D7B000C6018C599F4FAF4FBF4F8093E2069093A5
:10D7C000E306A093E406B093E5068091E006181600
:10D7D0002CF48091E006823074F408C08091E00659
:10D7E000992781950CF4909502972CF48091C211A1
:10D7F00081119DC0ADC08091CA11882309F470C009
:10D800008091E00618165CF48091E006992787FD68
:10D81000909597FD0196BC01759567950DC0809117
:10D82000E006992787FD909597FD01969595879538
:10D8300066277727681B790B8090A1119090A21121
:10D84000A090A311B090A41181149104A104B1047B
:10D8500029F421E030E040E050E039C0882777FD2E
:10D860008095982F0F94621A2B013C01C701B601D5
:10D87000681979098A099B090F94601A9B01AC0108
:10D88000C301B2010F949C1F20E030E04AE754E44A
:10D890000F94C11A4B015C0120E030E040E253E4F8
:10D8A0000F94E62087FF0FC020E030E046E952E405
:10D8B000C501B4010F94E62087FDCBCF2AE030E00C
:10D8C00040E050E004C024E630E040E050E0C09288
:10D8D000A111D092A211E092A311F092A41104C060
:10D8E00021E030E040E050E0A091E006BB27A7FD3A
:10D8F000B0950F94AA1E22E030E040E050E00F9473
:10D90000841E8091C6119091C711A091C811B09149
:10D91000C911820F931FA41FB51F8093C611909346
:10D92000C711A093C811B093C9111092E006D70196
:10D93000C6018856954CAF4FBF4F8093DC0690933D
:10D94000DD06A093DE06B093DF0681E08093A80297
:10D9500020912B0230912C0245E42F3D340749F4ED
:10D9600080911A029FEF980F90931A02882309F46E
:10D9700026C1285D3E4979F48091D9069091D80658
:10D98000891748F490911A022FEF290F20931A0259
:10D99000992309F424C12FB7F894809141099091FB
:10D9A0004209A0914309B09144092FBF4091A802B8
:10D9B000411105C02091E106222309F465C02AE047
:10D9C000B695A795979587952A95D1F7009721E069
:10D9D000A207B10520F08FEF9FEFA0E0B0E0969591
:10D9E0008795009741F02091DA063091DB062817E1
:10D9F000390708F049C08091E106811111C0423019
:10DA000050F0443028F0443031F41092A80203C0A2
:10DA100081E08093A8020E943F5681E08093E10656
:10DA200084E00E9462A781E08093FB11E0912B02C9
:10DA3000F0912C0219951092C2118091E106882371
:10DA400051F00E94DCC591E0811101C090E09093FB
:10DA5000E1069111DCC08090DA069090DB06A12CE3
:10DA6000B12C0F94A2046C197D098E099F098616AA
:10DA70009706A806B90640F40F94A2046C197D0914
:10DA80007093DB066093DA0680912B0290912C0252
:10DA90008F5D954421F080918A06882379F048E9CA
:10DAA000C40E4AE3D41EE11CF11CC092DC06D092E5
:10DAB000DD06E092DE06F092DF060FC08091DC0604
:10DAC0009091DD06A091DE06B091DF06C81AD90A52
:10DAD000EA0AFB0AF7FE0E94E4E18091E106811167
:10DAE000AFC08091A802813049F008F4A9C0843009
:10DAF00008F0A6C081E08093A802A2C01092A802FC
:10DB00009FC054E01502F0011124E05DFC4F20E0BD
:10DB100030E040E752E460817181828193810F940B
:10DB20009C1F4B015C018091B10E9091B20EA091AF
:10DB3000B30EB091B40E89839A83AB83BC8380917A
:10DB4000B50E9091B60EA091B70EB091B80E8D8320
:10DB50009E83AF83B8878091B90E9091BA0EA09141
:10DB6000BB0EB091BC0E89879A87AB87BC87AE018C
:10DB7000475F5F4FBE016B5F7F4FCE0101960E94F2
:10DB800074DDC12C850174012DEB3EE0AE01475FD1
:10DB90005F4FBE016B5F7F4FCE0101960E94DA5E40
:10DBA0008FEF8093190280CD1092A7121092A812C5
:10DBB000423009F4DCCD60E087E097E1D6CD8CE01F
:10DBC00080931A028091DA069091DB060197909378
:10DBD000DB068093DA0681E08093A802CACE96E045
:10DBE00090931A0291E09093A8028F5F8093D906D8
:10DBF000D701C6018856954CAF4FBF4F8093DC06C6
:10DC00009093DD06A093DE06B093DF06C4CE80902D
:10DC1000DA069090DB06A12CB12C0F94A2046C19AB
:10DC20007D098E099F0986169706A806B90640F455
:10DC30000F94A2046C197D097093DB066093DA06D9
:10DC40002E960FB6F894DEBF0FBECDBFDF91CF91F9
:10DC50001F910F91FF90EF90DF90CF90BF90AF900A
:10DC60009F908F907F906F905F904F900895CF928C
:10DC7000EF92FF920F931F93CF93DF93CDB7DEB751
:10DC80002C970FB6F894DEBF0FBECDBFC0909206A2
:10DC90008091B90E9091BA0EA091BB0EB091BC0EBE
:10DCA0004091B50E5091B60E6091B70E7091B80EBE
:10DCB0000091B10E1091B20E2091B30E3091B40EBE
:10DCC00009831A832B833C834D835E836F8378871C
:10DCD00089879A87AB87BC87AE01475F5F4FBE01DC
:10DCE0006B5F7F4FCE0101960E9474DDE0900A02C7
:10DCF000F0900B0200910C0210910D022DEB3EE012
:10DD0000AE01475F5F4FBE016B5F7F4FCE01019653
:10DD10000E94DA5E2C960FB6F894DEBF0FBECDBF20
:10DD2000DF91CF911F910F91FF90EF90CF900895C9
:10DD30008F929F92AF92BF92CF92EF92FF920F93EA
:10DD40001F93CF93DF93CDB7DEB72C970FB6F89420
:10DD5000DEBF0FBECDBF4B015C01C090920680912B
:10DD60003E0490913F04A0914004B0914104409141
:10DD70003A0450913B0460913C0470913D04009141
:10DD80003604109137042091380430913904098306
:10DD90001A832B833C834D835E836F8378878987C7
:10DDA0009A87AB87BC87AE01475F5F4FBE016B5F51
:10DDB0007F4FCE0101960E9474DD8501740122E43B
:10DDC00034E0AE01475F5F4FBE016B5F7F4FCE0116
:10DDD00001960E94DA5E2C960FB6F894DEBF0FBE55
:10DDE000CDBFDF91CF911F910F91FF90EF90CF901A
:10DDF000BF90AF909F908F900895CF92DF92EF9257
:10DE0000FF9280911402882309F4F1C00E94FFAEB2
:10DE100086E394E00F9465010F94D70480919D06EA
:10DE200083FD93C0C0904204D0904304E09044042A
:10DE3000F09045042091BD0E3091BE0E4091BF0E72
:10DE40005091C00EC701B6010F945C1A882309F4E3
:10DE50007CC08091830681113AC06091120270915A
:10DE60001302882777FD8095982F0F94621A9B01E3
:10DE7000AC016091560670915706809158069091BA
:10DE800059060F945C1A87FF22C0C092BD0ED09233
:10DE9000BE0EE092BF0EF092C00EE5EBFEE4849160
:10DEA0007F019FEFE91AF90A882321F00E94857FFC
:10DEB000F701F5CFECEEF6E184917F019FEFE91ACF
:10DEC000F90A882321F00E94857FF701F5CFC090E1
:10DED0004204D0904304E0904404F0904504209123
:10DEE000BD0E3091BE0E4091BF0E5091C00EC701C5
:10DEF000B6010F94BF1E20E030E048E453E40F94D5
:10DF0000E620181614F5C092BD0ED092BE0EE09217
:10DF1000BF0EF092C00EE5EBFEE484917F019FEF0F
:10DF2000E91AF90A882321F00E94857FF701F5CFCD
:10DF3000EDECF6E184917F019FEFE91AF90A88235D
:10DF400021F00E94857FF701F5CF209136043091B2
:10DF5000370440913804509139046091B10E7091AA
:10DF6000B20E8091B30E9091B40E0F945C1A811191
:10DF70001DC020913A0430913B0440913C045091E3
:10DF80003D046091B50E7091B60E8091B70E9091E0
:10DF9000B80E0F945C1A811109C060910A02709149
:10DFA0000B0280910C0290910D021AC06091A602A2
:10DFB0007091A702882777FD8095982F0F94621A99
:10DFC00020910A0230910B0240910C0250910D02F7
:10DFD0000F94C11A2AE037ED43E25CE30F94C11AB3
:10DFE000A7DEFF90EF90DF90CF900D94C401FF90DB
:10DFF000EF90DF90CF900895CF92DF92FF920F9332
:10E000001F93CF93DF931F921F92CDB7DEB76901A5
:10E01000DB0112960D911C911397423309F471C0E4
:10E02000B8F4453109F47AC0473109F48BC0443162
:10E0300009F0A1C0D80115962C9115971696ED916F
:10E04000FC911797CF01820F911D820F911D5EC029
:10E05000463409F487C0473409F488C04B3309F0CB
:10E060008AC0F90181819381913029F0933031F494
:10E07000282F885004C028E0280F01C0282F31E045
:10E08000D80113964C91481708F430E051E0F8019C
:10E090004281241708F450E041E0281708F040E0DE
:10E0A000832F842B85233423832B09F464C0D6016A
:10E0B0001296FC90913039F070F0923039F0933034
:10E0C00041F020E001C021E030E007C020E03FEF58
:10E0D00004C02FEFF9CF20E031E0F7FE08C0B60111
:10E0E000C8012A8339830F94430339812A81F601B9
:10E0F0008081830F80838181820F8183FF0C69F788
:10E100003AC0B901C8010F94430335C01192E81712
:10E11000F907E1F7C8010F946E032DC0C8010F94F1
:10E120005803882351F1F80125810680F781E02DFD
:10E13000CF01820F911D820F911D1192E817F907EF
:10E14000E1F719C0D9011C92F801828111968C93D4
:10E1500011978581815012968C9312978381139623
:10E160008C9309C0D80115968C9103C0D8011196E3
:10E170008C91F601808381E001C080E00F900F90C8
:10E18000DF91CF911F910F91FF90DF90CF90089575
:10E190006F927F928F929F92AF92BF92CF92DF92B7
:10E1A000EF92FF920F931F93CF93DF935C017B015C
:10E1B000942E69018AE0481709F466C0A5E14A1364
:10E1C00042C0DB011296ED91FC9113978280C681CB
:10E1D000D781A49A0F94750380EE782E780C90E185
:10E1E000692E680C88EF72D60F947503BFE1B815DD
:10E1F00008F43CC0882D8077806868D6882D829589
:10E20000807F64D60F94750380E860D680E05ED688
:10E210000F9475038AEF5AD60F9475038E01005F31
:10E220001F4F8881807F52D689918295807F4ED6FC
:10E230000C171D07B1F7E8010F94750383947394CD
:10E240008610D0CFA4989601492DB701C501DF9162
:10E25000CF911F910F91FF90EF90DF90CF90BF90E3
:10E26000AF909F908F907F906F90C6CE872D8077D4
:10E2700080682CD6872D8295807F28D60F947503D1
:10E2800080E824D680E8C3CF9C9AA4989B9AA39850
:10E29000809104018460809304019FB7F894809179
:10E2A00005018460809305019FBFA49A0F947503B4
:10E2B00088E790E00F947A0388EF08D60F947503EF
:10E2C00080E004D680E802D60F94750380E0FED586
:10E2D00080E1FCD50F9475038FE090E00F947A03F2
:10E2E00080E3F4D580EEF2D50F947503D0E08D2F46
:10E2F00080778068EBD58D2F8295807FE7D50F944E
:10E30000750380E8E3D580E0E1D50F9475038AEFCB
:10E31000DDD50F947503C0E280E0D8D580E0D6D576
:10E320000F947503C150C1F788EFD0D50F947503D2
:10E33000DF5FD032E1F680E0C9D580ECC7D50F941D
:10E340007503A49880CF10929E1110929D11109287
:10E35000A01110929F110E9453840C94E4E18F92BB
:10E360009F92BF92CF92DF92EF92FF920F931F93F3
:10E37000CF93DF931F92CDB7DEB74C01D62EE42E9C
:10E38000522FF22EC62EC20EBB24BA948C01045E0C
:10E390001F4F2C2D2F1987E08F1588F4F40162810F
:10E3A0007381248FE58E178EB68E98014BE3C401DE
:10E3B00059830F94A603F8EFFF0E5981EACF852FFA
:10E3C000887F8D0D577021F137E03527F401628188
:10E3D0007381848FE58E178E3F5F37708FEF90E0EB
:10E3E00001C0880F3A95EAF7868F9401245E3F4F6B
:10E3F0004BE3C4010F90DF91CF911F910F91FF90DC
:10E40000EF90DF90CF90BF909F908F900D94A603D8
:10E410000F90DF91CF911F910F91FF90EF90DF90C0
:10E42000CF90BF909F908F900895EF92FF920F939F
:10E430001F93CF93DF93EC01F62EE22E142F040FDF
:10E440002E2D412F6F2DCE018ADF1F5F0113F8CFD4
:10E45000DF91CF911F910F91FF90EF900895DF9280
:10E46000EF92FF920F931F93CF93DF93EC01162F40
:10E47000F42EE22E0F948403882329F02E2D4F2DA5
:10E48000612FCE01D2DFDF91CF911F910F91FF90CD
:10E49000EF90DF9008950F934CE0849F402D11245E
:10E4A000E1E0E40FE0935D082CE0240F20935E0888
:10E4B000A0910F12B0E030E02E5F3F4F2A173B07CC
:10E4C000FCF0F0E02091111230E0E217F307C4F401
:10E4D000662369F081E08093FB114D5F0BE020E83B
:10E4E00060E08BED91E1BBDF1092FB1103C081E096
:10E4F0008093FB1180915E08109212128093131288
:10E500000F910895EF92FF920F931F93CF93DF9394
:10E510001F92CDB7DEB7182F062F682F802F4983A3
:10E52000BADF90910F1280915E084981891708F433
:10E530005AC09091111280915D08981708F453C049
:10E540008091B712882309F44BC0112371F1602F19
:10E5500080E0E82FF0E0EB55FD4E9581992329F0FE
:10E56000660F611D69278F5FF4CF8091EB078617D7
:10E57000B1F0E7EBF2E120E030E08191882319F07F
:10E580002F5F3F4FFACF2531310514F0255101C0DF
:10E5900020E02093D8066093EB071092D9060091F3
:10E5A000D90610E009541D4E02C007EB12E14423C6
:10E5B00019F082E00E9485A7780115E1F7018191A9
:10E5C0007F01882331F0112321F00E9416C6181B09
:10E5D000F5CF112341F080E20E947AA71150F9CFC4
:10E5E0000AEA12E1E4CF0F90DF91CF911F910F91D2
:10E5F000FF90EF9008950F931F93CF93DF93982F81
:10E60000862FEA01022F692F46DF90910F12809129
:10E610005E08891750F19091111280915D0898174A
:10E6200020F114E1FE018491811102C0C12F05C0C7
:10E630000E9416C6181B2196F5CFCC2329F080E244
:10E640000E947AA7C150F9CF80915E089AE7909313
:10E65000121280931312802F0E9485A780E2DF910F
:10E66000CF911F910F910C947AA7DF91CF911F91B9
:10E670000F9108951F93CF93DF931092CA11809149
:10E68000C6119091C711A091C811B091C9118130E4
:10E690009048A105B10540F01092C6111092C71123
:10E6A0001092C8111092C911C091C6114091E9078A
:10E6B0001416D4F4842F992787FD909501972C2F59
:10E6C000332727FD30952817390774F0CFEFC40F93
:10E6D0008C2F90E0A0E0B0E08093C6119093C7111A
:10E6E000A093C811B093C9111092C4118091C311A5
:10E6F000C81714F4C093C3118091C311992787FDE3
:10E70000909504962C2F332727FD30958217930779
:10E7100024F48CEF8C0F8093C3111091C311D0E0BF
:10E7200011111AC08091C211811106C08091A802F6
:10E73000882309F48CC009C0C111F8CF0E94EAE116
:10E740008091C411882391F389C081E0C11180E0D8
:10E7500024E043E757E179C01130E9F48091C21118
:10E76000811106C08091A802882309F470C00BC0F3
:10E77000C130C1F781EA96EA0E94AFE18091C411ED
:10E78000882381F36BC081E0C13009F080E023E091
:10E790004CE657E15AC01230E9F48091C211811160
:10E7A00006C08091A802882309F451C00BC0C23072
:10E7B000C1F78DE996EA0E94AFE18091C4118823E8
:10E7C00081F34CC081E0C23009F080E023E045E6EF
:10E7D00057E13BC01330E1F48091C211811105C0B3
:10E7E0008091A802882399F10BC0C330C9F789E949
:10E7F00096EA0E94AFE18091C411882389F32EC06C
:10E8000081E0C33009F080E023E04EE557E11DC010
:10E810001430E9F48091C211811105C08091A802E1
:10E820008823A9F00BC0C430C9F785E996EA0E9495
:10E83000AFE18091C411882389F310C081E0C43016
:10E8400009F080E023E045E557E16D2FD4DEDF5F7E
:10E850001F5FD53009F064CFD093E907DF91CF91E6
:10E860001F910895DF92EF92FF920F931F93CF9322
:10E87000DF93CDB7DEB76E970FB6F894DEBF0FBE4D
:10E88000CDBF60913F09709140096115710511F18B
:10E890004DE150E08E010F5F1F4FC8010F94CD195D
:10E8A0001E8EF8017F01E01AF10AD190DD2019F0E7
:10E8B0008AE0D812F7CFF801EE0DFF1D108260E05C
:10E8C000C8010E948281882329F0C8010E9482D653
:10E8D000811109C081E020913F0930914009232B2B
:10E8E000A9F480E013C0DD2051F08FEFE81AF80A98
:10E8F00080913F09909140098E0D9F1D02C080E0DC
:10E9000090E09093400980933F09E4CF6E960FB654
:10E91000F894DEBF0FBECDBFDF91CF911F910F9155
:10E92000FF90EF90DF900895AF92BF92CF92DF9269
:10E93000EF92FF920F931F93CF93DF931092CA1120
:10E940008091C6119091C711A091C811B091C911C1
:10E9500081309048A105B10540F01092C611109287
:10E96000C7111092C8111092C911C091C6114091DF
:10E97000EA071416D4F4842F992787FD9095019700
:10E980002C2F332727FD30952817390774F0CFEF48
:10E99000C40F8C2F90E0A0E0B0E08093C61190935C
:10E9A000C711A093C811B093C9111092C4118091DE
:10E9B000C311C81714F4C093C3118091C3119927D0
:10E9C00087FD909504962C2F332727FD30958217CD
:10E9D000930724F48CEF8C0F8093C311D091C31153
:10E9E000B12C53EEC52E57E1D52E07E917E168EAA1
:10E9F000E62E67E1F62ED11119C08091C211811166
:10EA000005C08091A802882389F109C0C111F9CFFE
:10EA10000E94EAE18091C411882399F3B7C081E094
:10EA2000C11180E024E047EE57E11EC0D130F1F47F
:10EA30008091C211811105C08091A8028823B1F094
:10EA40000CC0C130C9F7D0924009C0923F090ADF1B
:10EA50008091C411882381F399C081E0C13009F00D
:10EA600080E020E249ED57E16B2DC5DD8091830602
:10EA7000811118C06091120270911302882777FDEE
:10EA80008095982F0F94621A9B01AC0160915606F5
:10EA90007091570680915806909159060F945C1A10
:10EAA00087FD22C0D23019F58091C211811106C0B4
:10EAB0008091A802882309F466C00CC0C230C1F757
:10EAC000F0924009E0923F09CDDE8091C411882385
:10EAD00079F35CC081E0C23009F080E020E24BE9CC
:10EAE00057E16B2D88DD4FC042E0A42E02C033E019
:10EAF000A32EDA111EC08091C211811105C0809130
:10EB0000A8028823A9F00CC0CD13F9CF10934009B7
:10EB100000933F09A7DE8091C411882381F336C09A
:10EB200081E0CD1380E020E246E857E16B2D63DD04
:10EB3000AD2E81E08A0DD8131CC08091C2118111C5
:10EB400005C08091A8028823A1F00BC0CD13F9CF96
:10EB50008AE393E70E94AFE18091C411882389F38F
:10EB600015C081E0CD1380E023E04CE757E16B2D29
:10EB700042DDB394DF5F85E0B8123DCFA394A39448
:10EB8000A092EA0703C023E0A22ED3CFDF91CF915A
:10EB90001F910F91FF90EF90DF90CF90BF90AF90BB
:10EBA0000895CF92DF92EF92FF920F931F93CF932E
:10EBB000DF93CDB7DEB7CDB6DEB6FC010190002005
:10EBC000E9F7E81BF90B34962DB73EB72E1B3F0B28
:10EBD0000FB6F8943EBF0FBE2DBF0DB71EB70F5F27
:10EBE0001F4F9F938F9385E497E19F938F931F937C
:10EBF0000F930F94F619780134E0E30EF11C0F9097
:10EC00000F900F900F900F900F90F7018081882345
:10EC100039F090E00F94B921F70181937F01F5CF8E
:10EC200060E0C8010E948281882319F0C8010E9417
:10EC300082D681E497E19093400980933F0912DEE8
:10EC40000FB6F894DEBE0FBECDBEDF91CF911F91FF
:10EC50000F91FF90EF90DF90CF9008957F928F9269
:10EC60009F92AF92BF92CF92DF92EF92FF920F935B
:10EC70001F93CF93DF93CDB7DEB7AA970FB6F89463
:10EC8000DEBF0FBECDBF8091FA128F938091F91233
:10EC90008F938CE497E19F938F938E010F5D1F4FAD
:10ECA0001F930F930F94F6190F900F900F900F90E2
:10ECB0000F900F90D12CF80101900020E9F73197C7
:10ECC000E01BF10BDE1674F47801ED0CF11CD7FC9F
:10ECD000FA94F701808190E00F94B921F7018083C5
:10ECE000D394E9CF40E050E0BA018FEF92E10E9467
:10ECF000D9AB912CCE0101967C0140E050E0B701E8
:10ED00008FEF92E10E9453AB18168CF5F70101903A
:10ED10000020E9F73197EE19FF09C12CD12C8E2E76
:10ED200077247A947E0E872D8C198C1481F05701EC
:10ED3000A80EB11C87FDBA94F501808190E00F9474
:10ED4000B921F5018083FFEFCF1ADF0AECCF8A8566
:10ED50008E3799F245E050E0B801C7010F940722C1
:10ED6000892B59F6C8011DDF99249394C6CF9110C1
:10ED700003C08FEF9FEF05C08091F9129091FA12B6
:10ED800001969093FA128093F912AA960FB6F8940E
:10ED9000DEBF0FBECDBFDF91CF911F910F91FF90CE
:10EDA000EF90DF90CF90BF90AF909F908F907F902B
:10EDB000089580919D0683FD18C08091830681117E
:10EDC00014C020917A0E30917B0E809112029091A6
:10EDD0001302281739074CF40E9456DF40E050E038
:10EDE000BA0183E09CE40C948CE181E080938A0674
:10EDF00040E050E0BA0183EE9AE40E948CE189E39E
:10EE000097E19093400980933F092CCD1092A7126F
:10EE10000E949DAF84E397E19093400980933F095E
:10EE200021DD6FEF87E297E10C94CBDE83E297E17F
:10EE30009093400980933F0915DD6FEF82E297E1DF
:10EE40000C94CBDE40E060E080915E0690915F061E
:10EE50000C94E184E0915E06F0915F068081882346
:10EE600029F0803209F410823196F8CF40E061E059
:10EE700080915E0690915F060C94E18480915E061D
:10EE800090915F0621E02093A61240E060E00C9490
:10EE9000E184CF93DF932FB7F89494E08902E001E7
:10EEA0001124FE01EB5CF14F6081718182819381BD
:10EEB0002FBF0F94621ACA53D14F288139814A81DA
:10EEC0005B810F94C11ADF91CF9108952FB7F89409
:10EED000909105019B7F909305012FBF87FD96C000
:10EEE000A3982FB7F8949091050194609093050131
:10EEF0002FBF880F2FB7F894909105019B7F9093B7
:10EF000005012FBF87FD8EC0A3982FB7F89490916D
:10EF100005019460909305012FBF880F2FB7F894D7
:10EF2000909105019B7F909305012FBF87FD78C0CD
:10EF3000A3982FB7F89490910501946090930501E0
:10EF40002FBF880F2FB7F894909105019B7F909366
:10EF500005012FBF87FD62C0A3982FB7F894909149
:10EF600005019460909305012FBF880F2FB7F89487
:10EF7000909105019B7F909305012FBF87FD4CC0A9
:10EF8000A3982FB7F8949091050194609093050190
:10EF90002FBF880F2FB7F894909105019B7F909316
:10EFA00005012FBF87FD36C0A3982FB7F894909125
:10EFB00005019460909305012FBF982F990F2FB7EB
:10EFC000F894809105018B7F809305012FBF97FDF9
:10EFD0001FC0A3982FB7F894809105018460809397
:10EFE00005012FBF2FB7F894809105018B7F809387
:10EFF00005012FBF96FD18C0A3989FB7F894809184
:10F0000005018460809305019FBF0895A39A69CF8D
:10F01000A39AE0CFA39AC9CFA39AB3CFA39A9DCFC7
:10F02000A39A87CFA39A71CFA39AE7CFFC0120E0E0
:10F030003EE2DB014C91403241F0283011F4308344
:10F040003196DB014C91408331962F5F6F5F7F4F8C
:10F050002B3079F710820895CF92DF92EF92FF92D2
:10F06000C0905A06D0905B06E0905C06F0905D067A
:10F070006091760E7091770E68507109882777FD40
:10F080008095982F0F94621A9B01AC01C701B601BD
:10F090000F945C1A87FF1DC020E030E040E050E490
:10F0A000C701B6010F94C01E0F94092070932F085A
:10F0B00060932E080F94A204605A75418F4F9F4FA2
:10F0C000609330087093310880933208909333082E
:10F0D00008C0109230081092310810923208109235
:10F0E0003308FF90EF90DF90CF900895CF92DF929A
:10F0F000EF92FF92C0905606D0905706E0905806C7
:10F10000F090590660917A0E70917B0E65517109ED
:10F11000882777FD8095982F0F94621A9B01AC0188
:10F12000C701B6010F945C1A87FF1DC020E030E0D4
:10F1300040E251E4C701B6010F94C01E0F940920AC
:10F1400070933508609334080F94A204605C734692
:10F150008F4F9F4F6093360870933708809338081D
:10F160009093390808C01092360810923708109210
:10F17000380810923908FF90EF90DF90CF900895F3
:10F180004F925F926F927F928F929F92AF92BF92B7
:10F19000CF92DF92EF92FF920F931F93CF93DF9363
:10F1A0002C0121ED3AE181E090E0F9014591549183
:10F1B000441655060CF062C0AC0141505109DA0109
:10F1C000AA0FBB1FAA0FBB1FA153B54EFD0165912E
:10F1D0007491440F551F440F551F4353554EFA0168
:10F1E00065907490FC01EE0FFF1FEE0FFF1FE153BF
:10F1F000F54EA590B490FD0105911491F901C591CA
:10F20000D491FA0185909490882777FD8095982F66
:10F210000F94621A6B017C01B20166197709882785
:10F2200077FD8095982F0F94621A2B013C01B50150
:10F23000601B710B882777FD8095982F0F94621AB9
:10F240009B01AC01C301B2010F94C11A2B013C0117
:10F25000BE0168197909882777FD8095982F0F944A
:10F26000621A9B01AC01C301B2010F949C1F9B0168
:10F27000AC01C701B6010F94C01E11C001962C5FEE
:10F280003F4F8A33910509F090CFE3EBFBE16591A5
:10F290007491882777FD8095982F0F94621ADF91DB
:10F2A000CF911F910F91FF90EF90DF90CF90BF9083
:10F2B000AF909F908F907F906F905F904F90089548
:10F2C0004F925F926F927F928F929F92AF92BF9276
:10F2D000CF92DF92EF92FF92CF93DF93CDB7DEB75D
:10F2E0002C970FB6F894DEBF0FBECDBF80915A06A3
:10F2F00090915B06A0915C06B0915D0689839A832C
:10F30000AB83BC836091760E7091770E882777FD72
:10F310008095982F0F94621A29813A814B815C81E4
:10F320000F94BF1E6B017C016093190870931A083B
:10F3300080931B0890931C0820917F0630918006D3
:10F3400040918106509182060F94C11A6D837E838D
:10F350008F83988760931508709316088093170819
:10F3600090931808209111083091120840911308C9
:10F3700050911408C701B6010F94C01E4B015C01E7
:10F3800060931108709312088093130890931408E7
:10F3900020917B0630917C0640917D0650917E063F
:10F3A0000F94C11A69877A878B879C8760930D08B1
:10F3B00070930E0880930F089093100820ED3CEC9A
:10F3C0004CE45DE360917706709178068091790650
:10F3D00090917A060F94C11A2B013C0120910908E3
:10F3E00030910A0840910B0850910C0869817A818C
:10F3F0008B819C810F94BF1E9B01AC01C301B201A4
:10F400000F94C11A2B013C0123E333E343E75FE38D
:10F41000609105087091060880910708909108088E
:10F420000F94C11A9B01AC01C301B2010F94C01E1D
:10F430002B013C0160930508709306088093070830
:10F440009093080889819A81AB81BC8180930908D7
:10F4500090930A08A0930B08B0930C0829853A856D
:10F460004B855C856D817E818F8198850F94C01E50
:10F47000A30192010F94BF1E2B013C0120E030E05C
:10F480004EE453E40F94E62020E030E0A901181682
:10F49000ACF4C701B6010F94E62018166CF5A7016D
:10F4A0009601C501B4010F94BF1E609311087093BB
:10F4B000120880931308909314081EC0C301B20170
:10F4C0000F945C1A87FF22C020E030E0A901C70139
:10F4D000B6010F945C1A87FF16C0A7019601C501FB
:10F4E000B4010F94BF1E60931108709312088093AB
:10F4F00013089093140807C0412C512C8EE4682EF9
:10F5000083E4782E03C0412C512C3201C301B20197
:10F510002C960FB6F894DEBF0FBECDBFDF91CF9112
:10F52000FF90EF90DF90CF90BF90AF909F908F9023
:10F530007F906F905F904F9008954F925F926F927F
:10F540007F928F929F92AF92BF92CF92DF92EF9273
:10F55000FF920F931F93CF93DF9300D01F92CDB7ED
:10F56000DEB700917A0E10917B0E80905606909037
:10F570005706A0905806B0905906B801882777FD25
:10F580008095982F0F94621AA50194010F94BF1EC5
:10F590006B017C016093010870930208809303085B
:10F5A0009093040820ED3CEC4CE45DE36091A310E3
:10F5B0007091A4108091A5109091A6100F94C11A7B
:10F5C0002B013C012091FD073091FE074091FF0780
:10F5D00050910008C501B4010F94BF1E9B01AC01FE
:10F5E000C301B2010F94C11A2B013C0123E333E3A1
:10F5F00043E75FE36091F9077091FA078091FB0799
:10F600009091FC070F94C11A9B01AC01C301B20198
:10F610000F94C01E69837A838B839C836093F90760
:10F620007093FA078093FB079093FC078092FD0785
:10F630009092FE07A092FF07B092000880918F067B
:10F64000882321F081E08093F807B9C020E030E002
:10F6500040E251E4C701B6010F94E620181624F4E5
:10F6600081E08093F807A4C020E030E040E251EC54
:10F67000C701B6010F945C1A87FDE4CF012B11F38B
:10F680008091F807882351F01092F4071092F50743
:10F690001092F6071092F7071092F8072091AB101E
:10F6A0003091AC104091AD105091AE10C701B60131
:10F6B0000F94C11A2B013C016093F0077093F1077E
:10F6C0008093F2079093F3072091F4073091F507A8
:10F6D0004091F6075091F707C701B6010F94C01E7D
:10F6E0004B015C016093F4077093F5078093F60774
:10F6F0009093F7072091A7103091A8104091A9107E
:10F700005091AA100F94C11A9B01AC016093EC07B1
:10F710007093ED078093EE079093EF07C301B2015A
:10F720000F94C01E29813A814B815C810F94BF1ECA
:10F730002B013C0120E030E04FE753E40F94E6203A
:10F7400020E030E0A9011816ACF4C701B6010F940F
:10F75000E62018166CF5A7019601C501B4010F94B7
:10F76000BF1E6093F4077093F5078093F60790939C
:10F77000F7071EC0C301B2010F945C1A87FF22C0B5
:10F7800020E030E0A901C701B6010F945C1A87FFA1
:10F7900016C0A7019601C501B4010F94BF1E609366
:10F7A000F4077093F5078093F6079093F70707C067
:10F7B000412C512C9FE7692E93E4792E03C0412CF4
:10F7C000512C3201C301B2010F900F900F900F9096
:10F7D000DF91CF911F910F91FF90EF90DF90CF902D
:10F7E000BF90AF909F908F907F906F905F904F9061
:10F7F000089560915A0670915B0680915C06909125
:10F800005D0608954F925F926F927F928F929F92C2
:10F81000AF92BF92CF92DF92EF92FF920F931F931E
:10F82000CF93DF932C0126E138E181E090E0F901EC
:10F8300045915491441655060CF062C0AC014150FC
:10F840005109DA01AA0FBB1FAA0FBB1FAC5EB74E4E
:10F85000FD0165917491440F551F440F551F4E5E75
:10F86000574EFA0165907490FC01EE0FFF1FEE0FEA
:10F87000FF1FEC5EF74EA590B490FD010591149129
:10F88000F901C591D491FA0185909490882777FD6C
:10F890008095982F0F94621A6B017C01B201661952
:10F8A0007709882777FD8095982F0F94621A2B018E
:10F8B0003C01B501601B710B882777FD8095982F5F
:10F8C0000F94621A9B01AC01C301B2010F94C11ADB
:10F8D0002B013C01BE0168197909882777FD8095C5
:10F8E000982F0F94621A9B01AC01C301B2010F94CF
:10F8F0009C1F9B01AC01C701B6010F94C01E11C033
:10F9000001962C5F3F4F8032910509F090CFE0E9DE
:10F91000F8E165917491882777FD8095982F0F9471
:10F92000621ADF91CF911F910F91FF90EF90DF90BE
:10F93000CF90BF90AF909F908F907F906F905F908F
:10F940004F90089560915606709157068091580621
:10F9500090915906089567FD5CC0823021F128F42A
:10F96000882349F0813069F054C0833071F18430CC
:10F9700009F43DC04EC0662311F0A19A8FC0A19832
:10F980008DC09FB7662329F0F894809108018068A4
:10F9900004C0F894809108018F77809308019FBF7D
:10F9A00047FF4CC07FC09FB7662329F0F894809131
:10F9B0000801806404C0F894809108018F7B8093D3
:10F9C00008019FBF47FF40C06FC09FB7662329F063
:10F9D000F89480910801886004C0F894809108012F
:10F9E000877F809308019FBF47FF3EC05AC09FB7E3
:10F9F000662329F0F89480910801826004C0F8948D
:10FA0000809108018D7F809308019FBF47FF39C017
:10FA10004AC047FD49C08230B9F028F4882341F03C
:10FA2000813061F008958330F9F0843051F1089508
:10FA3000442311F0A09A0895A0980895442311F04A
:10FA4000A29A0895A29808959FB7442329F0F894A4
:10FA500080910801806204C0F894809108018F7D34
:10FA6000809308019FBF08959FB7442329F0F8941D
:10FA7000809108018061F4CFF894809108018F7E15
:10FA8000EFCF9FB7442329F0F89480910801846058
:10FA9000E7CFF894809108018B7FE2CF47FFC8CF72
:10FAA00008950895089508950895643079F028F42C
:10FAB000613041F0623041F00895683051F06031BA
:10FAC00041F0089540E003C040E004C041E060E040
:10FAD00002C041E061E03FCF24E08202C001112476
:10FAE000FC01EB5CF14F4081518162817381FC012B
:10FAF000EA52F14F4083518362837383E091680E31
:10FB0000F091690E82899389A489B5898093450E05
:10FB10009093460EA093470EB093480E089580E050
:10FB2000B8D96093AF087093B0088093B1089093F0
:10FB3000B20881E0AED96093B3087093B4088093A3
:10FB4000B5089093B60882E0A4D96093B708709383
:10FB5000B8088093B9089093BA0808958091670E09
:10FB60009FB780FF09C0F89480910B018D7F80932F
:10FB70000B019FBF8FEF08C0F89480910B0182604A
:10FB800080930B019FBF81E0809343028091670EB9
:10FB90009FB781FF09C0F89480910B018160809329
:10FBA0000B019FBF8FEF08C0F89480910B018E7FEF
:10FBB00080930B019FBF81E0809344028091670E88
:10FBC0009FB782FF09C0F89480910B018B7F8093CF
:10FBD0000B019FBF8FEF08C0F89480910B018460E8
:10FBE00080930B019FBF81E0809345028091670E57
:10FBF0009FB783FF09C0F89480910B0180648093C4
:10FC00000B019FBF8FEF08C0F89480910B018F7B91
:10FC100080930B019FBF81E08093460208954F922D
:10FC20005F926F927F92AF92BF92CF92DF92EF92EC
:10FC3000FF920F931F93CF93DF938C01EB01FC0195
:10FC400047A050A461A472A4AFA0B8A4C9A4DAA428
:10FC50009501A601C301B2010F945C1A87FF40C051
:10FC6000A3019201C301B2010F94C11A2B013C01FF
:10FC7000F80183A994A9A5A9B6A9BC01CD01905802
:10FC80009B01AC010F94C01EF80127A530A941A922
:10FC900052A90F94C11A9B01AC01C301B2010F9488
:10FCA000BF1E0F942B217B018C019B01AC01B50180
:10FCB000C6010F945C1A87FF02C075018601970187
:10FCC000A801B501C6010F945C1A882349F0A70169
:10FCD000B8014FA358A769A77AA788818160888354
:10FCE000DF91CF911F910F91FF90EF90DF90CF9018
:10FCF000BF90AF907F906F905F904F9008958F92DC
:10FD00009F92AF92BF92CF92DF92EF92FF920F93AA
:10FD10001F93CF93DF9300D01F92CDB7DEB716EAC3
:10FD2000812E11E1912E09E6A02E08E0B02E0CE7FD
:10FD300011E1C12CD12C7601C394F4016191719130
:10FD4000819191914F01F501219131914191519111
:10FD50005F0129833A834B835C830F94601A298166
:10FD60003A814B815C810F94C11A0F940920F801EC
:10FD700061937193819391938F01C616D706E8061C
:10FD8000F90610F46B017C01F6EB8F16F1E19F068A
:10FD9000A1F66FEF7FEFCB01A70196010F94621ED2
:10FDA0002093C7063093C8064093C9065093CA06ED
:10FDB0000F900F900F900F90DF91CF911F910F91A7
:10FDC000FF90EF90DF90CF90BF90AF909F908F907B
:10FDD000089561E0FC0180810D946D048EBD0DB429
:10FDE00007FEFDCF08958FEF8EBD0DB407FEFDCF4A
:10FDF0008EB508950F931F93CF93DF93EB010F946C
:10FE0000A2048B01F0DF8F3F49F00F94A204601B26
:10FE1000710B6C177D07B0F380E001C081E0DF91CA
:10FE2000CF911F910F910895CF92DF92FF920F9380
:10FE30001F93CF93DF9300D01F92CDB7DEB76C0135
:10FE4000F62EFC018281982F906A96959CBD80FDCC
:10FE500006C091E0863009F490E0892F01C080E06F
:10FE60008DBD60E0F601808129833A834B835C83FA
:10FE70000F946D046CE271E0C601BCDF8F2D8064CD
:10FE8000ADDF08E110E05C814B813A812981DA0124
:10FE9000C901002E04C0B695A795979587950A9439
:10FEA000D2F729833A834B835C8398DF085011098A
:10FEB00029813A814B815C81083FFFEF1F0739F7A9
:10FEC000FF2029F088E0F81621F08FEF03C085E9C4
:10FED00001C087E883DFECE0FE1201C084DF10E0A0
:10FEE00082DFF601838387FF04C01F3F11F01F5F8D
:10FEF000F7CF0F900F900F900F90DF91CF911F9140
:10FF00000F91FF90DF90CF9008959091C00095FFE2
:10FF1000FCCF8093C6000895EF92FF921F93CF937A
:10FF2000DF931F92CDB7DEB7182FE5ECFAE184918D
:10FF30007F012FEFE21AF20A882329F09983E5DF87
:10FF4000F7019981F4CFE12FF92F84917F019FEF81
:10FF5000E91AF90A882319F0D8DFF701F6CFECEA9D
:10FF6000FAE184917F01AFEFEA1AFA0A882319F0C7
:10FF7000CCDFF701F6CF0F90DF91CF911F91FF906B
:10FF8000EF900895DF92EF92FF920F931F93CF931C
:10FF9000DF9383E50F94ED02882319F00F94C300DB
:10FFA00001C080E080939D06E5EBFEE48491EF01C3
:10FFB0002196882319F0A9DFFE01F8CFE5EAFAE1DE
:10FFC0008491EF012196882319F09FDFFE01F8CF7D
:10FFD00080919D06882371F107E91AE1C0E0D0E025
:10FFE00020E080919D0690E00C2E02C095958795AB
:10FFF0000A94E2F780FF15C0DD24D394D20E2223A9
:020000021000EC
:1000000011F08CE282DFF80125913491F90184919D
:100010007901FFEFEF1AFF0A882321F076DF9701BD
:10002000F5CFD22E21960E5F1F4FC530D10561F05E
:100030002D2DD7CFE1EAFAE18491EF0121968823B3
:1000400019F063DFFE01F8CF8AE0DF91CF911F91B5
:100050000F91FF90EF90DF9058CFCF93DF9383E520
:100060000F94ED02882319F00F94B30002C060E0F2
:1000700070E0EB01DD27C230D105A8F0EEE7FEE429
:100080008491EF012196882319F03FDFFE01F8CF1C
:10009000E5E7FAE18491EF012196882309F44DC048
:1000A00034DFFE01F7CF88E40F94ED028823A9F036
:1000B0000F94B300683771053CF0633281E0780734
:1000C0002CF062E271E002C068E770E0FE01EE0F22
:1000D000FF1FEB56FE4E7183608386E40F94ED02A2
:1000E000882399F00F94B3006F3F710519F014F055
:1000F0006FEF70E0FE01EE0FFF1FE357FE4E77FF3C
:1001000002C060E070E07183608382E40F94ED02CE
:10011000882399F00F94B3006530710534F0683886
:1001200071052CF067E870E002C065E070E0CC0F6C
:10013000DD1FCF56DE4E79836883DF91CF9108951E
:10014000CF93DF93E0E8F9E18491EF0121968823D2
:1001500019F0DBDEFE01F8CFE2E7F9E18491EF016F
:100160002196882319F0D1DEFE01F8CFEBE5F9E105
:100170008491EF012196882319F0C7DEFE01F8CFA4
:10018000EBE4F9E18491EF012196882319F0BDDEBB
:10019000FE01F8CFEAE3F9E18491EF01219688238B
:1001A00019F0B3DEFE01F8CFE9E2F9E18491EF0145
:1001B0002196882319F0A9DEFE01F8CFEAE1F9E1E2
:1001C0008491EF012196882319F09FDEFE01F8CF7C
:1001D000E5E0F9E18491EF012196882319F095DE9D
:1001E000FE01F8CFEFEEF8E18491EF01219688232C
:1001F00019F08BDEFE01F8CFEAEDF8E18491EF0112
:100200002196882319F081DEFE01F8CFEDEBF8E1AD
:100210008491EF012196882319F077DEFE01F8CF53
:10022000E5EAF8E18491EF012196882319F06DDE6B
:10023000FE01F8CFDF91CF910895CF93DF9385E44E
:100240000F944D02882371F00F94D400882351F04D
:10025000E5EBFEE48491EF012196882319F055DE49
:10026000FE01F8CF81E40F944D02882371F00F94C2
:10027000D400882351F0E1EAF8E18491EF0121965E
:10028000882319F042DEFE01F8CFC0915E06D091BE
:100290005F068991882311F038DEFBCF8AE0DF9179
:1002A000CF9133CECF93DF93EEE7FEE48491EF015D
:1002B0002196882319F029DEFE01F8CFE2E9F8E162
:1002C0008491EF012196882319F01FDEFE01F8CFFB
:1002D000DF91CF9108953FB7F89420913E09809126
:1002E0003D09821759F0E22FF0E0E354F74F808187
:1002F00090E02F5F2F7720933E0902C08FEF9FEF92
:100300003FBF0895CF93FC01C62F80818B33A1F0AE
:1003100080916410843080F42091B01030E6239FE7
:10032000C0011124BF018D51914F0F9400228C2FD9
:100330000F94380281E001C080E0CF910895CF9200
:10034000DF92EF92FF921F93CF93DF9300D01F9223
:10035000CDB7DEB78091C6119091C711A091C81199
:10036000B091C911B7FF08C01092C6111092C71101
:100370001092C8111092C91180917A0890917B084F
:10038000A0917C08B0917D084091C6115091C71191
:100390006091C8117091C91184179507A607B70716
:1003A00044F48093C6119093C711A093C811B093E1
:1003B000C9118091A802882359F16091C6117091EA
:1003C000C7118091C8119091C911C0907E08D0903A
:1003D0007F08E0908008F09081086C0D7D1D8E1DD7
:1003E0009F1D0F94601A20E030E048EC52E40F9417
:1003F000C11A69837A838B839C83CE0101960E9404
:10040000D8D7BC0180918408909185080E94B08C57
:100410008091C21110911D08811106C01123C1F1F4
:100420008091A8028823A1F16091C6117091C71133
:100430008091C8119091C911C0907E08D0907F081A
:10044000E0908008F09081086C0D7D1D8E1D9F1D31
:100450000F94601A20E030E048EC52E40F94C11A87
:100460000F940920E0918208F0918308309721F0E1
:100470006083718382839383112329F0E0911E08A6
:10048000F0911F0819958091C21181110E94EAE133
:100490008091C211882329F0E0911E08F0911F0875
:1004A00019950F900F900F900F90DF91CF911F91A2
:1004B000FF90EF90DF90CF900895CF92DF92EF9270
:1004C000FF921F93CF93DF9300D01F92CDB7DEB77B
:1004D0008091C6119091C711A091C811B091C91116
:1004E000B7FF08C01092C6111092C7111092C81120
:1004F0001092C91180917A0890917B08A0917C0894
:10050000B0917D084091C6115091C7116091C811FA
:100510007091C91184179507A607B70744F4809313
:10052000C6119093C711A093C811B093C9118091BF
:10053000A802882359F16091C6117091C71180916A
:10054000C8119091C911C0907E08D0907F08E090AA
:100550008008F09081086C0D7D1D8E1D9F1D0F94ED
:10056000621A2AE037ED43E25CE30F94C11A698313
:100570007A838B839C83CE0101960E94A2D6BC0114
:1005800080918408909185080E94B08C8091C2115E
:1005900010911D08811106C01123B1F18091A802AC
:1005A000882391F16091C6117091C7118091C81193
:1005B0009091C911C0907E08D0907F08E09080088B
:1005C000F09081086C0D7D1D8E1D9F1D0F94621A89
:1005D0002AE037ED43E25CE30F94C11AE091820810
:1005E000F0918308309721F0608371838283938335
:1005F000112329F0E0911E08F0911F0819958091B0
:10060000C21181110E94EAE18091C211882329F070
:10061000E0911E08F0911F0819950F900F900F9010
:100620000F90DF91CF911F91FF90EF90DF90CF90CF
:100630000895CF92DF92EF92FF921F93CF93DF93B3
:1006400000D01F92CDB7DEB78091C6119091C7112F
:10065000A091C811B091C911B7FF08C01092C6117E
:100660001092C7111092C8111092C91180917A0886
:1006700090917B08A0917C08B0917D084091C611B3
:100680005091C7116091C8117091C91184179507D5
:10069000A607B70744F48093C6119093C711A0939F
:1006A000C811B093C9118091A802882359F16091B3
:1006B000C6117091C7118091C8119091C911C09055
:1006C0007E08D0907F08E0908008F09081086C0D43
:1006D0007D1D8E1D9F1D0F94621A2AE037ED43E2A7
:1006E0005CE30F94C11A69837A838B839C83CE0168
:1006F00001960E9457D7BC0180918408909185088B
:100700000E94B08C8091C21110911D08811106C009
:100710001123B1F18091A802882391F16091C61153
:100720007091C7118091C8119091C911C0907E0835
:10073000D0907F08E0908008F09081086C0D7D1DBE
:100740008E1D9F1D0F94621A2AE037ED43E25CE391
:100750000F94C11AE0918208F0918308309721F03C
:100760006083718382839383112329F0E0911E08B3
:10077000F0911F0819958091C21181110E94EAE140
:100780000F900F900F900F90DF91CF911F91FF90DE
:10079000EF90DF90CF900895CF92DF92EF92FF928B
:1007A0000F931F93CF9380917D128150823010F070
:1007B000C0E070C010927D120F94A2046093861264
:1007C00070938712809388129093891280918C1273
:1007D00090918D12019690938D1280938C12C090FF
:1007E000A012D090A112E090A212F090A3128DE777
:1007F00092E10E9461D96093A0127093A11280933C
:10080000A2129093A31200918E1210918F12209138
:100810009012309191120C191D092E093F09060FF3
:10082000171F281F391F00938E1210938F122093C9
:100830009012309391128DE792E10E9461D9C0909D
:100840009212D0909312E0909412F0909512C616E6
:10085000D706E806F90660F48DE792E10E9461D9B7
:1008600060939212709393128093941290939512C6
:10087000C091A412CC2369F060919A1270919B12DE
:100880006F5F7F4F40E150E08AE892E10F942A1DAC
:1008900001C0C1E08C2FCF911F910F91FF90EF907D
:1008A000DF90CF90089510927B0E10927A0E80E028
:1008B0000E9476781092770E1092760E0E942C7815
:1008C0006BDF10927B0E10927A0E80E00E94767899
:1008D0001092900E9FB7F894E2E0F1E080818F7B58
:1008E00080839FBF1092770E1092760E10928E0E1C
:1008F00075980895EC01EEE7FEE484918F010F5F97
:100900001F4F882319F001DBF801F7CFE1EDFBE180
:1009100084918F010F5F1F4F882319F0F6DAF801D9
:10092000F7CFC1DF0F9416010E94719261E0CE01F2
:100930000E94CBDE0E94E4E10E943F5684E00E94C8
:1009400062A78091DC118695869510921212809391
:1009500013120E9497A78091DC1186958695880FC7
:10096000109212128093131282EC9BE10E942EC609
:100970008091DC1186958695982F990F980F10928B
:1009800012129093131285EB9BE10E942EC60E94D7
:10099000DCC58111D3CF2FEF8BE49DE12150804046
:1009A0009040E1F700C00000F8942FEF84E39CE052
:1009B000215080409040E1F700C0000074DFA8950E
:1009C000FECF6F927F928F929F92AF92BF92DF92F3
:1009D000EF92FF920F931F93CF93DF93CDB7DEB7C4
:1009E000AD970FB6F894DEBF0FBECDBF7C01D62EFB
:1009F0008091A812882309F4E5C180919C14882372
:100A000009F498C0442309F4B5C18091B414882333
:100A100009F1EEE7FEE484918F010F5F1F4F8823F9
:100A200019F073DAF801F7CFE4E5FDE184918F0165
:100A30000F5F1F4F882319F068DAF801F7CF61E0E4
:100A400070E080E090E00E9485C28AE05EDA8BE48C
:100A50009DE150DF8FE28093B914B12C21E00AEBC5
:100A600014E19FE1A92E80917114B816B8F4AB9CE3
:100A7000C0011124B801815C9C4E2DA70E94F6553F
:100A8000C8012DA58C010196F8013081332321F096
:100A90002D3810F42F5FF6CFB394E5CF27FD06C0B5
:100AA000B80189E994E10E94F65502C0F80110826C
:100AB000E5EBFEE484918F010F5F1F4F882319F04F
:100AC00024DAF801F7CFB70182E39DE10E945AD6FC
:100AD0006091B414FDE86F9FB001112467547B4E00
:100AE00087E29DE10E945AD640914A1550914B15DC
:100AF00060914C1570914D1581E29DE10E944BEC87
:100B00008AE003DA8091B41494E0899FF001112403
:100B1000EB54FB4E40914A1550914B1560914C158A
:100B200070914D1540835183628373838F5F8093EF
:100B3000B4140CC01092B41482E0B82E1DC1B701D9
:100B400084E19DE10E945AD68AE0DFD90E94FE51DD
:100B50001D8218861C821B8284E293E09A8389831B
:100B60008BEF92E190931B1380931A13F70180810E
:100B70008F3209F069C087010F5F1F4FCE010196C8
:100B80003C010115110509F465C06FE270E0C80170
:100B90000F94F5215C01009709F45DC0081719074F
:100BA00008F059C04C01801A910AA401B801CE0185
:100BB00080960F941522E0E2F0E0EC0FFD1FE80DA7
:100BC000F91D10828E01005E1F4FF80181918F0187
:100BD000882311F09AD9F9CF8AE097D960911A1336
:100BE00070911B136115710519F06C5F7F4F02C086
:100BF00060E070E021E0AE01405E5F4FCE010596FF
:100C00000E945553811118C0E0E0FDE184918F01ED
:100C10000F5F1F4F811104C08E01005E1F4F03C084
:100C200074D9F801F3CFF80181918F01882311F075
:100C30006CD9F9CF8EE289C070921B1360921A139F
:100C400085010F5F1F4F9DCF8CE193E190931B13A4
:100C500080931A13870160911A1370911B13DD2082
:100C600009F45BC06115710519F06C5F7F4F02C01C
:100C700060E070E021E0A80189E994E10E94555309
:100C8000882309F446C08091AA149091AB14A091D6
:100C9000AC14B091AD148093461590934715A09372
:100CA0004815B0934915B80182EF9CE10E945AD6CD
:100CB000409146155091471560914815709149151E
:100CC0008AEE9CE10E944BEC8AE01FD910924A15F3
:100CD00010924B1510924C1510924D15EBEDFCE156
:100CE00084917F019FEFE91AF90A882319F00DD941
:100CF000F701F6CFB80180E090E00E94599480910E
:100D0000B712811102C0C80102C087EB92E160E016
:100D10002AC0B80187EC9CE113C06115710519F078
:100D20006C5F7F4F02C060E070E026E5A80189E9B2
:100D300094E10E94555381110AC0B80183EB9CE1F4
:100D40000E945AD68EE2E1D88AE0DFD80EC081E058
:100D50008093A512B70181EA9CE10E945AD68AE0ED
:100D6000D4D860E0C8010E94BBDECE0101960E948B
:100D70004A5428C0BB24B394E5EBFEE484918F0170
:100D80000F5F1F4F882319F0C0D8F801F7CFECE1AF
:100D9000FDE184918F010F5F1F4F882319F0B5D8B3
:100DA000F801F7CFE1E0BE1203C006E413E002C091
:100DB00000E413E0F80181918F01882309F4BFCE8C
:100DC000A4D8F8CFAD960FB6F894DEBF0FBECDBF56
:100DD000DF91CF911F910F91FF90EF90DF90BF9027
:100DE000AF909F908F907F906F90089560E080917A
:100DF0007C0E90917D0E0E94027C6093560670934B
:100E0000570680935806909359068091780E9091DA
:100E1000790E0E94C07860935A0670935B068093A7
:100E20005C0690935D06A8958FB7F89410927E0E9D
:100E30008FBF0895CF92DF92FF920F931F93CF93AE
:100E4000DF931F921F92CDB7DEB7F82E6A01809113
:100E50001402882309F43CC0EEE7FEE484918F017C
:100E60000F5F1F4F882339F069837A834ED8F801CA
:100E700069817A81F3CFFB0184918F010F5F1F4F4E
:100E8000882319F042D8F801F7CFE6EFFBE184910F
:100E90008F010F5F1F4F882319F037D8F801F7CF64
:100EA000F7FC0BC06F2D772767FD7095872F972F65
:100EB0000E9485C28AE029D80BC0E1EFFBE1849152
:100EC0008F010F5F1F4F882319F01FD8F801F7CF4C
:100ED00080912008811107C01092140281E0809354
:100EE0002008C60107DD0F900F90DF91CF911F9171
:100EF0000F91FF90DF90CF90D6CC2F923F924F92E0
:100F00005F926F927F928F929F92AF92BF92CF9299
:100F1000DF92EF92FF920F931F93CF93DF9300D056
:100F20001F92CDB7DEB74C011B0129833A834B8357
:100F30005C8327013801D7FE12C08091A106882367
:100F400009F4A7C0F4011082109225081092260817
:100F5000109227081092280801E010E015C0F60151
:100F6000E157F94F8081882309F4BEC0F401108253
:100F7000F601EE0FFF1FEE0FFF1FEF5DF74F108220
:100F80001182128213828601F40180818230E1F0A5
:100F9000833009F455C0813009F0A8C0F801EE0F84
:100FA000FF1FEE0FFF1FEF5DF74F20813181428160
:100FB000538169817A818B819C810F945C1A87FDB2
:100FC00095C082E0F4018083000F111F000F111FF4
:100FD0000F5D174FB501882777FD8095982F0F94E7
:100FE000621A9B01AC01F801608171818281938159
:100FF0000F94BF1E9B01AC0169817A818B819C811A
:101000000F94E62087FD0CC00F94A2046856754C1F
:101010008F4F9F4FF101608371838283938366C0FA
:101020000F94A204F1010081118122813381601BA0
:10103000710B820B930B97FD59C083E0F401808301
:10104000FFEFCF16DF0631F0C114D10431F44BE4C9
:101050005CE105C044E15CE102C048E35CE168E2B8
:101060007CE18C2D0F900F900F900F90DF91CF911E
:101070001F910F91FF90EF90DF90CF90BF90AF90B6
:101080009F908F907F906F905F904F903F902F90A8
:10109000D1CE01E010E07801EE0CFF1CEE0CFF1C3D
:1010A000C7018F5D974F7C01A3019201FC01608114
:1010B0007181828193810F945C1A882309F464CF33
:1010C000F7014082518262827382FF24F39420E010
:1010D00030E0A901C301B2010F94E62018160CF00C
:1010E000F12CF401F08250CF8601D5CF0F900F90F4
:1010F0000F900F90DF91CF911F910F91FF90EF9084
:10110000DF90CF90BF90AF909F908F907F906F9027
:101110005F904F903F902F9008958F3F29F081115D
:1011200006C04BEE5BE405C048EB5BE402C04BED50
:101130005BE469EC7BE47ECE8F3F29F0811106C031
:101140004EE25CE405C04BEF5BE402C04EE15CE4C0
:101150006CE07CE46FCE4F925F926F927F92AF9281
:10116000BF92CF92DF92EF92FF920F931F93CF9394
:10117000DF9300D01F92CDB7DEB780917E0E811134
:1011800013C00F900F900F900F90DF91CF911F9190
:101190000F91FF90EF90DF90CF90BF90AF907F9036
:1011A0006F905F904F90089521DE0F94A2046983A1
:1011B0007A838B839C838091290290912A0218164E
:1011C00019060CF026C1019790932A0280932902F8
:1011D00040905606509057066090580670905906F9
:1011E00080918F06811119C080918B0690918C0699
:1011F000A0918D06B0918E060097A105B10569F00A
:1012000029813A814B815C81281B390B4A0B5B0B8E
:1012100057FD03C081E080938F0660917A0E709134
:101220007B0E882777FD8095982F0F94621A1EE118
:10123000A12EB12CC12CD12C7B018C01A3019201D8
:101240006BE378E08AE398E058DE409056065090D1
:101250005706609058067090590660919D0E7091E7
:101260009E0E882777FD8095982F0F94621A9B0118
:10127000AC01C301B2010F94E6201816D4F46091BA
:10128000500270915102882777FD8095982F0F9416
:10129000621A9B01AC01C301B2010F945C1A87FF73
:1012A00008C080E00E949D7A0F9404207595679590
:1012B00001C060E06093900E8091360890913708ED
:1012C000A0913808B09139080097A105B10521F126
:1012D00029813A814B815C81281B390B4A0B5B0BBE
:1012E00057FD1AC00E94A27C2B013C01609134087A
:1012F0007091350880E090E00F94601A9B01AC017A
:10130000C301B2010F945C1A87FFA5C04FE85CE1EE
:1013100060E87CE180E08EDD8091300890913108BA
:10132000A0913208B09133080097A105B10521F1D1
:1013300029813A814B815C81281B390B4A0B5B0B5D
:1013400057FD1AC00E94F97B2B013C0160912E08C9
:1013500070912F0880E090E00F94601A9B01AC011F
:10136000C301B2010F945C1A87FF72C04EE55CE1C5
:1013700061E77CE18FEF5EDD6091760E7091770E14
:10138000882777FD8095982F0F94621A20915A062E
:1013900030915B0640915C0650915D06FAE0AF2EFD
:1013A000B12CCC24CA94DC2C7B018C0169E278E05E
:1013B0008DE298E0A2DD8091A106811127C04090C6
:1013C0005A0650905B0660905C0670905D0620E0C7
:1013D00030E040EA50E4C301B2010F94E62087FFF9
:1013E00004C060E060938E0ECCCE20E030E046E199
:1013F00053E4C301B2010F945C1A181694F30E94CF
:1014000060790F94042075956795ECCF10928E0E3D
:10141000B8CE40905606509057066090580670908F
:10142000590620E030E848E953E4C301B2010F94C3
:10143000E6201816A4F020E030E040EA50E4C301B2
:10144000B2010F945C1A87FFCBCE80E066DEC0CE7F
:101450000E942C7891CF80E00E9476785DCF80E06A
:101460006BDE40905606509057066090580670907C
:101470005906E1CF0F931F93CF93DF93EC018B01BC
:1014800060916B1240916C12641306C08FE592E17B
:101490000E948B5560DEF4CF28813981F80180816C
:1014A000918150916A1274E0579FF0011124ED5917
:1014B000FD4E33872287958784876F5F60936B1219
:1014C00081E0850F841719F080936A1202C0109290
:1014D0006A12DF91CF911F910F9108950F931F937F
:1014E000CF93DF93CDB7DEB728970FB6F894DEBF62
:1014F0000FBECDBF8823C1F083E992E098878F8328
:1015000004E610E01A830983BE01695F7F4FCE01B4
:101510000196B0DF8AEB92E09E838D831A83098364
:10152000BE016B5F7F4F0BC088EB91E09C838B8388
:1015300084E190E09A838983BE016D5F7F4FCE0185
:10154000019698DF28960FB6F894DEBF0FBECDBF88
:10155000DF91CF911F910F9108950E9468ECBECF4B
:10156000AF92BF92CF92DF92FF920F931F93CF93D0
:10157000DF9300D01F92CDB7DEB7F82E662351F06F
:101580001092430810923F081092400810924108B0
:10159000109242080F94A20400913F081091400855
:1015A00020914108309142085B016C01A01AB10AF8
:1015B000C20AD30AD7FC3DC0F7FE05C004EC19E00F
:1015C00020E030E015C0E09143082F2D332727FDA0
:1015D00030952C5F3F4F4E2F552747FD50952417D0
:1015E00035073CF1EF1554F300E911E020E030E05D
:1015F000DC01CB01800F911FA21FB31F80933F0816
:1016000090934008A0934108B093420880ED97E082
:101610009C838B838CE291E09A838983BE016D5F0A
:101620007F4FCE01019626DF809143088F5F809324
:1016300043080F900F900F900F90DF91CF911F9163
:101640000F91FF90DF90CF90BF90AF900895CF9310
:10165000DF9300D01F92CDB7DEB783E50F94ED0284
:10166000882319F00F94B30002C064E071E07C831A
:101670006B8380E50F94ED02882339F00F94B3005B
:10168000693823E1720730F402C068EE73E07A83B0
:10169000698304C088E893E19A838983BE016D5F02
:1016A0007F4FCE010196E6DE0F900F900F900F90C6
:1016B000DF91CF910895CF92DF92EF92FF926B016D
:1016C0007C0183E3C816D104E104F10468F082E3ED
:1016D000C81AD108E108F10862E370E080E090E008
:1016E0000F940F0438DDEDCFC701B6010F940F043E
:1016F000FF90EF90DF90CF902ECD5F926F927F9210
:101700008F929F92AF92BF92CF92DF92EF92FF9211
:101710000F931F93CF93DF93EC01C62ED42EB22EDE
:10172000EC80FD80C7010F943703182F8C819D81B9
:101730000F943A03982E113011F00FEF01C00FE013
:101740008C819D810F942F03182F8C819D810F9484
:101750002B03A82E8C819D810F94330320E62B153B
:1017600030F4009721F0E80EF91E11E610C08C81CC
:101770009D810F943503E0E4EB1530F4009721F0E0
:10178000E80EF91E11E403C0F1E1EF0EF11CAB14F9
:1017900030F4188A1B8A1C8A198A1A8A99C0A116E1
:1017A000C0F3A92DB0E0F70184918F3F21F4FFEF42
:1017B000EF1AFF0A3FC01B1135C08C819D810F9429
:1017C000370397012F5F3F4FF701882311F08230D5
:1017D00091F484918B8BF90124912C8BF701339632
:1017E000E491E88BF7013496E491E98BF7013596A3
:1017F000E491EA8B24C09491892F8F7082508A8B58
:1018000092959F70998BF9012491822F8F708C8B08
:1018100022952F702B8BF7013296E491E295EF70B1
:10182000E88B0DC0F7013296E491E023EE0EF11C37
:10183000EA0EFB1E1A1509F4ACCF1F5FB4CFE114FA
:10184000F10409F445C08C819D810F943A03A82EC0
:101850006B88BC8879887C0C9A899B0D1D2D191B7F
:101860000B2D262D412F672DCE010F948403882345
:1018700069F1EA0CF11CF7E06F0E669466946694C9
:10188000512E5B0C5E012CE1A20EB11C862C912C1A
:101890001515E1F0072D67018C2D8E19861590F432
:1018A000F60184916A817B810C8F1D8F1F8E8E8F34
:1018B00095014BE3CE010F94A603FFEFCF1ADF0A89
:1018C000085FEACFE80CF91C1F5FE2CF888901C0EE
:1018D00080E0DF91CF911F910F91FF90EF90DF900B
:1018E000CF90BF90AF909F908F907F906F905F90C0
:1018F0000895CF92DF92EF92FF920F931F93CF93B1
:10190000DF931F92CDB7DEB76C01DC01DC96EC9063
:10191000DC97DB96FC90DB978C010C5F1F4F599690
:10192000ED91FC915A97C80169831995482F4E0D86
:1019300029816F2DC801E1DEF60123AD992787FDCE
:101940009095820F911D83AF81E090E00F90DF9121
:10195000CF911F910F91FF90EF90DF90CF9008955E
:10196000BF92CF92DF92EF92FF920F931F93CF938C
:10197000DF937C018B0120E030E0F701E20FF31FE1
:10198000E491EE2319F02F5F3F4FF7CFF801CF011D
:10199000801B910B41914111FACFC4E1D0E0C81BEB
:1019A000D1093327C217D3071CF492E0C92E02C015
:1019B000CC24C3948091DC1190E06C2D70E06F5FBB
:1019C0007F4F0F949C21B62E86E0D82ED60E8091A4
:1019D0000F12D81650F08091111290E02D2D30E0AA
:1019E0002B5031098217930794F5F12C011511053D
:1019F000C1F18AE30E947AA782E0C8120FC0DB0C13
:101A000080910F12D81668F12091111230E08D2DBF
:101A100090E00B97281739071CF423C0FF2009F129
:101A20008C2F880F8C0F880F80931212D092131274
:101A300080E20E947AA7C801DF91CF911F910F9198
:101A4000FF90EF90DF90CF90BF900C943CC6109227
:101A50001212D0921312C7010E942EC6FF24F394D3
:101A6000C5CFDF91CF911F910F91FF90EF90DF9045
:101A7000CF90BF900895CF92DF92EF92FF921F9385
:101A8000CF93DF9300D01F92CDB7DEB78091C61100
:101A90009091C711A091C811B091C911B7FF08C0AA
:101AA0001092C6111092C7111092C8111092C9114C
:101AB00080917A0890917B08A0917C08B0917D0874
:101AC0004091C6115091C7116091C8117091C91110
:101AD00084179507A607B70744F48093C61190931F
:101AE000C711A093C811B093C9118091A80288238F
:101AF00051F16091C6117091C7118091C8119091F8
:101B0000C911C0907E08D0907F08E0908008F090C6
:101B100081086C0D7D1D8E1D9F1D0F94621A20E0A3
:101B200030E048EC52E40F94C11A69837A838B83C6
:101B30009C83CE0101960E94D8D7BC018091840875
:101B4000909185080DDF8091C21110911D088111BF
:101B500006C01123B1F18091A802882391F1609110
:101B6000C6117091C7118091C8119091C911C09090
:101B70007E08D0907F08E0908008F09081086C0D7E
:101B80007D1D8E1D9F1D0F94621A20E030E048ECF1
:101B900052E40F94C11AE0918208F09183083097C3
:101BA00021F06083718382839383112329F0E09174
:101BB0001E08F0911F0819958091C21181110E9491
:101BC000EAE10F900F900F900F90DF91CF911F914E
:101BD000FF90EF90DF90CF9008950F931F93CF93D6
:101BE0008091C6119091C711A091C811B091C911EF
:101BF000B7FF08C01092C6111092C7111092C811F9
:101C00001092C91180917A0890917B08A0917C086C
